:10000000086E0120790F0000750F0000750F0000C9
:10001000750F0000750F0000750F00000000000054
:10002000000000000000000000000000750F00004C
:10003000750F000000000000750F0000750F000034
:10004000750F0000750F0000750F0000750F0000A0
:10005000750F0000750F0000750F0000750F000090
:10006000750F0000750F0000750F0000750F000080
:10007000750F0000750F0000750F0000750F000070
:10008000750F0000750F0000750F0000750F000060
:10009000750F0000750F0000750F0000750F000050
:1000A000750F0000750F0000750F0000750F000040
:1000B000750F0000750F0000750F0000750F000030
:1000C000750F0000750F0000750F0000750F000020
:1000D000750F0000750F0000750F0000750F000010
:1000E000750F0000750F0000000000000000000008
:1000F00000000000711C0000750F0000750F00006B
:10010000750F0000750F0000750F0000750F0000DF
:10011000750F0000750F0000CD1E0000E11E0000ED
:10012000F51E0000091F0000750F0000750F00008C
:10013000750F0000750F0000750F0000750F0000AF
:10014000750F0000750F0000750F0000750F00009F
:10015000750F0000750F0000750F0000750F00008F
:10016000750F0000750F0000750F0000750F00007F
:10017000750F0000750F0000750F0000750F00006F
:10018000750F0000750F0000750F0000750F00005F
:10019000750F0000750F0000750F0000750F00004F
:1001A000750F0000750F0000750F0000750F00003F
:1001B000750F0000750F0000750F0000750F00002F
:1001C000750F0000750F0000750F0000750F00001F
:1001D000750F0000750F0000750F0000750F00000F
:1001E000750F0000750F0000750F000091210000D1
:1001F000750F0000750F0000750F0000750F0000EF
:10020000750F0000750F0000750F0000750F0000DE
:10021000750F0000750F0000750F0000750F0000CE
:10022000750F0000750F0000750F0000750F0000BE
:10023000750F0000750F0000750F0000750F0000AE
:10024000750F0000750F0000750F0000750F00009E
:10025000750F0000750F0000750F0000750F00008E
:10026000750F000010B5054C237833B9044B13B15A
:100270000448AFF300800123237010BD78000020F4
:10028000000000003C9A02000C4B43B10C480D49A1
:1002900010B5AFF300800C48036823B910BD0A48BD
:1002A000036833B97047094B002BF7D0BDE8104005
:1002B0001847064B002BF5D0184700BF0000000080
:1002C0003C9A02007C0000203C9A020000000000E2
:1002D00070B500BF8C4C1026A66132208B4DA8470C
:1002E000666100BF3220A847A6613220A84700BF40
:1002F000402666610A20A847A6610520A8476661D6
:10030000834B1B7823B9202262610122804B1A7033
:10031000012280498048814B98477B4C4025A5614C
:1003200014207A4B98476561794B1B7823B92022BA
:1003300062610122764B1A70012276497648774B2A
:100340009847714C4025A5611420704B9847656112
:100350006F4B1B7823B92022626101226C4B1A700B
:1003600001226C496C486D4B9847674C4025A5614C
:100370001420664B984765616561654B1B7823B90E
:10038000202262610122624B1A70E22261496248B6
:10039000624B98475C4B40229A615A615C4B1B78D8
:1003A0002BB12022584B9A610022594B1A702322FC
:1003B00058495948594B9847534B40229A615A61C2
:1003C000534B1B782BB120224F4B9A610022504B8C
:1003D0001A7002224F495048504B98474A4B4022CE
:1003E0009A615A614A4B1B782BB12022464B9A6185
:1003F0000022474B1A70542246494748474B9847BA
:10040000414B40229A615A61414B1B782BB9202203
:100410003D4B5A6101223E4B1A70E0223D493E4855
:100420003E4B9847384B40229A615A61384B1B78B3
:100430002BB12022344B9A610022354B1A700122D5
:1004400034493548354B98472F4C4025A5616420E9
:10045000334B984765612E4B1B7823B9202262618C
:1004600001222B4B1A70E0222A492B482B4B98472C
:10047000254B40229A615A61254B1B782BB12022D3
:10048000214B9A610022224B1A70032221492248F3
:10049000224B98471C4C4025A56101201B4B9847D7
:1004A00065611B4B1B7823B9202262610122184B26
:1004B0001A70012217491848184B9847124C4025CA
:1004C000A5610120114B98476561114B1B7823B939
:1004D0002022626101220E4B1A70E6220D490E485D
:1004E0000E4B9847084B40229A615A61084B1B7883
:1004F0002BB12022044B9A610022054B1A70042272
:10050000044905480EE000BF0080004121150000AD
:1005100000000020F7C3031C808000414110000050
:10052000011500008A4B98478A4B40229A615A6114
:10053000894B1B782BB12022864B9A610022864B77
:100540001A703A2285498648814B9847814B402250
:100550009A615A61804B1B782BB120227D4B9A61A6
:1005600000227D4B1A70B6227C497D48784B984713
:10057000784B40229A615A61774B1B782BB9202225
:10058000744B5A610122744B1A70B022734974483B
:100590006F4B98476F4B40229A615A616E4B1B78A4
:1005A0002BB120226B4B9A6100226B4B1A702822D0
:1005B0006A496B48664B9847664B40229A615A617C
:1005C000654B1B782BB12022624B9A610022624B53
:1005D0001A708022614962485D4B98475D4C402506
:1005E000A561604B9847604B9847421EC2F30722B3
:1005F0006561594B1B7823B12021A1610021564B25
:10060000197056495648524B9847524C4025A5619F
:10061000544B9847544B9847421ED2B265614E4B9B
:100620001B7823B12021A16100214B4B19704B494C
:100630004B48474B9847474C4025A561494B984745
:100640004A4B9847421EC2F307226561424B1B7812
:1006500023B12021A16100213F4B19703F4940483F
:100660003B4B98473B4C4025A5613E4B98473F4B41
:100670009847421ED2B26561374B1B7823B12021C7
:10068000A1610021344B197034493548304B9847EB
:10069000304B40229A615A612F4B1B782BB120229C
:1006A0002C4B9A6100222C4B1A7000222B492C48AB
:1006B000274B9847274B40229A615A61264B1B785B
:1006C0002BB92022234B5A610122234B1A70F022AE
:1006D000224923481E4B98471E4B40229A615A617B
:1006E0001D4B1B782BB120221A4B9A6100221A4B0A
:1006F0001A70032219491A48154B9847154B402286
:100700009A615A61144B1B782BB92022114B5A6104
:100710000122114B1A703A22104911480C4B98478C
:100720000C4B40229A615A610B4B1B782BB1202253
:10073000084B9A610022084B1A7055220749084855
:10074000034B9847034B40229A615A6110E000BF67
:10075000411000000080004100000020F7C3031C8E
:1007600080800041E10E0100ED0E0100150F010037
:100770008A4B1B782BB92022894B5A610122874B67
:100780001A70B42287498848884B9847844B402286
:100790009A615A61814B1B782BB12022804B9A6160
:1007A00000227E4B1A7002227E497F487F4B984779
:1007B0007B4B40229A615A61784B1B782BB12022E7
:1007C000774B9A610022754B1A700D227549764855
:1007D000764B9847724B40229A615A616F4B1B7857
:1007E0002BB120226E4B9A6100226C4B1A700022B2
:1007F0006C496D486D4B9847694B40229A615A612C
:10080000664B1B782BB12022654B9A610022634B0B
:100810001A702B2263496448644B9847604B40220E
:100820009A615A615D4B1B782BB120225C4B9A6117
:1008300000225A4B1A7028225A495B485B4B984752
:10084000574B40229A615A61544B1B782BB120229E
:10085000534B9A610022514B1A7000225149524861
:10086000524B98474E4B40229A615A614B4B1B7832
:100870002BB120224A4B9A610022484B1A70002269
:1008800048494948494B9847454B40229A615A612B
:10089000424B1B782BB12022414B9A6100223F4BE7
:1008A0001A7000223F494048404B98473C4B402239
:1008B0009A615A61394B1B782BB92022384B5A6107
:1008C0000122364B1A70B62236493748374B9847C3
:1008D000334B40229A615A61304B1B782BB1202256
:1008E0002F4B9A6100222D4B1A7001222D492E4860
:1008F0002E4B98472A4B40229A615A61274B1B780E
:100900002BB12022264B9A610022244B1A701D2203
:1009100024492548254B9847214B40229A615A612A
:100920001E4B1B782BB120221D4B9A6100221B4BC2
:100930001A7000221B491C481C4B9847184B402238
:100940009A615A61154B1B782BB12022144B9A6186
:100950000022124B1A700C2212491348134B98476D
:100960000F4B40229A615A610C4B1B782BB120220D
:100970000B4B9A610022094B1A70092209490A4857
:100980000A4B9847064B40229A615A61034B1B78E9
:100990008BB12022024B9A610AE000BF00000020C8
:1009A00000800041F7C3031C80800041411000001B
:1009B00000228B4B1A7000228A498B488B4B984738
:1009C0008B4B40229A615A61854B1B782BB12022B8
:1009D000874B9A610022824B1A700022814982481B
:1009E000824B9847824B40229A615A617C4B1B781C
:1009F0002BB920227E4B5A610122794B1A702A2290
:100A000078497948794B9847794B40229A615A61E5
:100A1000734B1B782BB12022754B9A610022704BCF
:100A20001A7000226F497048704B9847704B4022F3
:100A30009A615A616A4B1B782BB120226C4B9A61E8
:100A40000022674B1A70002266496748674B984737
:100A5000674B40229A615A61614B1B782BB120226F
:100A6000634B9A6100225E4B1A7001225D495E4819
:100A70005E4B98475E4B40229A615A61584B1B78F7
:100A80002BB120225A4B9A610022554B1A70DF225B
:100A900054495548554B9847554B40229A615A61E5
:100AA0004F4B1B782BB92022514B5A6101224C4BE2
:100AB0001A702B224B494C484C4B98474C4B4022C8
:100AC0009A615A61464B1B782BB12022484B9A61A0
:100AD0000022434B1A70002242494348434B984737
:100AE000434B40229A615A613D4B1B782BB1202227
:100AF0003F4B9A6100223A4B1A70002239493A481A
:100B00003A4B98473A4B40229A615A61344B1B78D2
:100B10002BB12022364B9A610022314B1A700122F0
:100B200030493148314B9847314B40229A615A61E4
:100B30002B4B1B782BB120222D4B9A610022284B86
:100B40001A700F2227492848284B9847284B4022E3
:100B50009A615A61224B1B782BB92022244B5A618F
:100B600001221F4B1A7029221E491F481F4B98470C
:100B70001F4B40229A615A61194B1B782BB92022D6
:100B80001B4B5A610122164B1A70BE22154916489A
:100B9000164B9847164B40229A615A61104B1B78AE
:100BA0002BB12022124B9A6100220D4B1A700622A3
:100BB0000C490D480D4B98470D4B40229A615A61E4
:100BC000074B1B782BB12022094B9A610022044B62
:100BD0001A70FF2203490448044B98470AE000BFFB
:100BE00000000020F7C3031C80800041411000007A
:100BF00000800041264B40229A615A61254B1B78A8
:100C00002BB12022224B9A610022224B1A70012222
:100C100021492248224B98471D4B40229A615A6134
:100C20001C4B1B782BB12022194B9A610022194BC7
:100C30001A70FF2218491948194B9847144B402243
:100C40009A615A61134B1B782BB12022104B9A6189
:100C50000022104B1A7000220F491048104B984781
:100C60000B4B40229A615A610A4B1B782BB1202210
:100C7000074B9A610022074B1A7001220649074868
:100C8000074B9847024B40229A619A6170BD00BFA2
:100C90000080004100000020F7C3031C8080004159
:100CA000411000002DE9F84FB1F90430002B0FDBA3
:100CB00081468A461546B1F90630002B08DBB1F9AA
:100CC0000040044B9847044B98470138844205DDA7
:100CD000BDE8F88FE10E0100ED0E0100BAF9024007
:100CE000944B9847944B984701388442F0DCBAF90A
:100CF000006026EAE676BAF9024024EAE474A346E4
:100D0000BAF904708B4B98478C4B9847013887424F
:100D100000F30A81BAF90470BAF90680854B984746
:100D2000854B98470138804500F31881BAF9068051
:100D30004022834B5A61834B1B782BB92022804B76
:100D40005A6101227F4B1A702A227F497F48804BCB
:100D500098477B4B40219961C6F307225961794B33
:100D60001B782BB12021764B99610021754B1970AE
:100D700075497648764B9847714B40229A615A6183
:100D8000704B1B782BB120226D4B9A6100226D4B6A
:100D90001A70F2B26C496D486D4B9847684B402110
:100DA0009961C7F307225961664B1B782BB120214B
:100DB000634B99610021634B197063496348644B2D
:100DC00098475F4B40219961FAB259615D4B1B789E
:100DD0002BB120215A4B996100215A4B19705A4965
:100DE0005A485B4B9847564B40229A615A61554B83
:100DF0001B782BB92022524B5A610122514B1A7099
:100E00002B2251495148524B98474D4B40219961F3
:100E1000CBF3072259614B4B1B782BB12021484B58
:100E200099610021474B197047494848484B9847FA
:100E3000434B40229A615A61424B1B782BB12022CE
:100E40003F4B9A6100223F4B1A70E2B23E493F4845
:100E50003F4B98473A4B40219961C8F307225961AB
:100E6000384B1B782BB12021354B99610021354B34
:100E7000197035493548364B9847314B40219961B7
:100E80005FFA88F259612F4B1B782BB120212C4B34
:100E9000996100212B4B19702B492C482C4B9847FA
:100EA000274B40229A615A61264B1B782BB920228E
:100EB000234B5A610122234B1A702C2222492348CA
:100EC000234B984740221E4B9A61BAF804300133F5
:100ED000BAF800209B1A9BB21A4A12782AB1202134
:100EE000174A91610021174A11704021144A51613B
:100EF000C6F101063E44B6B2D8450EDB5F00DFF80E
:100F000048B0DFF854A033462A4659460F48D04728
:100F10003D44013424B2A045F5DA4022084B9A61E1
:100F200048460C4B9847D3E6024B9847034B9847EB
:100F3000471EF1E6E10E0100150F0100ED0E010064
:100F40000080004100000020F7C3031C80800041A6
:100F500041100000AD0F010079100000034B9847CD
:100F6000034B984700F1FF38E2E600BFE10E0100B5
:100F7000150F0100FEE7000008B51C4B1C4A9A4201
:100F800010D01C4B194A9A420CD2013B9B1A23F0F9
:100F9000030304331344164951F8040B42F8040BBD
:100FA0009A42F9D1144B154A9A420AD2013B9B1A34
:100FB00023F0030304331344002142F8041B93423B
:100FC000FBD10F4B0F4A22F07F029A60D3F88820A2
:100FD00042F47002C3F88820BFF34F8FBFF36F8FC6
:100FE000094B9847094B9847FEE700BF00000020D7
:100FF0003C9A020074000020046E0020780000205B
:1010000000ED00E00000000095B40100B1210000F7
:1010100010B4530003F47C73540104F4703423437C
:1010200002F007042343520302F0E0521A4302EA9B
:101030000103836121EA020141615DF8044B7047BD
:1010400010B540240A4B5C610A4B9847082300BF47
:10105000013BFCD18022064B5A61082300BF013BB3
:10106000FCD1034B80229A6140229A6110BD00BFDF
:1010700000800041111000008BB12DE9F0410F46B6
:101080000646144602EB4305DFF8148034F8022BC1
:1010900039463046C047AC42F8D1BDE8F0817047D0
:1010A000411000002DE9F04F83B08B4600924001C3
:1010B000C3B201930026DFF8949165E009EBC713F2
:1010C0005D60AAB242F080429A622A0C42F040422D
:1010D0009A62009B1B78012B77D023B3022B00F080
:1010E0008480892257490020574B984724E009EB18
:1010F000C7125560ABB243F0804343F400339362B0
:101100002B0C43F0404343F400339362E1E709EBD7
:10111000C7139D60AAB242F080429A622A0C42F044
:1011200040429A62D5E709EBC713434493F8402045
:1011300002F0FB0283F84020009B5A686409B2F178
:10114000FF3F62D0E4B209EBC411414491F8403052
:1011500003F0FE0343F0010381F840301AF0010F61
:101160005ED109EBC41404EB580898F8303003F052
:10117000F00302F00F021A4388F8302009EBC7177A
:101180007D610136202E59D0F4B22BFA06F313F00C
:10119000010FF6D004F01F04019B1C445FFA84FA8F
:1011A0004FEA5A170AF01F08012505FA08F5009BB7
:1011B0005B78012B9BD0002B80D0022BA7D046223E
:1011C00020490020204B984783E7012303FA08F3C6
:1011D00009EBC712536002EB080090F8401041F091
:1011E000040180F840109361A6E7012303FA08F395
:1011F00009EBC712536002EB080090F8401041F071
:10120000040180F84010536196E7E4B209EBC4147E
:10121000A04498F8403003F0FE0388F84030ADE772
:1012200009EBC41404EB580898F8303003F00F03AE
:1012300043EA0212D2B288F830209FE703B0BDE83B
:10124000F08F00BF30B50100D519000000800041CB
:1012500070B582B00023009302238DF801304FF067
:10126000FF3301936A463F4901203F4B98473F4B6C
:1012700040269E603E4A9A624FF040429A6293F83E
:10128000461001F0FB0183F8461093F8461001F078
:10129000FE0183F8461010259D60364999629A62D6
:1012A00093F8441001F0FB0183F8441093F84410C4
:1012B00001F0FE0183F8441008249C602E499962D5
:1012C0009A6293F8431001F0FB0183F8431093F8FE
:1012D000431001F0FE0183F843102021996001F1D1
:1012E000804199629A6293F8451001F0FB0183F8FE
:1012F000451093F8451001F0FE0183F84510802059
:1013000098601E4999629A6293F8472002F0FB02A6
:1013100083F8472093F8472002F0FE0283F8472025
:101320004FF48072C3F8842101F500318031C3F895
:10133000A8111349C3F8A811C3F8842193F8C81160
:1013400041F0040183F8C811C3F8942193F8C8212F
:1013500002F0FE0283F8C8219E619D619C61986144
:1013600002B070BDF7C3031CA5100000008000414F
:101370004000004010000040080000408000004095
:10138000000002C07047000008B50649D1E90023FB
:10139000013243F10003C1E900230120024B9847C9
:1013A00008BD00BF980000204510010010B511488D
:1013B000114B9847114A536943F4804353614022CB
:1013C0000F4BC3F8A4200F4B98470F4C02460F4910
:1013D00020460F4B98470F4901230B610E4A4A6183
:1013E0000B76083120460D4B984720460C4B98470A
:1013F00010BD00BF10E000E0ED1400000008004048
:10140000001C00404B210000046C0020003800400C
:10141000491600009800002089130000C116000042
:101420008516000030B583B01F4B4022C3F8DC2086
:101430004322C3F88C201D4A936943F400739361DF
:101440001B4C0023009310231A4A1B4920461B4DB6
:10145000A8471B4B93F8D82002F0FE0242F001028D
:1014600083F8D82093F8BC2002F0F00242F0030287
:1014700083F8BC2093F8D92002F0FE0242F001026A
:1014800083F8D92093F8BC2002F00F0242F030021A
:1014900083F8BC2020460B4B98470C220A49204673
:1014A0000A4B984703B030BD001C004000080040C4
:1014B000206C0020B4000020002001411919000018
:1014C00000800041A919000004000020411500001F
:1014D000EFF31083036072B6BFF35F8F7047BFF303
:1014E0005F8F036883F310887047000008B5024BD4
:1014F0001860024B984708BDC4000020891B0000FB
:1015000010B5044B1C68044B984701462046034B1A
:10151000984710BDC4000020511B0000911B000023
:1015200010B5044B1C68044B984701462046034BFA
:10153000984710BDC4000020691B0000911B0000EB
:1015400070B50D461646044660B1081C18BF012050
:1015500034220549054B98472368324629462046E0
:10156000984770BD0020F3E74CB50100D519000085
:10157000F8B5844607682FB18D683C460026C2F155
:10158000010E0BE00E4B9847F8BD7344A06803446E
:10159000AB420AD22368264653B11C466368934285
:1015A000F3D8A06803449B1AF2E7A74204D034465C
:1015B0002046044B9847F8BD6046014B9847F8BD5C
:1015C000FD190000291A00002DE9F0474469076958
:1015D00001370761037E13F0010F13D1037E13F06F
:1015E000020F0FD154B36368FB1AA268934207D36A
:1015F000064600F11408DFF84890DFF848A012E032
:10160000BDE8F087037E43F002030376BDE8F08770
:101610007569E3682046984785B12C466B68FB1ACC
:10162000AA6893420AD34046C847237C012BEFD1D6
:1016300067603A4621464046D047E9E7BDE8F08773
:10164000311A00007115000038B50D46044678B116
:10165000081C18BF01203B220649074B9847294622
:101660002046064B984700202061054B236038BD7B
:101670000020F0E760B50100D51900007D1F0000D3
:10168000C915000010B5044653220949003018BF9F
:101690000120084B98472046074B984720B9204621
:1016A000064B9847002010BD6FF0100010BD00BF22
:1016B00060B50100D5190000392100002521000086
:1016C00070B582B00D46044618B3081C18BF01203F
:1016D0007A221E491E4B9847237E43F0010323764E
:1016E00004F11406294630461A4B984798B92369E5
:1016F0006B60226929463046174B9847237E03F0DA
:10170000FE032376237E13F0020F10D1002002B0D7
:1017100070BD0020DCE7237E03F0FE0323767F22EA
:101720000A4900200A4B98476FF01100EFE701A823
:101730000A4B9847237E03F0FD0323762046084B8F
:10174000984701A8074B98470020E0E760B50100E3
:10175000D5190000DB19000071150000D11400003C
:1017600051210000DF14000008B500238362C36923
:101770001BB1A0F108021046984708BD08B5002328
:101780008362436A1BB1A0F108021046984708BD66
:1017900038B50446A0F108052C30034B9847236A5E
:1017A0000BB12846984738BDD11A000070B50E46D7
:1017B00015460446E0B1E9B1101C18BF012040F203
:1017C0003B120F490F4B9847B4F84420B4F84C3003
:1017D0009A4211D1A664A4F84C500023A4F84430D6
:1017E0000123236304F10800074B9847284670BD86
:1017F0000020E4E70020E2E76FF01B0070BD00BFAF
:1018000078B50100D5190000BB1E000010B50446D4
:10181000838FB0F844209A4209D0026C591C81870A
:10182000D15C044B98472046034B984710BD034BAF
:10183000984710BDB51E0000BB1E0000C31E00006F
:101840002DE9F04782B00F4690460646A0B199B107
:10185000002A2DD14FF4AC7229490020294B98471A
:1018600001A8294B984706F13400284B984701A856
:10187000274B984700253EE04FF4AC7220490020EA
:10188000204B984701A8204B984706F1340A504650
:101890001E4B9847814601A81D4B9847B9F1000F90
:1018A00004D0B8F1000F19D1002524E0002522E072
:1018B0004FF4AC7212490120124B984701A8124B09
:1018C000984706F1340A5046104B9847814601A8C4
:1018D0000F4B98470025B9F1000F0CD000240D4E96
:1018E000601C85B239195046B04701344C4502D2CC
:1018F000A3B29845F4D8284602B0BDE8F08700BFEF
:1019000078B50100D5190000D1140000111B0000AA
:10191000DF1400008D1A0000F8B50D4616461F466C
:10192000044620B329B332B3181C18BF01203A2251
:101930001349144B98473A46314604F13400124B90
:101940009847D0B9294604F10800104B9847034640
:1019500058B90F4A62600F4A22600F4AA2600F4ACC
:10196000E2600F4A22610F4A62611846F8BD00200A
:10197000DDE70020DBE70020D9E76FF00C03F4E798
:1019800078B50100D51900003D1A00001D1E0000A9
:1019900041180000AD1700000D180000911700005D
:1019A000691700007D17000010B504466122064942
:1019B000003018BF0120054B984704F10800044B84
:1019C0009847002010BD00BF78B50100D519000070
:1019D000A11E000000B900BE704703684BB18B42E6
:1019E00009D01B681BB19942FBD101207047002030
:1019F00070470020704701207047000038B504464A
:101A00000D46064B984780F0010039220449C0B2C8
:101A1000044B984723682B60256038BDDB19000014
:101A200098B50100D519000003680B60016070478C
:101A300003680BB11A6802601846704770B50E460D
:101A40001546044678B181B1A2B1012028220D4982
:101A50000D4B98476B1E1D4209D163600020A060AA
:101A6000E060266070BD0020F0E70020EEE76FF038
:101A70000C0070BD282203490020034B98476B1EC1
:101A8000EBE700BFB8B50100D519000038B50D4629
:101A90000446A0B1081C18BF012040220A490B4B84
:101AA0009847A368E2689A420BD0626813402268A4
:101AB000D35C2B70A3680133A360002038BD0020E5
:101AC000EBE76FF0090038BDB8B50100D51900008B
:101AD00038B50D46044651220B49003018BF01208D
:101AE0000A4B9847E368626813402268D554E3685C
:101AF0006168A2689A1A8A4284BF591AA1600133A8
:101B0000E360002038BD00BFB8B50100D519000062
:101B100010B5044667220549003018BF0120044B68
:101B20009847E068A368C01A10BD00BFB8B50100AF
:101B3000D5190000430900F01F00012202FA00F04D
:101B40004033024A42F82300704700BF00E100E042
:101B5000C0EBC00000EB00100230024BA3FB0030D2
:101B600040087047ABAAAAAAC0EBC00000EB001067
:101B70000230044BA3FB003040084FF47A7303FBA0
:101B800000F07047ABAAAAAA70470000000000004E
:101B90000139FDD8704700BF08B5094A13889BB2C8
:101BA00043F4A0631380074B9847074B9847074BB4
:101BB0009847074B984740F6FF70064B984708BD7B
:101BC00000400041091C0000291C0000FD1B000012
:101BD0002D1C0000D91B000010F0010F08D0054A91
:101BE000054B1A62194643F6FD724B681342FCD14D
:101BF000704700BF07010100001C00400122014B9B
:101C00005A71704700080040064B42F28E329A82A9
:101C100000229A75DA75DA6902F47C52DA610122DF
:101C20001A74704700140040704700000E4A0F4BB2
:101C30005A631A46D36B13F0060FFBD10B4B4FF4CC
:101C400002629A63022283F830201A46D36B13F0A3
:101C5000020FFBD1054B1A6C12F0010F03D11A6C65
:101C600012F0020FF7D070474D0E01000010004037
:101C700000B583B00D4B9B78DBB20193019B13F051
:101C8000020F06D00A4B1B681BB1084A50689847E0
:101C900009E0019B13F0010F05D0054B5B6813B100
:101CA000024A5068984703B05DF804FB0000024107
:101CB000706C002070B489B006466C460D4D0FCD97
:101CC0000FC495E80F0084E80F00009BB3420DD0CD
:101CD000314601AB012053F8042B8A4207D0013072
:101CE0000828F8D1002009B070BC70470020C0B2AD
:101CF000F9E700BFDCB5010010B58469237E13F05D
:101D0000010F03D0A37D13F0010F12D1237E13F036
:101D1000020F03D0A37D13F0020F0FD1237E13F027
:101D2000040F15D0638B03F0370363B1FF23638384
:101D300010BD012323750368984710BD0223237546
:101D40008368984710BDA16A4368C9B2984710BD1F
:101D5000237EDB0900D110BD80232376C36898471A
:101D6000638B9BB26383F6E708B5034B984780000B
:101D70002E3000F0FE0008BDB51C000010B5044672
:101D8000214B9847022805D040F26B221F490020C2
:101D90001F4B9847E36913F0010F19D1E36913F062
:101DA000030FFBD1236813F0020F0BD0236823F03D
:101DB00002032360E36913F0030FFBD1E36913F01F
:101DC000020FFBD105232360E36913F0030FFBD15E
:101DD000E36913F0010FFBD10E4B2360E36913F0AD
:101DE000030FFBD14FF440336360E36913F01F0F1F
:101DF000FBD1094BA3604FF61143A3810020A073D0
:101E000084F8300010BD00BFB51C000014B60100FE
:101E1000D5190000040010400200700070B50D4696
:101E20000646CB221849003018BF0120174B9847AF
:101E30002846174B9847044608B1204670BDB56147
:101E4000144B9D4204BF144B1E602846134B984709
:101E5000011DC9B2012500F01F0205FA02F2430973
:101E60009B0003F1604303F56143C3F88020BFF397
:101E70004F8FBFF36F8FC3F880211A600130C0B25B
:101E80008142E8D1D9E700BF14B60100D51900009E
:101E90007D1D000000200141C8000020691D0000D8
:101EA0008269136843F002031360D36913F0030FD0
:101EB000FBD17047836999627047836901229A75E3
:101EC0007047836902229A757047000008B5024B7B
:101ED0001868024B984708BDC8000020F91C000094
:101EE00008B5024B1868024B984708BDC80000208F
:101EF000F91C000008B5024B1868024B984708BD52
:101F0000C8000020F91C000008B5024B1868024BFD
:101F1000984708BDC8000020F91C000070B588B0C3
:101F200006466C46124D0FCD0FC495E80F0084E8AD
:101F30000F00009BB3420BD0304601AA012352F898
:101F4000041B814205D00133082BF8D100200BE09F
:101F5000002313F0FF0F09D04FF49E7205490020B3
:101F6000054B98474FF0FF3008B070BD0020FBE7ED
:101F700030B6010064B60100D519000070B5064600
:101F80000C460846604B98470546F4608D225F4931
:101F900001205F4B9847236913F0010F19D1236982
:101FA00013F0030FFBD1236813F0020F0BD023684B
:101FB00023F002032360236913F0030FFBD123698D
:101FC00013F0020FFBD101232360236913F0030FE9
:101FD000FBD1236913F0010FFBD105EB85034D4ABB
:101FE00002EB83035A6A2260236913F0030FFBD1CB
:101FF00005EB8503474901EB830393F82A10E1734E
:102000001B8DE3800123237302F00C02082A48D0C1
:10201000002A58D105EB85033E4A02EB83039B8DD2
:10202000A383236913F0C00FFBD10023E38323694B
:1020300013F0C00FFBD101236372374B9C4204BFE6
:10204000364B1E6005EB8503324A02EB8303B3F97E
:102050002230002B23DB5A0903F01F03012101FA70
:1020600003F320322E4941F82230BFF34F8FBFF3E4
:102070006F8F05EB8505274B03EB8505B5F92230FE
:10208000002B0CDB590903F01F03012202FA03F3B2
:10209000234A01F1600042F8203042F8213000204C
:1020A00070BD05EB85031B4A02EB8303DB6AE3612A
:1020B000236913F0C00FFBD100232362236913F0BF
:1020C000C00FFBD1B7E7042AB5D105EB8503114A50
:1020D00002EB830393F82C302377236913F0C00FAE
:1020E000FBD100236377236913F0C00FFBD105EB0D
:1020F0008503084A02EB830393F82B30E3762369C8
:1021000013F0200FFBD196E71D1F000064B60100FD
:10211000D519000030B6010000380040CC00002086
:1021200000E100E0C268136843F002031360136922
:1021300013F0030FFBD17047C268136913F0030F4C
:10214000FBD11068C0F340007047002070470000CA
:1021500010B5C068094B9847044640F20F12084971
:102160000120084B984704EB8404074B03EB8404DD
:1021700094F82200054B984710BD00BF1D1F0000BA
:1021800064B60100D519000030B60100351B00000F
:1021900008B5064B1868C3689A7A12F0010F00D18F
:1021A00008BD01229A7203689847F9E7CC00002025
:1021B00008B5024B9847024CA047FDE7C521000037
:1021C0009922000030B58DB01E4B98471E4B9847A2
:1021D0001E4B98471E4B98471E4B98471E4B9847DF
:1021E0001E4B98471E4C4FF4965300221D49204623
:1021F0001D4DA84701A81D4B98471D4B0493029401
:1022000001A81C4B984700201B4B9847054600210E
:102210001A4B984704461A491A4B98470022114610
:102220002046194CA04700212846184B98470546E0
:1022300023225A21A04716492846164B98470DB02D
:1022400030BD00BF991B000025140000851300005D
:1022500051120000AD13000069280000D1020000F7
:1022600050260020D0000020710D0100110D01004A
:10227000A50C0000910D01004D2300006D98010098
:1022800078B60100119601003D34000005AB010055
:10229000E03B020005A8010008B50120024B984769
:1022A000024B984708BD00BF21150000CD37010043
:1022B000003018BF01207047F0B5C3B00546144682
:1022C0001C4B9847E5282CD8064602AF0246294603
:1022D0003846194B9847BD192023BB5528236B70EE
:1022E0003023AB707823EB70291D1C22134824FA8D
:1022F00002F303F00F0303441B7D01F8013B043A92
:1023000012F1040FF3D129232B7300236B7302AB5B
:1023100000930B4BBC220B4903200B4CA04743B04E
:10232000F0BD0095064BBF2206490320064CA0478E
:10233000F5E700BF1FB5010055260100EC3B020088
:10234000143C0200283C02005D22010008B1C06B71
:10235000704710B582B0084B984710B1C06B02B0FF
:1023600010BD064B0093064B2E2206490220064C58
:10237000A0470020F3E700BFE10E0100043E020089
:10238000303D0200D83D02005D22010008B1006C22
:10239000704710B582B0084B984710B1006C02B07E
:1023A00010BD064B0093064B4B2206490220064CFB
:1023B000A0470020F3E700BFE10E0100403E02000D
:1023C000443D0200D83D02005D22010008B1406C8E
:1023D000704710B582B0084B984710B1406C02B0FE
:1023E00010BD064B0093064B5C2206490220064CAA
:1023F000A0470020F3E700BFE10E01007C3E020091
:102400005C3D0200D83D02005D220100A0B138B55C
:1024100003460024094D93F8342002F02002002ADC
:1024200018BF1C461846A84703460028F3D114B12C
:102430002046034B984738BD704700BF7D2C0000F5
:10244000B53300002DE9F84F037D13F0010F2AD1B9
:1024500017468A460646C4684FF001090025DFF892
:10246000C480AB464AE0337D13F0100F00D1D5B9DC
:10247000B9F1000F17D03046D0470446002D35D0B3
:10248000D94646E0F368A3420DD093B11868C369FA
:10249000002217219847F36800220E2118681E4B6E
:1024A0009847012801D0BDE8F88FF36818681B4BE6
:1024B0009847F4602068C369002216219847F368A2
:1024C00000220D211868144B98470128EBD1F368BE
:1024D0001868134B9847F3681868104B984733698E
:1024E000002BE0D030469847BDE8F88F0028DAD0BE
:1024F0000546D9462068C0470028C3D0002CB2D07A
:10250000002D08BF254621463046B8470446A8425C
:10251000C9D0002CEED1F1E7CD2A00002133000014
:102520000D240000A531000008B518210148024B18
:10253000984708BDEC6D0020F91E010008B5024A5D
:102540000249034B984708BDBD1F0100A91F0100A8
:102550004524000008B5024A0249034B984708BDCC
:10256000E91F0100B31F01004524000038B50446EF
:10257000037DC3F3001543F01003037513F0080F38
:102580000CBF044B044B9847237D65F3041323755C
:1025900038BD00BF3D2500005525000000284FD064
:1025A000F0B583B005460C460746264B98470146D2
:1025B000A0B103689C4207D0234E3846B04701467D
:1025C00060B10B68A342F8D1204B0093204B7522D9
:1025D00020490120204CA04703B0F0BDA36B73B18C
:1025E00020461E4B984750B1A06B1D4B98471D4B82
:1025F0000093174B7F2217490120174EB047A56360
:102600002846194B98470646184B984758B1002E54
:10261000E2D0346028460B4B98478642DCD12846EE
:102620000F4B9847D8E70A4B0093852209490320AE
:10263000094CA047324600230D480E498847FEE763
:10264000704700BFA91F0100BD1F0100E83F020045
:10265000983F0200AC3F02005D220100F94F0000EC
:102660006D250000244002005D1F0100B122000022
:10267000D83F0200B92200002DE9F041D0F838809F
:10268000B8F1000F51D0D8F80C30002B4DD00546D2
:102690001B6898421ED046464046254B9847044644
:1026A000002842D003689D4209D0224F214630467F
:1026B000B8470446002838D023689D42F6D1214609
:1026C00040461D4B984720461C4B98470023AB6360
:1026D000BDE8F08198F8143013F0010F05D098F898
:1026E00014306FF3000388F814304046104B9847BD
:1026F000D8F80C3083420BD04046114B9847D8F89D
:102700000C301B689D4204BF0023C8F80C30C2E7A0
:1027100040460C4B9847D8F80C309842ECD10068F2
:10272000C369002217219847E9E7BDE8F08100BF9F
:10273000A91F0100BD1F010095200100C524010053
:102740006D250000B31F010018B1C3681BB11868E4
:102750007047002070470020704718B1007DC0F31B
:102760004000704700207047014B5868704700BF19
:1027700074260020F8B5B0B1034690F8502042F01E
:10278000020280F85020184A5268904204D039B1B1
:10279000DA6B914204D0F8BD0020134A1060F6E7CE
:1027A0000022DA63F8BD0C460020104B9847034620
:1027B0000028F0D00C4D00270C4E05E0DF631846D2
:1027C000B04703460028E6D093F8502042F00202BA
:1027D00083F850206A689A4208BF2F60002CEDD021
:1027E000DA6B9442EBD1E9E7742600202110010056
:1027F00008B500210846014B984708BD7527000021
:10280000014B1868704700BF742600202DE9F0477F
:102810008946904600F1040A5046114B9847E0B1B2
:1028200004461FFA89F61FFA88F50E4F238A3344AF
:102830002382638A2B446382A38A3344A382E38A7C
:102840002B44E382424649462046FFF7DFFF2146FC
:102850005046B84704460028E8D1BDE8F08700BFDD
:10286000A91F0100BD1F010030B585B0214B1B78A9
:10287000002B36D1204B9847204B9847204B984748
:10288000204B9847204B984710212048204CA047C8
:10289000204B02930193009302224FF01F014FF649
:1028A00000001D4DA8471D4B98471D4B98474FF4FE
:1028B000B8711C48A04760211B48A0471B4B984794
:1028C0001B4B984701201B4B98470120094B187060
:1028D000194B0093194BA22219491A4CA04705B075
:1028E00030BD194B0093154B782215490220154C29
:1028F000A047F4E77C260020BD230100ED35010050
:10290000791C01009D120100292500003C6D00206A
:10291000F91E010010000020496B0100D1410100A7
:10292000555E0000986C00208C6C0020F1270000A0
:10293000C1FF00002DF400001C48020058400200B6
:10294000DC4702005D2201000448020030B583B07C
:1029500004460D460C4B984738B194F8343065F373
:10296000C71384F8343003B030BD084B009340F2F5
:10297000945207490320074DA847224600230648E2
:1029800006498847FEE700BFB1220000B4400200BC
:10299000DC4702005D2201003C480200B922000031
:1029A00030B583B004460D460C4B984738B194F8C7
:1029B000343065F3000384F8343003B030BD084B85
:1029C00000934FF4B46207490320074DA8472246FD
:1029D0000023064806498847FEE700BFB1220000F1
:1029E000CC400200DC4702005D2201003C480200AE
:1029F000B92200002DE9F04186B0074615461E4673
:102A00000C4621B10846284B9847002833D0039440
:102A100000238DF810300593244B5B6803B10593B8
:102A2000224B03AA5A60D3F808809E60204B984737
:102A300018B183680BB12946984717B1294620463B
:102A4000B8471A4BC3F808805A6892685A609DF8D4
:102A50001030F3B90CB394F8343013F0400F1ED09B
:102A60002068F0B132462946124B9847012814BF1E
:102A7000002001200EE0104B00934FF4DB620F4961
:102A800003200F4DA847224600230E480E498847D1
:102A9000FEE7002006B0BDE8F0810120FAE7012042
:102AA000F8E70120F6E700BFB12200007C260020F5
:102AB00069270000CD2A00009C410200DC4702008B
:102AC0005D2201003C480200B9220000E8B170B567
:102AD00082B0044616460D460D4B984768B90D4B1B
:102AE000009340F2C4620C4903200C4DA8472246D3
:102AF00000230B480B498847FEE733462A46214608
:102B0000A069094CA04702B070BD0120704700BF0A
:102B1000B1220000B0410200DC4702005D2201004A
:102B20003C480200B9220000F529000030B583B00E
:102B300004460D46094B984710B1E56103B030BD1E
:102B4000074B009340F21B7206490320064DA8472D
:102B500022460023054806498847FEE7B1220000C7
:102B6000C0410200DC4702005D2201003C48020037
:102B7000B922000020B110B5C4691CB1A04710BD36
:102B800001207047012010BD30B583B004460D46CA
:102B9000094B984710B1256203B030BD074B009335
:102BA00040F2377206490320064DA847224600230B
:102BB000054806498847FEE7B1220000D8410200D7
:102BC000DC4702005D2201003C480200B9220000FF
:102BD00030B583B004460D460D4B984768B90D4B90
:102BE000009340F249720C4903200C4DA84722463D
:102BF00000230B480B498847FEE72946606A0A4BC9
:102C00009847034600B16062184603B030BD00BF6C
:102C1000B1220000F0410200DC4702005D22010009
:102C20003C480200B92200009928010030B583B069
:102C300004460C4B984768B90B4B009340F259720D
:102C40000A4903200A4DA8472246002309480A4999
:102C50008847FEE700226286E369062120469847FE
:102C600003B030BDB12200000C420200DC4702007C
:102C70005D2201003C480200B922000030B583B05B
:102C800004460A4B984710B1206803B030BD084B8A
:102C9000009340F29F7207490320074DA847224640
:102CA0000023064806498847FEE700BFB12200001E
:102CB00028420200DC4702005D2201003C4802007D
:102CC000B922000030B583B004460E4B984708B1D6
:102CD0000D4D0EE00D4B009340F26B720C4903203A
:102CE0000C4DA847224600230B480C498847FEE7B5
:102CF0001C462046A84703460028F9D1204603B0C9
:102D000030BD00BFB12200007D2C00003C4202001B
:102D1000DC4702005D2201003C480200B9220000AD
:102D20002DE9F04383B00446224B984780B12368D5
:102D30001BB12046204B984704462048204B98471B
:102D4000054660B3DFF878901E4EDFF8708012E021
:102D50001D4B009340F27F721C4903201C4DA84775
:102D6000224600231B481C498847FEE72946404667
:102D7000B047054698B105F130073846C8470146C7
:102D80000028F3D0844206D03846B04701460028D8
:102D9000ECD08C42F8D1284603B0BDE8F0830F4B4D
:102DA0000093094B4FF4F26208490220084CA047F7
:102DB0000025F0E7B1220000C52C0000986C00202F
:102DC000A91F0100BD1F010050420200DC470200A4
:102DD0005D2201003C480200B92200004C4802007C
:102DE00030B583B004460D460D4B984730B19DB1C8
:102DF0002946201D0B4B984703B030BD0A4B00936A
:102E000040F2AD7209490320094DA847224600232C
:102E1000084809498847FEE7201D084B9847EBE71B
:102E2000B1220000BD1F010060420200DC47020029
:102E30005D2201003C480200B9220000A91F0100E8
:102E400030B583B005460C460E4B984760B105F18E
:102E50000F0204F10800234612F8011F03F8011BBA
:102E60008342F9D103B030BD074B009340F6010215
:102E700006490320064CA0472A4600230548064978
:102E80008847FEE7B1220000D8420200DC4702007A
:102E90005D2201003C480200B922000030B583B039
:102EA00004460F4B984768B90E4B009340F6220238
:102EB0000D4903200D4DA847224600230C480D491B
:102EC0008847FEE720460C4B9847034628B1208AE6
:102ED0001B8AC01A00B203B030BDB4F91000FAE783
:102EE000B1220000EC420200DC4702005D2201003A
:102EF0003C480200B92200007D2C000030B583B0B0
:102F000004460F4B984768B90E4B009340F63602C3
:102F10000D4903200D4DA847224600230C480D49BA
:102F20008847FEE720460C4B9847034628B1608A45
:102F30005B8AC01A00B203B030BDB4F91200FAE7E0
:102F4000B1220000FC420200DC4702005D220100C9
:102F50003C480200B92200007D2C000030B583B04F
:102F600004460C4B984730B1A08A0130238AC01A1E
:102F700000B203B030BD084B009340F64A02074947
:102F80000320074DA84722460023064806498847E4
:102F9000FEE700BFB12200000C430200DC47020044
:102FA0005D2201003C480200B922000030B583B028
:102FB00004460C4B984730B1E08A0130638AC01A4E
:102FC00000B203B030BD084B009340F656020749EB
:102FD0000320074DA8472246002306480649884794
:102FE000FEE700BFB122000020430200DC470200E0
:102FF0005D2201003C480200B922000009B92830D6
:10300000704700B583B08DF80010002301936A4625
:103010000821044B984701280CBF0198002003B0F9
:103020005DF804FB752B00002DE9F84F80468A46B9
:1030300093461E461C481D4B9847002831D0054634
:10304000B0422ED0DFF86090194F09E0AB885B45A5
:1030500014D0BBF1FF0F11D01CB32546A64220D0DF
:1030600029464846B847044628684045F4D1A9791E
:103070005145EBD0BAF1FF0FEED1E7E70D4B984782
:103080000D4B9847A9880D4B9847002128460C4BBB
:103090009847294648460B4B984728460A4B98477D
:1030A000DAE7BDE8F88F00BF3C6D0020B31F0100D8
:1030B000E91F0100FD2F0000E7700000ED67000030
:1030C0002913010095200100C524010030B583B00B
:1030D00004460D460B4B984748B10B4B98470023CD
:1030E000FF2229462046094CA04703B030BD084BBB
:1030F0000093084B40F2924207490220074CA04738
:10310000F3E700BFFD2F0000F97000002930000038
:1031100098480200E4430200DC4702005D220100FF
:10312000F8B504681748184B984708B301460027BC
:10313000144E164D03E03046A847014678B18C4244
:10314000F9D00A6823689A42F5D14B6823F07F4290
:10315000636823F07F439A4208BF0127EBE73FB142
:10316000214608480A4B984720460A4B9847F8BD25
:10317000A1792068084B9847084B9847A188084BCD
:103180009847EDE73C6D0020A91F0100BD1F01001D
:1031900095200100C5240100FD2F0000E77000000C
:1031A000ED67000030B583B004460B4B984728B15B
:1031B00094F83400C0F3001003B030BD074B009307
:1031C00040F6412206490320064DA8472246002327
:1031D000054806498847FEE7B12200003444020052
:1031E000DC4702005D2201003C480200B9220000D9
:1031F0002DE9F04186B004460E463A4B984768B92F
:10320000394B00934FF4F07238490320384DA847EA
:1032100022460023374838498847FEE72046374B87
:10322000984710B106B0BDE8F0812046344B98476E
:103230000746344B98470546334B9847874209D099
:103240002846324B9847874204D02846304B98474F
:103250008742E7D1B4F9323004F10F0204F11700CC
:1032600002A912F8017F01F8017B8242F9D19BB2D9
:10327000BDF80820D21AADF80820BDF80A20D21AED
:10328000ADF80A20BDF80C201A44ADF80C20BDF8AA
:103290000E201344ADF80E3002AA314604A81D4B8F
:1032A00098470028BED020461B4B9847044698B14B
:1032B000DFF86080114F184E04F1100204A908468F
:1032C000C0470028AED02046B8470028AAD12046E3
:1032D000B04704460028EFD104A928460F4B984771
:1032E000A0E700BFB122000048440200DC47020012
:1032F0005D2201003C480200B9220000A531000017
:10330000C52C0000212D00004D2300008D2300005E
:10331000CD230000191501007D2C0000595E00002E
:1033200030B585B004461C4B984738B3B4F93230F9
:1033300004F10F0204F1170502A912F8010F01F8B8
:10334000010BAA42F9D19BB2BDF80820D21AADF800
:103350000820BDF80A20D21AADF80A20BDF80C20CA
:103360001A44ADF80C20BDF80E201344ADF80E3011
:1033700002A92046094B984705B030BD084B009381
:1033800040F20D2207490320074DA847224600239B
:10339000064807498847FEE7B1220000F1310000E6
:1033A00060440200DC4702005D2201003C4802004C
:1033B000B9220000F0B583B00546164B984768B9AE
:1033C000154B009340F2622214490320144CA0478D
:1033D0002A460023134814498847FEE72846134B22
:1033E00098470446061D3046114B984785420FD03A
:1033F0002046104FB84701232A46314630460E4E2C
:10340000B047E3692A460121204698472046B8473D
:1034100003B0F0BDB122000074440200DC4702009A
:103420005D2201003C480200B92200007D2C000012
:10343000A91F010021330000212101002DE9F047DF
:1034400084B004468A4617462D4B984700283ED044
:103450002668002E49D0338A228A9B1A53441FFAC9
:1034600083FA0FFA8AF8758A638AED1A3D44ADB281
:103470000FFA85F9B8F1000F02D1B9F1000F23D08E
:103480002046204FB84702A920461F4B9847238A61
:1034900053442382638A2B446382A38A5344A382C6
:1034A000E38A1D44E5824A4641462046174B984729
:1034B000E36902AA022120469847F36922460121C6
:1034C000304698472046B84704B0BDE8F087104B17
:1034D000009340F296220F4903200F4DA847224641
:1034E00000230E480E498847FEE70E4B0093084B19
:1034F0004FF4277207490220074CA047E4E700BFBA
:10350000B122000021330000412E00000D280000F0
:10351000A4440200DC4702005D2201003C48020096
:10352000B9220000D048020030B583B004460D46F1
:103530000D4B984768B90D4B00934FF433720C490B
:1035400003200C4DA847224600230B480B4988470F
:10355000FEE720460A4B9847024629462046094B7B
:10356000984703B030BD00BFB1220000B444020050
:10357000DC4702005D2201003C480200B922000045
:10358000FD2E00003D34000030B583B004460D46EA
:103590000D4B984768B90D4B00934FF436720C49A8
:1035A00003200C4DA847224600230B480B498847AF
:1035B000FEE720460A4B98472A4601462046094B1B
:1035C000984703B030BD00BFB1220000C4440200E0
:1035D000DC4702005D2201003C480200B9220000E5
:1035E0009D2E00003D3400002DE9F04385B00446D7
:1035F0000D4690461F46BDF930602C4B984768B980
:103600002B4B009340F26D322A4903202A4DA847E4
:103610002246002329482A498847FEE78DB12846DB
:10362000224B984790B9224B009340F271322149C6
:103630000320214CA0472A460023204820498847E0
:10364000FEE720461F4B98470546E8E703AB424696
:1036500004F1100105F11000DFF87090C847204612
:10366000184B9847B0F91230BDF80E203244BDF81F
:103670000C103944008A091A09B2ADF80C10D21A9C
:1036800012B2ADF80E2020460F4B984784F84880C0
:10369000A4F84470A4F84660256494F849306FF3A8
:1036A000410384F8493005B0BDE8F083B122000041
:1036B000D4440200DC4702005D2201003C480200C5
:1036C000B92200007D2C00003D34000025180100C7
:1036D0002DE9F04F85B081460E4692460393BDF921
:1036E00038B0A34B984768B9A24B009340F295328B
:1036F000A1490320A14CA0474A460023A048A14964
:103700008847FEE74846A04B9847054648469F4BEA
:103710009847044648469E4B984700EBD07040F3CC
:103720004F0848469B4B984700EBD07040F34F073B
:10373000EEB130468E4B9847F0B1BAF1140F39D83C
:10374000DFE81AF028005C0062006D0076007F0060
:103750008D009900A500B400BA00C500CE00D700C6
:10376000E500F100F70003010C012E013D01484680
:10377000894B98470646DCE77E4B009340F2A13226
:103780007D4903207D4CA047324600237C487D497B
:103790008847FEE730467E4B984700EBD070C8EB79
:1037A00060052DB230467B4B984700EBD070C7EBDD
:1037B000600424B24846784B9847318A039F3944C5
:1037C0002944038AC91A728A5A442244438AD21A63
:1037D00012B209B24846714B984789F848A0A9F837
:1037E0004470A9F846B0C9F8406099F8493043F0F0
:1037F000020389F8493005B0BDE8F08FC8F1000533
:103800002DB27C4224B2D5E73046614B984700EB9D
:10381000D070C8EB60052DB27C4224B2CAE73046B6
:103820005B4B9847A0EB080005B27C4224B2C1E78D
:10383000C8F100052DB23046564B9847C01B04B264
:10384000B8E73046524B984700EBD070C8EB6005A4
:103850002DB230464F4B9847C01B04B2AAE7304602
:103860004B4B9847A0EB080005B23046494B9847B0
:10387000C01B04B29EE7C8F100052DB23046454B8F
:10388000984700EBD070C7EB600424B292E7304653
:103890003F4B9847A0EB080005B230463D4B984798
:1038A00000EBD070C7EB600424B283E7C8F10005D9
:1038B0002DB27C4224B27DE73046354B984700EB71
:1038C000D070C8EB60052DB27C4224B272E730465E
:1038D0002F4B9847A0EB080005B27C4224B269E761
:1038E000C8F100052DB230462A4B9847C01B04B2E0
:1038F00060E73046264B984700EBD070C8EB600578
:103900002DB23046234B9847C01B04B252E73046D5
:103910001F4B9847A0EB080005B230461D4B984757
:10392000C01B04B246E7C8F100052DB27C4224B2A8
:1039300040E7C8F100052DB23046164B984700EB22
:10394000D070C7EB600424B234E7C8F100052DB293
:103950003046104B9847C01B04B22BE730460C4B47
:103960009847A0EB080005B27C4224B222E700BFD2
:10397000B1220000E4440200DC4702005D220100A5
:103980003C480200B92200009D2E0000FD2E0000E0
:103990005D2F0000AD2F00007D2C00003D340000A5
:1039A00030460D4B9847A0EB080005B230460B4B54
:1039B000984700EBD070C7EB600424B2FAE63046BB
:1039C000054B9847A0EB080005B23046034B9847DB
:1039D000C01B04B2EEE600BF5D2F0000AD2F00005B
:1039E00030B583B00446124B984790B194F84930F3
:1039F00013F0020FB4F9443094F84820B4F946109B
:103A00000091216C204614BF0A4C0B4CA04703B018
:103A100030BD0A4B009340F22A4209490320094D68
:103A2000A84722460023084808498847FEE700BF08
:103A3000B1220000D1360000E9350000F844020050
:103A4000DC4702005D2201003C480200B922000070
:103A50002DE9F041064600210D4B9847B0B10446D0
:103A60000C4D4FF000080A4F2046A847E369424634
:103A70000421204698472046A8472046FFF7E8FF44
:103A800021463046B84704460028EDD1BDE8F08114
:103A9000E12D00002133000030B583B005460C460F
:103AA000364B984798B1712C46D8702C23D2412CB4
:103AB0001BD8402C1FD2022C05D3072C1BD9A4F1F4
:103AC0001003082B17D928462D4B98472FE02D4B74
:103AD000009340F21D522C4903202C4CA0472A464B
:103AE00000232B482B498847FEE7532C21D8502C24
:103AF00001D24C2CE7D12846214B9847EB69002294
:103B0000042128469847152C09D3182C01D9FF2CDD
:103B100005D1286818B1C3690022012198472846B9
:103B2000174B9847FF2C24D014F4004F21D103B039
:103B300030BD5C2CC7D1DEE77F2C0CD948F2810365
:103B40009C4211D848F280039C42D4D2902CD2D00F
:103B5000FF2CB8D1CFE77E2CCDD2732CB3D3752CEC
:103B6000C9D97C2CAFD1C6E748F28E039C42AAD1BA
:103B7000C1E72846084B9847D9E700BFB1220000AB
:103B80002133000008450200DC4702005D220100ED
:103B90003C480200B9220000513A000010B504462A
:103BA000034B9847FF212046024B984710BD00BFAA
:103BB000CD300000993A00002DE9F84304460F4645
:103BC0000026DFF888803546DFF8849005E0FF2185
:103BD0003846C8470136402E22D0F1B23846C04799
:103BE0008646E8B101790029F4D090F805C00CF0C0
:103BF000060C0023DAB2BCF1060F04BF0132D2B2C8
:103C00008A423ABFDEF8000050F822202A46944249
:103C1000DDD0002CDBD00133DAB28A42EAD3D9E717
:103C200000213846084B9847054650B1064E2946B4
:103C30002046FFF7C1FF29463846B0470546002811
:103C4000F5D1BDE8F88300BFE12D0000FD2F000095
:103C5000993A00002DE9F047804600200F4B984725
:103C6000C8B18146DFF840A00D4F0E4E09F1300576
:103C70002846D047044640B121464046B847214631
:103C80002846B04704460028F6D14846034B9847DB
:103C900081460028EAD1BDE8F08700BFB90F0100D6
:103CA000B93B0000BD1F0100A91F0100F8B5044683
:103CB0000D4681790068424B9847424B9847A1884E
:103CC00001F00F03082B19DC45B9B4F908203E4B6D
:103CD0009847A18820683D4B9847F8BDFF2D0AD032
:103CE000B4F90820B4F90C309B1A05FB03F502EB7C
:103CF000252212B2EBE7B4F90C20E8E70B2B43DCEA
:103D0000002D05DDFE2D05DDA289314B9847E0E74A
:103D10002289FAE7EDB2C5F1FF02637BDB08667A20
:103D2000F60802FB06F605FB036303EB032703EB30
:103D3000C713C3F3C457A389C3F345132689C6F336
:103D4000451602FB06F605FB036303EB032603EBB4
:103D5000C613C3F3C556237B03F01F0394F808E092
:103D60000EF01F0E02FB0EF205FB032505EB0523EB
:103D700005EBC315ED0D4FF0000265F3040266F389
:103D80004A1267F3CF22C0E70D2B12DC002D05DDB0
:103D9000FE2D05DD227B0F4B98479AE7227AFAE742
:103DA000227A237B9B1A05FB03F502EB2522D2B274
:103DB000F1E77F2DD4BFA268E268074B984788E7F8
:103DC000FD2F0000E7700000E1680000993A000054
:103DD000256A0000696B0000996C000030B583B063
:103DE00004460A4B984710B1002003B030BD084B81
:103DF000009340F6B12207490320074DA847224609
:103E00000023064806498847FEE700BFB1220000AC
:103E1000D8450200DC4702005D2201003C48020058
:103E2000B9220000F0B583B00D46064688B19D4B1F
:103E30009847002840F064819B4B0093ED229B49FA
:103E400003209B4CA047324600239A489A49884752
:103E5000FEE79A4B984748B9994B0093924BCF2273
:103E600092490220924CA0473446F5E13030954B00
:103E7000984704468B4B984760B98B4B0093D422EC
:103E80008A4903208A4DA847224600238E488A4942
:103E90008847FEE7002C00F0DF814C2120468B4B49
:103EA000984794F835306FF3051384F83530884B14
:103EB000E361884B23620027A76127826782384627
:103EC000854B98470138A0823846844B9847013883
:103ED000E0824C21201D824B98470023638684F8A2
:103EE000303084F8313084F84830A4F84430A4F8F5
:103EF0004630236494F8492063F3000284F8492093
:103F0000A36394F8342002F07F0242F0010294F897
:103F10003510032060F3430184F83C3002F0C10205
:103F200063F3861284F8342041F0010184F83510DF
:103F300084F83D30636204F128073846694B98479E
:103F4000002D00F06C8105F128013846664B98473A
:103F500005F10F0204F1180104F1100312F8010F2A
:103F600003F8010B8B42F9D1B5F93230638695F82D
:103F7000303084F8303095F8313084F8313095F8AD
:103F8000483084F84830B5F94430A4F84430B5F9E5
:103F90004630A4F846302B6C236495F8492094F8F9
:103FA000493062F3000384F84930AB69A36195F8A6
:103FB0003430DB0994F8342063F3C71284F83420DA
:103FC00095F8342094F8343062F3000384F83430E8
:103FD00095F83430C3F3400394F8342063F341027E
:103FE00084F8342095F83530C3F3420394F8352033
:103FF00063F3430284F8352095F83430C3F380032B
:1040000094F8342063F3820284F8342095F8343035
:10401000C3F3C003D2B263F3C30284F8342095F82B
:104020003430C3F30013D2B263F3041284F83420A3
:1040300095F83430C3F34013D2B263F3451284F8D9
:10404000342095F83430C3F38013D2B263F3861270
:1040500084F8342095F83C3084F83C3095F83520CD
:1040600094F8353062F3000384F83530A86B10B152
:1040700021461E4B984728461D4B9847002800F0C4
:10408000D980002E00F0DF8028461A4B984707465B
:104090002846194B9847024639462046174B984701
:1040A000C9E000BFB1220000EC450200DC4702007D
:1040B0005D2201003C480200B9220000E10E01002F
:1040C00038490200111F0100D83F0200372B0100C0
:1040D000055A000029540000ED0E0100150F0100E3
:1040E000F91E0100E9640000697100009D250000CF
:1040F0007D2C00009D2E0000FD2E00003D340000B0
:10410000301D574B98470446564B9847002847D0D8
:10411000002C00F0A1804C212046534B984726608C
:1041200094F835306FF3051384F835304F4BE36165
:104130004F4B23620020A061B6F912306382778A68
:104140004C4B9847322303FB00F35033B3F5A07F69
:1041500033DA01233B44E3822046474B984701284A
:104160003AD0B6F910302382378A0020414B984765
:10417000642303FB00F35033B3F5A07F4DDB002035
:104180003C4B9847642303FB00F350333B4A82FBCC
:104190000312DB17C3EBA2139BB23B44A38298E646
:1041A000374B0093F02237490320374DA84722466A
:1041B0000023364836498847FEE700202D4B9847B4
:1041C000322303FB00F350332C4A82FB0312DB172C
:1041D000C3EBA2139BB2BDE7B6F91430A382B78A32
:1041E0000020244B9847642303FB00F35033B3F5BE
:1041F000A07F10DB00201F4B9847642303FB00F3D4
:1042000050331E4A82FB0312DB17C3EBA2139BB28F
:10421000FB1A23825DE60123FAE70123BDE726B1FD
:10422000022120461B4B984705E001212046194BEF
:10423000984708E03EB1F36922460121304698478D
:104240002046154B9847154B00930D4B40F28712B3
:104250000C4901200C4DA847204603B0F0BD00BF1B
:10426000111F0100B1220000372B0100055A000088
:10427000295400003D0F0100DD3D000067666666C1
:10428000EC450200DC4702005D220100D83F02003D
:10429000B9220000E94101002133000088490200F1
:1042A0002DE9F04184B004460D461646324B98473E
:1042B00068B9324B009340F2E52231490320314D79
:1042C000A84722460023304830498847FEE7204669
:1042D0002F4B9847A8423FD020462E4B984702A923
:1042E00020462D4B9847731E628A1344E382204672
:1042F0002A4B9847012835D06B1E228A1344A3828B
:10430000E36902AA0221204698472046244B984799
:1043100018B1C56922460121A847261D3046214B08
:104320009847054668B14FF003081F4FEB6902AA92
:1043300041462846984729463046B8470546002852
:10434000F4D12046134B984794F8493013F0010FED
:104350000ED104B0BDE8F0812046144B9847B0421E
:10436000BAD1F6E7C5F10103A28A13442382C7E755
:1043700020460F4B9847ECE7B122000010460200A0
:10438000DC4702005D2201003C480200B922000027
:104390005D2F000021330000412E0000DD3D0000B4
:1043A0007D2C0000A91F0100BD1F0100AD2F0000E2
:1043B000E139000030B583B004460D460D4B9847F7
:1043C00068B90D4B009340F227320C4903200C4D85
:1043D000A847224600230B480B498847FEE72046A2
:1043E0000A4B98472A4601462046094B984703B096
:1043F00030BD00BFB122000034460200DC4702009D
:104400005D2201003C480200B92200005D2F00003F
:10441000A142000030B583B004460D460C4B9847CE
:1044200038B194F83C301D4214BF0120002003B085
:1044300030BD084B009340F6D72207490320074DB3
:10444000A84722460023064806498847FEE700BFE2
:10445000B12200005C460200DC4702005D22010040
:104460003C480200B922000030B585B004460D4634
:10447000114B984728B13F2D11D894F83D0005B055
:1044800030BD0E4B009340F6DE220D4903200D4D4A
:10449000A847224600230C480C498847FEE78DF8C0
:1044A0000C5000238DF80D3003AA09212046084B3B
:1044B00098479DF80D00E2E7B12200007046020027
:1044C000DC4702005D2201003C480200B9220000E6
:1044D000752B00002DE9F04F85B0174660B30D46EF
:1044E0004FEA122B0646DFF88CA0DFF88C90DFF83D
:1044F0008C8006E0BDF90E0005B0BDE8F08F002508
:10450000DEB129463046D047019029463046C8479B
:1045100007EB002084B20DF10E0221460198C0473E
:104520000128E7D01BF0800F07D0002DE7D13046DF
:104530000F4B98470646E2E7144624F4FE44A4B223
:10454000222C0FD006D8032C0AD0072C0CD14FF404
:104550008070D1E7312C09D0C02C05D11020CBE7D9
:104560000620C9E7FF20C7E70020C5E70F20C3E703
:104570007D2C0000FD2F000069440000E572000062
:104580002DE9F04F85B0174648B30D464FEA122B80
:104590000646DFF86CA0DFF86C90DFF86C8004E072
:1045A000BDF80C0025E00025D6B129463046D0479D
:1045B000019029463046C84707EB002084B203AA81
:1045C00021460198C0470128EAD01BF0800F07D090
:1045D000002DE8D13046084B98470646E3E71446DD
:1045E00024F4FE44293C012C9ABF044BB3F8740612
:1045F000002005B0BDE8F08F7D2C0000584002007F
:10460000FD2F000069440000A97300002DE9F04F60
:1046100085B0174650B30D464FEA122B0646DFF819
:1046200074A0DFF87490DFF8748004E09DF80F0048
:1046300029E00025DEB129463046D04701902946C1
:104640003046C84707EB002084B20DF10F02214627
:104650000198C0470128E9D01BF0800F07D0002D3A
:10466000E7D130460A4B98470646E2E7144624F461
:10467000FE44A4B26D2C09D048F2AD039C4205D093
:104680002C2C03D0FF2005B0BDE8F08F0020FAE706
:104690007D2C0000FD2F0000694400006D740000B7
:1046A0002DE9F04F85B0174650B30D464FEA122B57
:1046B0000646DFF880A0DFF88090DFF8808005E014
:1046C000039805B0BDE8F08F0025D6B129463046E5
:1046D000D047019029463046C84707EB002084B2F6
:1046E00003AA21460198C0470128E9D01BF0800F9A
:1046F00007D0002DE8D130460B4B98470646E3E73C
:10470000144624F4FE44A4B2BE2C0AD048F28E0310
:104710009C4203D07E2C01D00020D2E7034B984767
:10472000CFE70348CDE700BF7D2C0000DD4101004D
:1047300000920200FD2F0000694400003175000066
:1047400070B50468A58805F00F03082B13DD0B2B4B
:1047500018DD0D2B1DDD2A46A1792068104B9847E6
:10476000A0600023A38023462A46A17920680D4E2D
:10477000B047A58070BD2A46A17920680A4B9847AA
:104780002081EEE72A46A1792068084B98472081CE
:10479000E7E72A46A1792068054B98472072E0E7B1
:1047A000A146000029300000D544000081450000EA
:1047B0000D46000090F83D308B4200F052822DE90A
:1047C000F04FA1B089468246AB4B984740B19AF86A
:1047D0003DB08AF83D9000230693A84DD846D2E11B
:1047E000A74B009340F23762A6490320A64CA0478E
:1047F00052460023A548A6498847FEE7737943F04F
:10480000040373718AF83D802246DDF80CB05946E6
:104810005046A84707468AF83D902246CDF80CB08E
:1048200059465046A847834673796FF382037371E4
:1048300087424AD08AF83D80224603995046A847CD
:1048400006468AF83D90024621460498914B9847C7
:10485000012C00F094809048904B98470746864B77
:104860009847002800F0A280002F2ED03E81A7F8A4
:104870000CB0C7F800A0BC809DF80C30BB7110A82C
:10488000874B98471097874B1193874B1293874B11
:10489000139300231693FF2317930A9B1893099BE6
:1048A0005B421993089A531ED01D14AA13F8011FD6
:1048B00002F8011B8342F9D19DF876306FF30003B3
:1048C0008DF8763010A87A4B9847059B10AA934232
:1048D00000F05481059B33F8024B0593002CF4D073
:1048E0000798744B984703995046734B9847064670
:1048F000724B9847049004F00F03082B7FF77EAFAC
:104900000B2B61DD0D2B00F3E980737943F0040379
:1049100073718AF83D802246DDF80CB05946504646
:10492000674FB8470B908AF83D902246CDF80CB0FF
:1049300059465046B847834673796FF382037371C3
:104940000B9B8342C1D08AF83D8022460399504692
:10495000B84706468AF83D90024621460498594BCE
:1049600098474D484D4B98470746434B984700287A
:1049700074D0002FA9D03E7287F80CB079E747F6C3
:10498000FF739E4200F04C819B457FF464AF50461C
:10499000DFF844B1D84700EBD07040F34F075046E2
:1049A000D84700EBD07040F34F0351E1464B0093E2
:1049B00040F6B26233490320334CA0473A46002305
:1049C000424833498847FEE7737943F00403737123
:1049D0008AF83D802246039950463D4FB8478346AA
:1049E0008AF83D90224603995046B847ADF82C000E
:1049F00073796FF3820373711FFA8BFB83B29B454C
:104A00003FF463AF8AF83D80224603995046B84789
:104A100083468AF83D900246214604982D4B9847DC
:104A20001D481E4B98470746134B984740B1002F2F
:104A30003FF44BAFA7F808B0BDF82C30BB8118E7A6
:104A4000214B009340F6C6620E4903200E4CA0474E
:104A50003A4600231D480E498847FEE71A4B00934B
:104A600040F6DB6207490320074CA0473A46002383
:104A7000164807498847FEE7B1220000D5440000E8
:104A8000D0460200DC4702005D2201003C480200E3
:104A9000B9220000E16800003C6D0020111F0100F8
:104AA000E5120100AD3C000041470000213100004B
:104AB000A113010035720000FD2F0000E770000017
:104AC0000D460000696B0000E4460200D83F02007A
:104AD00081450000256A00005D2F00008AF83D80B6
:104AE000737943F0040373712246DDF80CB0594624
:104AF00050465C4FB8470C908AF83D902246CDF85E
:104B00000CB059465046B847834620A941F8400D9D
:104B100073796FF38203737104220CA8524B984788
:104B200000283FF4D2AE8AF83D80224603995046D1
:104B3000B84706460C908AF83D90024621460498F4
:104B40004A4B98474A484B4B984707464A4B984729
:104B500030B1002F3FF4B9AEBE60C7F80CB088E6A4
:104B6000464B009340F6EF6245490320454CA04771
:104B70003A460023444845498847FEE7069B0133EF
:104B80000693402B45D09DF81830039319465046A4
:104B90003F4B9847079000283BD0437913F0080F0C
:104BA000ECD1B022039C21465046A8470A90B1227E
:104BB00021465046A8470990BE2221465046294B1F
:104BC00098470890B22221465046A847ADF83400D5
:104BD000B32221465046A847ADF83600B4222146FC
:104BE0005046A847ADF83800B52221465046A847A0
:104BF000ADF83A00B62221465046A847ADF83C0031
:104C0000B72221465046A847ADF83E000DAB0593AC
:104C100060E6FF2150461F4B984721B0BDE8F08F5A
:104C200050461D4EB04700EBD07040F34F07504642
:104C3000B04700EBD07040F34F035E1C7A1C9642E5
:104C4000A8BF164636B247F6FF7293457FF403AE0F
:104C500003F1010B0137BB45A8BFBB460FFA8BFB25
:104C6000F9E57047A1460000DDB40100996C000031
:104C70003C6D0020111F0100B1220000E44602003B
:104C8000DC4702005D220100D83F0200B92200008B
:104C9000FD2F0000993A00005D2F000030B583B071
:104CA00005460C460D4B984750B195F83D3043EA08
:104CB00004018B4202D02846094B984703B030BD0F
:104CC000084B009340F27E6207490320074CA0473F
:104CD0002A460023064807498847FEE7B12200001C
:104CE000B5470000F4460200DC4702005D220100E7
:104CF0003C480200B922000030B583B005460C469E
:104D00000D4B984750B195F83D3023EA04018B4292
:104D100002D02846094B984703B030BD084B00939A
:104D200040F28F6207490320074CA0472A46002320
:104D3000064807498847FEE7B1220000B547000052
:104D400008470200DC4702005D2201003C480200E7
:104D5000B922000030B583B004460A4B984710B121
:104D6000E06903B030BD084B009340F6F5220749D7
:104D70000320074DA84722460023064806498847D6
:104D8000FEE700BFB12200001C470200DC47020022
:104D90005D2201003C480200B922000030B583B01A
:104DA00004460A4B984710B1606A03B030BD084B07
:104DB000009340F61E3207490320074DA8472246BC
:104DC0000023064806498847FEE700BFB1220000DD
:104DD00060470200DC4702005D2201003C480200FF
:104DE000B922000030B583B004460A4B984710B191
:104DF000A06B03B030BD084B009340F66F320749FB
:104E00000320074DA8472246002306480649884745
:104E1000FEE700BFB122000084470200DC47020029
:104E20005D2201003C480200B92200002DE9F84350
:104E30000546002215213C4B984728463B4B984796
:104E4000074610B128463A4B984700212846394B6F
:104E500098470023FF2211462846374CA04705F10A
:104E600004084046354B9847044658B1DFF8E890AF
:104E700021464046C84706462046FFF7D7FF34463E
:104E8000002EF5D12E4B5B683BB101211A6895428B
:104E900008BF19719B68002BF8D10020294B984757
:104EA000044610B3DFF8B480DFF8B490254E0EE06E
:104EB00029462046C047E36B9D4204BF0023E363BD
:104EC000A36D9F420AD02046B047044668B1636B89
:104ED0009D42EDD0A36B9D42EDD1E9E7C8478542E5
:104EE000F1D129462046C047EDE7EB690022114683
:104EF000284698472846144B984760B12946043005
:104F0000124B9847686A08B1114B98472846104BD6
:104F10009847BDE8F88328460E4B9847294630301D
:104F20000A4B9847EEE700BFCD2A0000E54D000090
:104F3000792600002913010029300000A91F010073
:104F40007C260020211001007D2C0000952001000E
:104F5000C5240100212D0000BD1F010075270000A0
:104F60000128000070B582B00446194B984768B913
:104F7000184B009340F2931217490320174DA8478E
:104F800022460023164817498847FEE72046164B5D
:104F900098472046154B9847054640B12046144B8C
:104FA0009847EB6900220121284698470CE02046EB
:104FB000104B9847054638B1C66B20460C4B9847B6
:104FC000B44201D10023EB63002002B070BD00BFEA
:104FD000B122000098470200DC4702005D22010078
:104FE0003C480200B9220000213300007D2C000063
:104FF0002D4E0000212D000030B583B004460E4B2D
:10500000984748B1A06BA8B10C4B9847844214BF95
:105010000020012003B030BD094B00934FF43862EB
:1050200008490320084DA84722460023074808499D
:105030008847FEE70020EDE7B12200004927000085
:10504000C8470200DC4702005D2201003C48020024
:10505000B922000000B583B090F83030028AD21A2D
:10506000ADF80020828A1344ADF8043090F8313056
:10507000428AD21AADF80220C28A1344ADF8063033
:1050800000226846024B984703B05DF804FB00BF5E
:10509000B915010003687BB110B4021D012352F859
:1050A000044B1CB10133DBB2072BF8D140F82310BD
:1050B00001205DF8044B7047002340F823100120C5
:1050C000704700002DE9F04105460E4614460122C6
:1050D000A84B9847208048F20C0231462846A64B40
:1050E0009847052842D90746237B002B49D1237DC9
:1050F000002B76D1237F002B40F0988094F8363037
:10510000002B40F0B88094F82830052B00F2018184
:1051100094F84430052B00F23781F92F24D8BFB220
:10512000237B13FB07F3C3F307232373237D13FBB5
:1051300007F3C3F30723237594F8283013FB07F311
:10514000C3F3072384F8283094F8363013FB07F3B1
:10515000C3F3072384F8363094F8443013FB07F781
:10516000C7F3072784F84470BDE8F0810023237358
:10517000237584F8283084F8363084F84430BDE84C
:10518000F0812C22314628467B4B98472073052816
:10519000ADD9292231462846784B98476080232292
:1051A00031462846734B9847C0B2A07130B92022CF
:1051B000314628466F4B9847607398E72A2231465C
:1051C00028466E4B9847A080212231462846DFF8BA
:1051D000A481C0472081222231462846C0476081F1
:1051E000E5E7302231462846624B98472082002866
:1051F00080D03C22314628465F4B984720750528D1
:1052000006D83222314628465A4B9847607571E7D6
:10521000312231462846574B9847C0B26082392226
:1052200031462846554B9847E081EAE7402231460F
:105230002846504B9847208300283FF45FAF4C220C
:10524000314628464C4B98472077052806D84222FD
:1052500031462846474B984760774FE74122314611
:105260002846444B98476083492231462846434BA1
:105270009847E082EBE76E2231462846404B98473C
:10528000E06200283FF43FAF6C22314628463A4B9B
:10529000984784F8360005287FF635AF6D223146F1
:1052A0002846354B984784F8370061223146284616
:1052B000304B9847003018BF012094F8383060F325
:1052C000000384F83830E06A2E4B984702280BD050
:1052D00094F83730052B15D8602231462846254BE7
:1052E000984784F839000EE7692231462846234B57
:1052F0009847A08648F28E0231462846204B9847B0
:105300002063E9E76922314628461C4B9847A0866E
:10531000E2E7502231462846164B98472084002861
:105320003FF4F6AE5C2231462846134B984784F88A
:10533000280005287FF6ECAE512231462846DFF8DA
:105340003480C0476084522231462846C047A0843A
:10535000532231462846C047E08459223146284628
:10536000064B9847E083542231462846C04784F8CC
:105370002900CDE6D54400000D460000814500001F
:10538000A1460000699900007F2231462846224B41
:105390009847E06300283FF4C0AE7C22314628469F
:1053A0001E4B984784F8440005287FF6B6AE73225A
:1053B00031462846DFF86C80C047A4F848007422C4
:1053C00031462846C047A4F84A007922314628468B
:1053D000134B9847A4F846007E22314628460E4BD0
:1053E00098472064702231462846C047A4F84C00F4
:1053F000712231462846C047A4F84E007522314636
:105400002846C04784F85000722231462846C047DB
:1054100084F8510081E600BFA14600000D4600005F
:1054200081450000D54400002DE9F04198B00446C4
:105430000E46022A08D0002A6CD0012A00F0CC8047
:10544000002018B0BDE8F08100218E4B984708B1CC
:105450000320F6E70122002120468A4DA84707468F
:10546000042200212046A84780460522002120462C
:10547000A84704F10F0304F1170503AA13F8011F4D
:1054800002F8011B9D42F9D11FFA88F8BDF80C30D3
:10549000A3EB0803ADF80C30BDF810309844ADF81C
:1054A000108080B2BDF80E301B1AADF80E30BDF87A
:1054B00012301844ADF812003A4603A93046724B38
:1054C000984708B90220BCE72C22002120466F4BE8
:1054D0009847F92801D80220B3E72022002120466E
:1054E000684B9847C0B208B10220AAE732220021D7
:1054F0002046644B9847C0B208B10220A1E748F2A9
:105500000C0200212046614B9847FA2834BF022044
:10551000012096E703A85E4B9847332200212046DE
:10552000584B984710B100238DF8203003AA002172
:105530002046584B9847042200212046514DA84749
:105540008046052200212046A84704F1100704F1F7
:105550000F0304F1170501AA13F8011F02F8011B3C
:10556000AB42F9D11FFA88F8BDF80430A3EB080369
:10557000ADF80430BDF808309844ADF8088080B22A
:10558000BDF806301B1AADF80630BDF80A301844D5
:10559000ADF80A0003AA314601A83F4B9847022202
:1055A00000212046374B984708B9002049E71C20C6
:1055B0003A4B98470546012200212046314B984737
:1055C0000023024639462846354EB04704F5187187
:1055D0002846344B9847E8E702220021294B984798
:1055E00038B9332200212046264B984740B9002085
:1055F00027E704F518702C4B98472C4B9847F0E799
:1056000003A8234B984700278DF818708DF8427037
:105610008DF8347003AA394620461E4B9847042261
:1056200039462046174DA847804605223946204670
:10563000A84704F10F03173401AA13F8011F02F859
:10564000011BA342F9D11FFA88F3BDF80420D21A36
:10565000ADF80420BDF808201344ADF8083080B23E
:10566000BDF806301B1AADF80630BDF80A301844F4
:10567000ADF80A0003AA314601A8074B984700205D
:10568000DFE600BFD54400006D1701000D460000A5
:1056900069C20000C550000031C300003D2901006F
:1056A0002DC00000C1BD000091BE000071250100A9
:1056B000F8B505460E46144648F28C02264B98472C
:1056C0002072052800D8F8BD48F20C023146284661
:1056D000214B9847F92805D8237A13FB00F0C0F333
:1056E00007202072237A052BEDD948F28902314632
:1056F00028461A4B9847208048F2800231462846B7
:10570000174FB847A08148F2810231462846B84772
:10571000608148F2820231462846B847207648F236
:10572000830231462846B847607648F28E023146F9
:1057300028460C4B98476060E2894FF6FF739A4207
:10574000C1D0228A9A42BED048F28A023146284607
:10575000024B98472080B6E70D46000081450000C7
:10576000D5440000A146000070B505460E4614461B
:1057700048F2AC02214B98472070052800D870BD34
:1057800048F20C02314628461C4B9847F92805D8A8
:10579000237813FB00F0C0F3072020702378052B3B
:1057A000EDD9002363804FF480732381AB8A0133EA
:1057B0002A8A9B1A1BB203EBD3735B10A380EB8A7C
:1057C00001336A8A9B1A1BB203EBD3735B10E3802D
:1057D00048F2AD0231462846084B9847A07248F27D
:1057E000A90231462846064B9847A08148F2A002FC
:1057F00031462846034B9847A073C0E70D4600008A
:1058000081450000D54400002DE9F04F89B00446E1
:105810000E465022764B9847074668BB7F2231469A
:105820002046744B9847804630B17C223146204652
:10583000714B984705284CD84022314620466C4B86
:1058400098470546002840F0BF8004223146204694
:10585000DFF89C81C0470546052231462046C047F7
:10586000A842B8BF284600B20028C4BFC01907B27A
:10587000384609B0BDE8F08F5C22314620465E4BC9
:105880009847052801D80027C8E75322314620460B
:10589000574DA84707EBD77700EB67070137BFB233
:1058A000512231462046A8478046522231462046A2
:1058B000A8470028B8BF4042B8F1000FB8BFC8F1F0
:1058C00000084045ACBF3F18474438B220EAE077B3
:1058D000A4E7702231462046454DA84782467022F3
:1058E00031462046A84783467E2231462046414B1A
:1058F00098474FF00009CDF8089047F618430193F8
:10590000CDF800B053460246414604A8DFF8EC80CB
:10591000C047ADF81890ADF81A90BDF81030013BB3
:10592000ADF81C30BDF81230013BADF81E307522C9
:1059300031462046A8478146732231462046A84773
:105940008046742231462046A847054605AB5FFADB
:1059500089F206A904F11000DFF8A490C847BDF849
:10596000143043449BB2BDF816202A4492B2B4F9D5
:105970001000BDF81810194409B2401AB842B8BF57
:105980003846B4F91210BDF81A7017443FB2CF1B55
:1059900000B28742B8BF0746BDF81C0003441BB2E3
:1059A000B4F91400181A3BB28342B8BF0346BDF8DD
:1059B0001E00104400B2B4F91670C71B18B2B842EA
:1059C000B8BF384607B237E74C22314620460A4B6B
:1059D000984705287FF639AF412231462046044BCF
:1059E00098472844B842B8BF384607B22DE700BFF1
:1059F000D5440000A14600000D4600007D40010096
:105A00002518010008291AD010B50446072920D00E
:105A1000012923D0062927D0032930D0042939D0E1
:105A20000B293BD0A1F10D03DBB2012B3BD9162989
:105A30003ED0172951D0002954D0012010BD137831
:105A40001BB92830506001207047002353600120AB
:105A5000704726491046264B984710BD254B98475E
:105A600080F00100C0B210BD0021234B9847B4F96B
:105A700032309842B8BF18466086012010BD90F8B9
:105A8000493013F0010F01D1012010BD1B4B984785
:105A9000012010BD1A4B9847012010BD1021194B51
:105AA0009847012010BD1021174B9847012010BDC9
:105AB000164B9847164B984728B106212046114BA4
:105AC0009847012010BD022120460E4B9847042123
:105AD00020460D4B9847012010BD06210A4B9847E0
:105AE000012010BD0B4B9847012010BDE849020072
:105AF000955000001544000009580000E1390000ED
:105B00002D2C00009D4C0000F94C0000E54D0000DC
:105B10005B270000CD3000002DE9F843054688469C
:105B2000002210311F4B984750B398F8343013F0CF
:105B3000100F27D1D8F8203043B30222294640461F
:105B40009847814603281FD008F104063046164BBB
:105B50009847044660B1154F21462846FFF7DCFF01
:105B6000034650B921463046B84704460028F3D1D1
:105B7000B9F1010F0CBF434600231846BDE8F88376
:105B80000023FAE70023F8E70023F6E708F104060C
:105B90003046054B984704464FF002090028DAD1F9
:105BA0000346EAE76D170100A91F0100BD1F0100B0
:105BB00090F8343013F0100F00D070472DE9F04307
:105BC0008BB00E460546B0F9324004A9354B9847D4
:105BD000A3B2BDF81020D21AADF81020BDF81220E3
:105BE000D21AADF81220BDF814201A44ADF81420D2
:105BF000BDF816201344ADF8163004AA314606A8A5
:105C0000294B9847A8B12B6A1BB1002206A9284648
:105C1000984704A92846234B984704AA314608A868
:105C2000214B984740B92B6A1BB1012206A928468F
:105C300098470BB0BDE8F08305F1040840461B4BC4
:105C4000984704460028EED0DFF85890164E184FBB
:105C500005E021464046B84704460028E3D002A9A3
:105C60002046C847638EBDF80820D21AADF8082038
:105C7000BDF80A20D21AADF80A20BDF80C201A444B
:105C8000ADF80C20BDF80E201344ADF80E3002AA7A
:105C900008A96846B0470028DBD069462046FFF7D0
:105CA00087FFD6E7412E000019150100B31F010040
:105CB000E91F01002DE9F0470F46044670B139464F
:105CC00020461A4B98472046194B9847814660B1A9
:105CD000184EDFF85880DFF858A00EE0164B186811
:105CE000164B984704460028E9D1BDE8F08748469E
:105CF000D0474C4681460028F7D009F104052146DB
:105D00002846B047044640B139462046C0472146A0
:105D10002846B04704460028F6D1D9F82030002B99
:105D2000E5D00122394648469847E0E7B15B0000DC
:105D30007D2C0000E91F0100882600204D23000073
:105D400038B51A4D28681A4B984704462868194BED
:105D5000984778B90123A361144B186843681A6AFD
:105D600012F0010F10D01B6A13F0020F0CD00123A8
:105D7000E3610BE00D4D2868A369002BEAD0C369ED
:105D8000002BF9D09847F6E70023E361C3681BB105
:105D9000A26804F110019847236833B1626822B108
:105DA000A1688B4208BF1346A36038BD8826002037
:105DB000DD0F0100E10F010070B582B006461A4DFB
:105DC00028681A4B984704462868194B984738B9F1
:105DD0002868A36923B1C369002BFAD09847F7E775
:105DE00004F1100231466846124B98470E4C206869
:105DF000114B984701466846104B98476946104D2D
:105E0000A84720680F4B98476946A84720680E4B63
:105E100098476946A84720680C4B984708B102B0DC
:105E200070BD0B4B9847FAE788260020DD0F010074
:105E3000E10F0100191501004D230000195B00005E
:105E4000B55C00008D230000CD230000F50F01009C
:105E5000415D000070470000F0B585B00C46054676
:105E6000002854D0002C57D00023ADF80830ADF8EE
:105E70000A302846364B98470138ADF80C002846C2
:105E8000344B98470138ADF80E0002AA2146684607
:105E9000314B9847002845D02B6913B169462846F5
:105EA0009847B5F86831C3F309039BB100210C464C
:105EB0000F462A4E09313A4605EBC1016846B04704
:105EC00080BB0134A4B22146B5F86831C3F309039D
:105ED0009C42EFDB1F2B27DC093305EBC3030DF1DD
:105EE000FF3203F1080012F8011F03F8011B83427F
:105EF000F9D1B5F86831C3F30902013262F309033D
:105F0000A5F868310321E86A154B98470AE0154B5C
:105F10009847054630B1A5E7B5F868316FF3090336
:105F2000A5F8683105B0F0BDB5F868316FF3090325
:105F3000A5F868310DF1070205F1500005F148039D
:105F400012F8011F03F8011B8342F9D1D1E700BF0A
:105F5000ED0E0100150F0100191501006D1701006C
:105F600059390100E10E0100014B1868704700BF6C
:105F7000882600202DE9F04F8DB00546B74B984795
:105F80000990B74CEB68236000212846B54B984731
:105F90002068C36B7BB1B0F86831C3F30903002BF1
:105FA00000F078824FF048080027AD4DDFF8E4A2FA
:105FB000DFF8C8B24DE0B0F868316FF30903A0F81C
:105FC000683162E22644012386F8483101342868AA
:105FD000B0F86831C3F309039C4230D2031993F837
:105FE0004831002BF2D1A742F0D004F10906F600A7
:105FF00081194044D0470028E8D029688A194144D3
:106000000AA8994B98470AA8D847039028684044A3
:10601000D847814628683044D8474844039B834288
:10602000D4D22E6806EB08030DF1270203F1080015
:1060300012F8011F03F8011B8342F9D1C2E70137AF
:106040002868B0F86831C3F3090308F108089F42D3
:106050000ED2384490F84831002BF0D12868B0F8BF
:106060006831C3F30903002B00F0FA810024B5E77F
:1060700000217B4A5160002B00F0FA815A1E114624
:10608000079232D4821892F848217AB103F247136A
:1060900003440A46013AB2F1FF3F05D013F8011D4F
:1060A0000029F7D1079201E000230793426892F894
:1060B00020306FF3000382F82030426892F82030DD
:1060C0006FF3410382F82030654B1C68B4F86831E7
:1060D000C3F30903002B00F0CB81482306934FF054
:1060E000000ADFF87CB1274645E000230793DDE78F
:1060F0007A6892F8203043F0010382F8203043E0C0
:10610000DBF80000594B9847044600250582DBF870
:106110000000574B98470138A0826582DBF80000E9
:10612000544B98470138E082DBF800305A6892F807
:10613000203043F0020382F8203003984E4B9847FA
:10614000DBF80000836943B1069B18444B4B98472A
:10615000DBF804300344CBF804300AF1010ADBF821
:106160000070069B08330693B7F86831C3F3090340
:106170009A4580F27D8107EB0A0393F84831002BA2
:10618000EBD1079B5345B3D07A6892F820306FF378
:10619000410382F82030069BFB1803933846384BA6
:1061A00098470028ACD1DBF80000304B98470646F2
:1061B00007EBCA07B7F84C400134B7F84830E41A87
:1061C00024B2B7F94E5005F10108B7F84A30A8EBF0
:1061D00003080FFA88F8DBF80000264B9847854241
:1061E00034DAB7F94E90F368B3FBF4F39845A8BFDF
:1061F0009846DBF800301B69002B52D00023ADF825
:106200002830ADF82C30ADF82A300FFA88F56C1E26
:1062100024B2ADF82E40DBF8000003690AA99847C4
:10622000BDF92E104B1CBDF82A209B1A1BB29845B5
:1062300032DA2546002CEADC124B0093124B40F276
:106240009F1212490220124CA04779E7DBF80000A8
:10625000084B984701380FFA80F9C4E7591001003C
:1062600088260020593901006F150100DD0F01005B
:10627000ED0E0100150F0100B95D0000FD140100D5
:10628000F50F01002C4A0200F0490200004A02000A
:106290005D22010029170100002DC8BF01F101088E
:1062A000CADDB7F94A40CDF8109004EB0803013B72
:1062B0004B454BDC1FFA88F30593013BCDF820A03A
:1062C0009A460DE0A9451CD00398784B9847059B4A
:1062D0001C4424B204EB0803013B049A93421ADCE9
:1062E000B7F948303382B7F94C30B3827482A4B224
:1062F00004EB0A052DB2F582A945E3DAA6F816905B
:106300004D46DBF800305A6892F8203043F0020323
:1063100082F82030D8E7DDF820A0A9453FF410AF7F
:10632000B7F948303382B7F94C30B3827482A6F89B
:106330001690DBF800305A6892F8203043F00203E0
:1063400082F820300398594B9847F9E60025E4E796
:10635000574B984718B1574B18684369EBB1554CE8
:1063600020684FF480714830534DA84720682021A1
:1063700000F5A470A8472368B3F868216FF30902F9
:10638000A3F8682109984D4B984701462068836916
:10639000002B76D06268984773E0494B98470446D3
:1063A000484B9847A369002BFCD1A3680393D4F80A
:1063B00000A0534508BFD4F804A03E4C2068424BCF
:1063C000984704902368B3F86821C2F30902002AB1
:1063D000C5D0450000229046A1460CE008F1010816
:1063E0001FFA88F84246D9F80030B3F86811C1F3B3
:1063F00009018845B3DA991891F848110029EDD1BF
:1064000003EBC203B3F94A70B3F94810049807FBD1
:1064100000167600B3F84C3001335B1A1BB25B00F8
:106420000593D9F8003003EBC203B3F94E30BB42F9
:10643000D4DB039B03EB060B56440932D400059AC8
:1064400031465846214B984701373FB2AB442E4462
:10645000D9F800302344B3F90630BB42EFDABDE788
:106460000022144B5A60B0F86831C3F309037BB9BA
:10647000104B1868B0F86831C3F30903002B7FF4A0
:1064800067AF134B9847134B98470DB0BDE8F08F9B
:1064900007920BE60022074B5A60B0F86831C3F34D
:1064A0000903002BEDD0079200E600BFB95D0000A4
:1064B000F50F010088260020372B01007110010024
:1064C000DD0F0100415D0000ED0E010055260100C9
:1064D000F9250100F50C010008B50421014B98478E
:1064E00008BD00BF372B010008B50821014B9847B4
:1064F00008BD00BF372B010070B582B00679002EB1
:1065000055D004460068036899420AD00346751EB8
:10651000EDB200EB85059D4249D053F8042F8A4225
:10652000F9D10D46012E0ED0711E8900214B9847DE
:106530000646214B984780B1EEB12179002933D02E
:106540000022134626E01D4B984700232360237149
:10655000627963F30002627129E0194B00934FF4F2
:10656000827218490320184CA0473246002317486E
:1065700017498847FEE7174B0093114B4FF483727E
:1065800010490220104CA04711E00133DBB2217901
:10659000994209D9216851F823108D42F5D046F867
:1065A00022100132D2B2F0E701392171266002B027
:1065B00070BD00BF99280100B1220000C524010070
:1065C0007C4A02003C4B02005D220100D83F0200E1
:1065D000B9220000684B0200002851D070B582B08B
:1065E00004460E46274B9847237963BB0420264B6D
:1065F000984705462846254B984758B3002D36D076
:106600006379C3F3400013F0010F18BF0130237901
:10661000984210D205EB830103F18042013A013B1D
:106620001B1ADBB2D31A05EB830351F8042C41F893
:1066300004299942F9D145F8206023790133237167
:10664000256002B070BD013399002068104B984757
:106650000546CFE70F4B0093D0220F4903200F4C84
:10666000A0472A4600230E480E498847FEE70E4BF6
:106670000093084BD22208490220084CA047E0E7CB
:10668000704700BFF9640000DD230100B122000063
:1066900099280100984A02003C4B02005D2201004B
:1066A000D83F0200B9220000A44B020030B583B0ED
:1066B000437913F0010F10D003F00603062B14BF2B
:1066C000002301230279002A34D09A4234D9026887
:1066D00052F82340204603B030BD05460420174B36
:1066E00098470446164B984760B1CCB12046154BED
:1066F000984721462846144B98476B7943F001038D
:106700006B71E7E7114B009340F2354210490320CB
:10671000104DA847224600230F4810498847FEE73E
:106720000F4B0093094B40F2374209490220094DB3
:10673000A847CFE70024CDE70024CBE7DD23010005
:10674000B1220000D9640000D9650000B44A0200FB
:106750003C4B02005D220100D83F0200B92200003C
:10676000D44B020010B504460068024B9847002342
:10677000236010BDC52401000268D2B11378FF2B3D
:1067800013D0002006E00B2B0ADC02300230135C31
:10679000FF2B0BD003F00F03082BF4DC0230F5E7DE
:1067A0000D2BD4BF01300430F0E70020023080B25E
:1067B000704700207047000081B170B50C460A6830
:1067C0005AB105460846064B98470646054B98477A
:1067D000286032462168044B984770BD704700BF5F
:1067E00079670000DD2301005526010000286BD0E9
:1067F0002DE9F8430746006800286AD0CDB20E0A9A
:10680000B4460378FF2B3BD04FF0FF3EF04600220A
:10681000CCF3060C27E08418647886EA040919F0A2
:106820007F0F0BD004F07F0434EA0C091DD14445DE
:10683000C4BF0FFA84F80FFA82FE16E09646BEF146
:10684000000F43DB7446704443785E4016F07F0FC0
:1068500019D00020BDE8F8830B2B0CDC0232023289
:10686000835CFF2BEBD09D42D5D003F00F03082BA8
:10687000F2DC0232F3E70D2BD4BF01320432EEE733
:106880004FF0FF3EDBE70D463846134B984705F0C7
:106890000F010B2904DD0E29B4BF0321062100E0FE
:1068A00004210D46411A8C4207D223463A685419F6
:1068B000E45CD45401338B42F8D13868074B9847D5
:1068C00038600120BDE8F883002070470020BDE853
:1068D000F8830020BDE8F88379670000992801005B
:1068E0002DE9F04186B0ADF80E10ADF80C2004682B
:1068F000002C48D0CFB20D0AAE462378FF2B2CD007
:106900004FF0FF3188460022CEF3060E18E0A6189D
:10691000767885EA060C1CF07F0F21D006F07F0602
:1069200036EA0E0C0ED14645C4BF0FFA86F811B2F6
:1069300008E00B2B0CDC02320232A35CFF2B0ED0E2
:106940009F42E4D003F00F03082BF2DC0232F3E79E
:106950000D2BD4BF01320432EEE74FF0FF310A466F
:10696000002A10DBA3185B785D4015F07F0F0AD179
:106970000232A3189DF80C10A1549DF80D205A70F6
:1069800006B0BDE8F0810646FF23ADF816301D4B7A
:106990009847002808BF0220051DADB229462046B1
:1069A000194B98473060194B9847E8B1002EE7D053
:1069B000AB1F3268D1189DF80E00D0549DF80F30EF
:1069C0004B702B1F3268D1189DF80C00D0549DF8E5
:1069D0000D304B70023D33685A199DF81610595509
:1069E0009DF817305370CBE7094B00934FF4C372F7
:1069F00008490320084CA04732680023074808498B
:106A00008847FEE77967000099280100B12200005D
:106A1000CC4A02003C4B02005D220100D83F02003C
:106A2000B92200002DE9F04186B0ADF80C20ADF898
:106A30000E100468002C48D0CFB20D0AAE46237861
:106A4000FF2B2CD04FF0FF3188460022CEF3060EEC
:106A500018E0A618767885EA060C1CF07F0F21D086
:106A600006F07F0636EA0E0C0ED14645C4BF0FFA7B
:106A700086F811B208E00B2B0CDC02320232A35C68
:106A8000FF2B0ED09F42E4D003F00F03082BF2DC63
:106A90000232F3E70D2BD4BF01320432EEE74FF0A0
:106AA000FF310A46002A10DBA3185B785D4015F021
:106AB0007F0F0AD10232A3189DF80C10A1549DF843
:106AC0000D205A7006B0BDE8F0810646FF23ADF8F0
:106AD00016301D4B9847002808BF0220051DADB297
:106AE00029462046194B98473060194B9847E8B122
:106AF000002EE7D0AB1F3268D1189DF80E00D0549D
:106B00009DF80F304B702B1F3268D1189DF80C0088
:106B1000D0549DF80D304B70023D33685A199DF8E2
:106B2000161059559DF817305370CBE7094B009359
:106B300040F2B51208490320084CA04732680023F0
:106B4000074808498847FEE779670000992801004F
:106B5000B1220000E04A02003C4B02005D2201002D
:106B6000D83F0200B92200002DE9F04387B0ADF80C
:106B70000E100468002C43D05FFA81FE0D0AAC466B
:106B80002378FF2B2CD04FF0FF37B8460021CCF3F1
:106B9000060C18E06618767885EA060919F07F0F6A
:106BA00021D006F07F0636EA0C090ED14645C4BF57
:106BB0000FFA86F80FB208E00B2B0CDC0231023121
:106BC000635CFF2B0ED09E45E4D003F00F03082B2F
:106BD000F2DC0231F3E70D2BD4BF01310431EEE7D3
:106BE0004FF0FF37394600290ADB63185B785D40B8
:106BF00015F07F0F04D121448A7007B0BDE8F083FF
:106C000017460646FF23ADF816301B4B9847002861
:106C100008BF0220C51CADB229462046174B984735
:106C20003060174B9847C0B1002EE6D06B1F32681A
:106C3000D1189DF80E00D0549DF80F304B7033687A
:106C40002B4403F8037C023D33685A199DF8161053
:106C500059559DF817305370CFE70A4B00934FF406
:106C6000F27209490320094CA04732680023084802
:106C700008498847FEE700BF7967000099280100AE
:106C8000B1220000F44A02003C4B02005D220100E8
:106C9000D83F0200B92200002DE9F04186B00292EF
:106CA000ADF80E100468002C4ED0CFB20D0AAE46DF
:106CB0002378FF2B2CD04FF0FF3188460022CEF3F3
:106CC000060E18E0A618767885EA060C1CF07F0FF1
:106CD00021D006F07F0636EA0E0C0ED14645C4BF21
:106CE0000FFA86F811B208E00B2B0CDC02320232EC
:106CF000A35CFF2B0ED09F42E4D003F00F03082BC0
:106D0000F2DC0232F3E70D2BD4BF01320432EEE79E
:106D10004FF0FF310A46002A16DBA3185B785D406E
:106D200015F07F0F10D10232A3189DF80810A1545E
:106D30009DF809205A709DF80A209A709DF80B2042
:106D4000DA7006B0BDE8F0810646FF23ADF81630D4
:106D5000204B9847002808BF0220851DADB2294668
:106D600020461D4B984730601C4B984720B3002E9F
:106D7000E7D0A5F108033268D1189DF80E00D05471
:106D80009DF80F304B70AA1F31688B189DF80800D2
:106D900088549DF809205A709DF80A209A709DF831
:106DA0000B20DA70023D33685A199DF816105955B8
:106DB0009DF817305370C4E7094B009340F213223B
:106DC00008490320084CA0473268002307480849B7
:106DD0008847FEE77967000099280100B12200008A
:106DE000084B02003C4B02005D220100D83F02002C
:106DF000B922000000284DD02DE9F04384460468F4
:106E0000002C4AD0CEB2090A8E462378FF2B3ED002
:106E10004FF0FF37B8460020CEF3060E2AE02518C3
:106E20006D7881EA050919F07F0F0AD005F07F051A
:106E300035EA0E0920D14545C4BF0FFA85F807B2DF
:106E40001AE00746002F2CDBBB1CE018E35C137034
:106E500043785370DCF8000007447878C1F30601EA
:106E60000840BDE8F0830B2B0CDC02300230235CC1
:106E7000FF2BE7D09E42D2D003F00F03082BF2DCA9
:106E80000230F3E70D2BD4BF01300430EEE74FF0B2
:106E9000FF37D7E74FF0FF3070474FF0FF30BDE8C6
:106EA000F0834FF0FF30BDE8F08300284AD02DE991
:106EB000F04386460468002C47D0CEB2090A8C46BF
:106EC0002378FF2B3BD04FF0FF37B8460020CCF3A0
:106ED000060C27E025186D7881EA050919F07F0F67
:106EE0000AD005F07F0535EA0C091DD14545C4BF20
:106EF0000FFA85F807B217E00746002F29DB3C445C
:106F0000A3781370DEF8000007447878C1F3060117
:106F10000840BDE8F0830B2B0CDC02300230235C10
:106F2000FF2BEAD09E42D5D003F00F03082BF2DCF2
:106F30000230F3E70D2BD4BF01300430EEE74FF001
:106F4000FF37DAE74FF0FF3070474FF0FF30BDE812
:106F5000F0834FF0FF30BDE8F08300284DD02DE9DD
:106F6000F04384460468002C4AD0CEB2090A8E460B
:106F70002378FF2B3ED04FF0FF37B8460020CEF3EA
:106F8000060E2AE025186D7881EA050919F07F0FB1
:106F90000AD005F07F0535EA0E0920D14545C4BF6A
:106FA0000FFA85F807B21AE00746002F2CDBBB1C4E
:106FB000E018E35C137043785370DCF8000007447A
:106FC0007878C1F306010840BDE8F0830B2B0CDC98
:106FD00002300230235CFF2BE7D09E42D2D003F078
:106FE0000F03082BF2DC0230F3E70D2BD4BF013086
:106FF0000430EEE74FF0FF37D7E74FF0FF30704730
:107000004FF0FF30BDE8F0834FF0FF30BDE8F08374
:10701000002850D02DE9F04307460468002C4DD0DD
:10702000CEB2090A8C462378FF2B2DD04FF0FF3EBD
:10703000F0460020CCF3060C19E025186D7881EAA3
:10704000050919F07F0F22D005F07F0535EA0C09FC
:107050000FD14545C4BF0FFA85F80FFA80FE08E04E
:107060000B2B0CDC02300230235CFF2B0ED09E4237
:10707000E3D003F00F03082BF2DC0230F3E70D2B13
:10708000D4BF01300430EEE74FF0FF3E70460028D9
:1070900018DB054601302318141D13F8010F02F800
:1070A000010B9442F9D13B682B445878C1F3060197
:1070B0000840BDE8F0834FF0FF3070474FF0FF30DD
:1070C000BDE8F0834FF0FF30BDE8F083437913F063
:1070D000010F06D013F0020F036814BF5868186838
:1070E000704700207047437913F0020F1ABF0368FE
:1070F000186800207047000000282CD038B50446DE
:10710000437913F0010F08D0134B9847054620B17F
:10711000124B98472846124B9847637913F0020F99
:1071200009D020460F4B9847054620B10B4B984796
:1071300028460B4B984723794BB9002222602271D5
:10714000637903F0FC0362F38203637138BD206846
:10715000034B9847F1E77047CD700000656700006A
:10716000C5240100E770000070B505460C462C4BA5
:1071700098472368002B41D0637913F0010F20D189
:1071800013F0020F10D0207901388000254B98476A
:1071900028602279013A216892000431224B9847F5
:1071A0002379013B2B7170BD207980001D4B9847DE
:1071B00028602279920021681B4B984723792B7114
:1071C00070BD13F0020F1AD0207902388000154BE1
:1071D000984728602279023A216892000831124BC0
:1071E00098472379023B2B712846104DA847064645
:1071F0002046A847014630460D4B984770BD207980
:1072000001388000074B984728602279013A2168AD
:1072100092000431044B98472379013B2B71E3E73B
:10722000F9700000DD23010055260100AD66000065
:10723000B967000030B583B00446437913F0020FFC
:1072400005D01D4B98470546284603B030BD0420A5
:107250001A4B984705461A4B9847A8B115B32846CC
:10726000184B984729462046174B9847637943F0B7
:107270000203637113F0010FE6D023681A6859689E
:10728000196023685A60DFE7104B009340F2CD226B
:107290000F4903200F4CA0472A4600230E480F49F0
:1072A0008847FEE70E4B0093084B40F2CF22084977
:1072B0000220084CA047C7E7E7700000DD2301006B
:1072C000B1220000D9640000D96500001C4B020007
:1072D0003C4B02005D220100D83F0200B9220000B1
:1072E000044C0200002859D02DE9F04F83B0054628
:1072F0000368002B54D04FEA11280023ADF8063064
:107300000079002842D0934689461C464FF0FF364C
:107310009A46244F1CE050460DF106024946B847F4
:10732000804527D06B7913F0020F05D0002803DBCE
:1073300014B913F0040F23D0B04204DDBDF80630B9
:10734000ABF800300646013424B2287984421FDAB3
:10735000E2B26B7903F00603062B04BF0132D2B20E
:107360000028D8D0824203D22B6853F82200D3E7FA
:107370005046D1E7BDF80630ABF8003001200AE0F6
:10738000BDF80630ABF80030012004E04FF0FF36C6
:10739000F043C0F3C03003B0BDE8F08F0020704769
:1073A0000020F8E7F56D0000002858D02DE9F04FD7
:1073B00083B005460368002B53D04FEA1128002301
:1073C000ADF804300079002841D0934689461C4628
:1073D0004FF0FF369A46244F1BE0504601AA49461B
:1073E000B847804527D06B7913F0020F05D00028ED
:1073F00003DB14B913F0040F23D0B04204DDBDF851
:107400000430ABF800300646013424B228798442B7
:107410001FDAE2B26B7903F00603062B04BF0132D8
:10742000D2B20028D9D0824203D22B6853F822006E
:10743000D4E75046D2E7BDF80430ABF80030012065
:107440000AE0BDF80430ABF80030012004E04FF052
:10745000FF36F043C0F3C03003B0BDE8F08F00202A
:1074600070470020F8E700BF5B6F0000002859D08C
:107470002DE9F04F83B005460368002B54D04FEA46
:10748000112800238DF807300079002842D0934658
:1074900089461C464FF0FF369A46244F1CE0504662
:1074A0000DF107024946B847804527D06B7913F0A4
:1074B000020F05D0002803DB14B913F0040F23D00A
:1074C000B04204DD9DF807308BF8003006460134E9
:1074D00024B2287984421FDAE2B26B7903F0060302
:1074E000062B04BF0132D2B20028D8D0824203D288
:1074F0002B6853F82200D3E75046D1E79DF80730B8
:107500008BF8003001200AE09DF807308BF800303E
:10751000012004E04FF0FF36F043C0F3C03003B069
:10752000BDE8F08F002070470020F8E7AB6E000048
:10753000002852D02DE9F04F83B005460368002B98
:107540004DD04FEA1128007900283ED09346894655
:1075500000244FF0FF36A246224F1AE0504601AAFF
:107560004946B847804526D06B7913F0020F05D005
:10757000002803DB14B913F0040F21D0B04203DD5F
:10758000019BCBF800300646013424B228798442AE
:107590001DDAE2B26B7903F00603062B04BF013259
:1075A000D2B20028DAD0824203D22B6853F82200EC
:1075B000D5E75046D3E7019BCBF80030012009E026
:1075C000019BCBF80030012004E04FF0FF36F04380
:1075D000C0F3C03003B0BDE8F08F0020704700203A
:1075E000F8E700BF11700000F0B501F01F0EC1F305
:1075F0004516C1F3C421052A3FD9C0F3C4240C4465
:107600001F2C28BF1F2404F01F04C0F3451333446C
:107610003F2B28BF3F2303F03F0500F01F007044BD
:107620001F2828BF1F2000F01F03FF2A2ED0C2F101
:10763000FF0707FB0EF002FB030000EB002300EB4B
:10764000C310C30D4FF0000063F3040007FB06F303
:1076500002FB053303EB032503EBC513DB0D63F3DB
:107660004A1007FB01F102FB041202EB022302EBBA
:10767000C312D20D62F3CF20F0BD4FF000006EF3C5
:10768000040066F34A1061F3CF20F0BD4FF0000014
:1076900063F3040065F34A1064F3CF20F0BDF0B546
:1076A00001F01F0EC1F34516C1F3C421052A3DD9CF
:1076B000C0F3C4240C1B24EAE47404F01F04C0F3D8
:1076C0004513F31A23EAE37303F03F0500F01F00AC
:1076D000AEEB000020EAE07000F01F03FF2A2ED07E
:1076E000C2F1FF0707FB0EF002FB030000EB0023D3
:1076F00000EBC310C30D4FF0000063F3040007FB61
:1077000006F302FB053303EB032503EBC513DB0D87
:1077100063F34A1007FB01F102FB041202EB0223A0
:1077200002EBC312D20D62F3CF20F0BD4FF0000088
:107730006EF3040066F34A1061F3CF20F0BD4FF002
:10774000000063F3040065F34A1064F3CF20F0BD3A
:107750002DE9F04F93B09DF870409DF874B09DF8FE
:107760007890BBF1040F00D914B913B0BDE8F08FC5
:107770000893ADF824200E460546BA4B984780463C
:10778000B94B98470746826806923246294610A8A8
:10779000B64B98470028E8D03A8ABDF840309B1A8B
:1077A00099B20D460A9108B20B90ADF840007B8A61
:1077B000BDF84210C91A0FFA81FCADF842C0BDF8FD
:1077C0004400801A80B2ADF84400BDF846E0AEEB4C
:1077D000030E0FFA8EFEADF846E0089AAAB198F8AB
:1077E000083013F0010F10D1411C491B09B20029C8
:1077F0000BDD134611441A78802A4FF0FF3298BFF0
:10780000002203F8012B8B42F5D1D8F81430002B5D
:1078100077D0BDF82480934B98470546BB8A013347
:107820003A8A9B1A1BB20793012C3ED0BDF9402027
:10783000089B9F1ABDF8443001339B1A1BB2089372
:10784000BDF942A0BDF946309A458EDCBDF94060D5
:107850003446BDF944309E421EDC3E440FFA8AF99C
:1078600005964B46B9461F46059A12F8013B05920C
:1078700003FB0BF3C3F307230293ADF804800097D7
:1078800023B2079A069928466E69B0470134BDF9BC
:1078900044309C42E8DD4F46089B1F440AF1010A30
:1078A000BDF946309A45D1DD5FE7BDF94290BDF99B
:1078B000463099453FF759AFDDF81CA05E46DDF82C
:1078C00018B0BDF94040BDF944309C4212DC0FFABB
:1078D00089F705970296ADF80480059B009323B2C3
:1078E0005246594628466F69B8470134BDF94430BD
:1078F0009C42EFDD09F10109BDF946309945E0DD13
:1079000033E7B9F1000F40F0A083BDF82430ADF8A3
:107910001C30544B98470646BB8A01333F8ADF1B15
:107920003FB2BDF94020BDF8443001339B1A1BB271
:107930000B931D46BDF94600BDF94230411CC91AE2
:1079400009B20C910A9303FB0722069901EB42014D
:107950000591012C29D0BBF1FA0F00F20881834276
:107960003FF703AF069B33F81230BDF82460C6F32F
:10797000C42CC6F34512104606F01F0214467A00C6
:107980000C920B9A08990139069152000E921946F1
:107990004FF0000E7246B6B20896CDF824B00D95A1
:1079A000A146CDF81CB0834645E3BBF1FA0F25D9BB
:1079B000736A23B110A82E4B9847F02813D80C9B5C
:1079C000002B7FF7D2AE7F0000242A4DDDF83080F7
:1079D000059E0B9ABDF81C103046A8473E44013462
:1079E000A045F6D1C1E6BDF82430ADF80030746A88
:1079F00010AB3A4606993046A047B6E6336A002BEC
:107A00003CD010A81A4B9847F02837D90B99002979
:107A10000CDDBDF82480184A931E01F100410139A4
:107A200002EB410223F8028F9A42FBD1BDF942508A
:107A3000BDF946309D423FF798AE4FEA4708DFF860
:107A400038A0DDF814905C4600940B9B52464946E2
:107A50003046376AB847C1440135BDF946309D42CA
:107A6000F2DD82E6695F0000DD0F010019150100FB
:107A7000FD1401003B1B0100902600204FF0000E7A
:107A8000BDF8242002F01F09C2F34518C2F3C42C2C
:107A90000BFB0CF303EB032103EBC113C3F3C45142
:107AA0000BFB08F303EB032403EBC413C3F3C5542C
:107AB0000BFB09F303EB032203EBC213C3F3C45222
:107AC0001FFA8BF30CFB03FC08FB03F809FB03F91B
:107AD0006FEA0B03DBB20C9800287FF746AE780004
:107AE00007900B9840000890002006909FB236E067
:107AF000307862F304003070308864F34A103080CC
:107B0000000A61F3C700707002339B451CD01E460B
:107B10001FFA8EF0B3F800A05045E9D0B3F800E0AA
:107B20005978C90801FB07C1C1F30421CEF34514FC
:107B300004FB0784C4F305241A7802F01F0202FB39
:107B40000792C2F30422D3E7059B079803440593E9
:107B5000069B013306930C9898423FF406AE002D25
:107B6000F2DD05980346089E00EB060BCFE70C9B61
:107B7000002B7FF7FAAD0B9B043B0D937B000F931B
:107B800000230A93BDF81C20C2F3C42CC2F3451E87
:107B9000C2F304030693DEE1BDF81C303B8043468C
:107BA00001318D4200F04C83023718F0030F00F0D2
:107BB000558318F8013B002BF1D0FF2BECD0C3F11B
:107BC000FF097A78D20809FB02F203FB0C2202EBD0
:107BD000022002EBC012C2F3C4523888C0F3451031
:107BE00009FB00F003FB0E0000EB002600EBC610C3
:107BF000C0F3C5503E7806F01F0A09FB0AF903FBE3
:107C0000049303EB032903EBC913DB0D63F30406B1
:107C10003E703B8860F34A133B801B0A62F3C70344
:107C20007B70BCE7BDF81C4020F8064C20F8044CE3
:107C300020F8024C04800431043308308F42C0F233
:107C400029811A4653F8044C002CF4D0B4F1FF3FBC
:107C5000E8D013F8048CB8F1000F3FD0B8F1FF0F53
:107C600000F00581C8F1FF0610F8054CE40806FB9A
:107C700004F408FB0C4404EB042504EBC514C4F322
:107C8000C454099430F8065CC5F3451506FB05F5A8
:107C900008FB0E5505EB052905EBC915C5F3C555C0
:107CA00010F8069C09F01F0B06FB0BF6069C08FB60
:107CB000046808EB082608EBC616F60D66F30409FF
:107CC00000F8069C30F8066C65F34A1620F8066C3E
:107CD000360A099C64F3C70600F8056C12F8038C99
:107CE000B8F1000F3FD0B8F1FF0F00F0C580C8F128
:107CF000FF0610F8034CE40806FB04F408FB0C44F0
:107D000004EB042504EBC514C4F3C454099430F8FF
:107D1000045CC5F3451506FB05F508FB0E5505EBA0
:107D2000052905EBC915C5F3C55510F8049C09F0E4
:107D30001F0B06FB0BF6069C08FB046808EB0826E5
:107D400008EBC616F60D66F3040900F8049C30F83B
:107D5000046C65F34A1620F8046C360A099C64F337
:107D6000C70600F8036C12F8028CB8F1000F3FD080
:107D7000B8F1FF0F00F08580C8F1FF0610F8014C44
:107D8000E40806FB04F408FB0C4404EB042504EBB4
:107D9000C514C4F3C454099430F8025CC5F3451506
:107DA00006FB05F508FB0E5505EB052905EBC91586
:107DB000C5F3C55510F8029C09F01F0B06FB0BF626
:107DC000069C08FB046808EB082608EBC616F60DAF
:107DD00066F3040900F8029C30F8026C65F34A1659
:107DE00020F8026C360A099C64F3C70600F8016C9F
:107DF00012F8018CB8F1000F3FF41DAFB8F1FF0F7E
:107E000044D0C8F1FF064478E40806FB04F408FBFC
:107E10000C4404EB042504EBC514C4F3C45B0588CF
:107E2000C5F3451506FB05F508FB0E5505EB0529C1
:107E300005EBC915C5F3C55590F8009009F01F0A68
:107E400006FB0AF6069C08FB046808EB082608EB0C
:107E5000C616F60D66F3040980F80090068865F3EF
:107E60004A160680360A6BF3C7064670E3E6BDF88D
:107E70001C4020F8064C31E7BDF81C4020F8044CAB
:107E800071E7BDF81C4020F8024CB1E7BDF81C407A
:107E90000480D0E60E9D8D424EDD541E059B03EB03
:107EA0004108069E08E0BDF81C30A8F800300131FA
:107EB00008F102088D423FDD14F8013F002BF6D097
:107EC000FF2BF0D0C3F1FF0998F80120D20809FB7D
:107ED00002F203FB0C2202EB022002EBC012C2F3FF
:107EE000C452B8F80000C0F3451009FB00F003FBD2
:107EF0000E0000EB002700EBC710C0F3C55098F848
:107F0000007007F01F0A09FB0AF903FB069303EB55
:107F1000032903EBC913DB0D63F3040788F8007032
:107F2000B8F8003060F34A13A8F800301B0A62F377
:107F3000C70388F80130BAE7059B0F9A13440593ED
:107F4000089B0B9A134408930A9B01330A930C9ADB
:107F50009A423FF40AAC002D40F37081089A12F067
:107F6000030F00F07981059F90460021069C20E6D2
:107F7000FF2A02D0DDF824E004E0DDF824E02A88BE
:107F80009A4232D0BEF1FF0F42D0CEF1FF046B789F
:107F9000DB080EFB0CF204FB032303EB032203EBD1
:107FA000C213C3F3C4532A88C2F345120BFB0EF16C
:107FB00004FB021202EB022102EBC112C2F3C55212
:107FC000297801F01F0109FB0EF604FB016101EBAA
:107FD000012601EBC611C90D61F3040A62F34A1AC6
:107FE00063F3CF2A1FFA8AF12B88298002460235D3
:107FF000A8450FD017F8010F0028F8D09042BED046
:10800000FF28B5D0079B03FB00FECEF3072EB9E790
:108010000899E9E705980C9C204405900A980130DE
:1080200004460A9006980B9D28440690BDF9460028
:1080300084423FF79AAB0D980028EBDD0598054682
:108040000E9C00EB0408069FD4E7BDF82450B9F15C
:10805000010F40D0B9F1020F32D1834B0593BDF827
:10806000242002F01F08C2F34516C2F3C423994628
:10807000BA8A01323B8AD31A1FB2CDF824C00CFB56
:1080800007F3069A02EB43020792012C26D0013037
:108090000A9A801A02B20C92089A0B99521A089204
:1080A000069A32F81320F4453FF75FAB7B000B9341
:1080B00010460021CDF818B0CDF828B0CB46B0E07E
:1080C0006A4B00936A4B4FF404726A4902206A4C6F
:1080D000A047FFF74ABB694B0593C0E74FF0000A82
:1080E0000BFB09F303EB032003EBC013C3F3C450F2
:1080F0000BFB06F303EB032203EBC213C3F3C552DE
:108100000BFB08F303EB032103EBC113C3F3C453CD
:10811000F4453FF72AAB79000891CDF818B0CB466B
:108120003AE0217863F304012170218862F34A1157
:108130002180090A60F3C701617009F10109023762
:10814000BDF9441089451ADC3C461FFA8AF1B7F89C
:1081500000E07145E5D0B7F800A068F3040566F3C8
:108160004A156BF3CF25069A51462846059B98473A
:1081700000F01F03C0F34512C0F3C420D1E70799F4
:10818000089C21440791099901310C460991BDF9D8
:1081900046108C423FF7E9AABDF94070B946BDF9D7
:1081A00044108F42EBDC079901EB4707CCE7F92B32
:1081B0009DBF0A9A5343C3F30722069A68F3040546
:1081C00066F34A156BF3CF2521882846059B98470F
:1081D00080B29AF800102288208009F10109013745
:1081E0000234BDF9443099450ADCBA463B78002B8D
:1081F000F3D08B42DBD1B4F800E09645D7D1EBE762
:10820000079B0B9C23440793089B0C9C23440893D7
:10821000099B01331C460993BDF946309C423FF748
:10822000A4AABDF94040A146BDF944309C42E7DC18
:10823000089B1F19079B03EB4404D6E7089B00210A
:108240000D9A8A42FFF678AE0433C81C059A02EBF9
:1082500040000E950D9FF4E4089B00210D9A8A4280
:10826000F2DA1A4619E600BF9F760000904C020031
:10827000444C0200604C02005D220100E9750000E0
:108280002DE9F04F91B09DF868409DF86CA09DF8E5
:108290007050BAF1040F00D914B911B0BDE8F08FD5
:1082A000049307920F4601463A460EA8BC4B9847E6
:1082B0000028F2D0BB4B98478046BB4B98470646F8
:1082C00083680593028ABDF838309B1A9BB20693E7
:1082D000BDF918C0ADF838C0438ABDF83AB0ABEB71
:1082E000030B1FFA8BFB0FFA8BFEADF83AE0BDF8DB
:1082F0003C10891A89B2ADF83C10BDF83E00C01A96
:1083000080B202B20892ADF83E20049AD2B198F839
:10831000083013F0010F15D101F10109069BA9EBFB
:1083200003090FFA89F9B9F1000F0BDD13469144E7
:108330001A78802A4FF0FF3298BF002203F8012BF1
:108340004B45F5D1D8F81430002B00F0A980954B9F
:1083500098470546B6F91000B38A01331B1A1BB2C1
:108360000693BDF93810B7F90020B7F8049009F169
:108370000109A9EB02090FFA89F9BDF93AE0B7F949
:108380000230B6F912609B1BAEEB0303121A8A1A75
:1083900009FB03234FEA410BCBEB430B079B5B44E9
:1083A0009B46012C46D0049B5B1A0793BDF93E30D7
:1083B0009E453FF772AFBDF93C304FEA4902089243
:1083C0000133591A0BB20993F146BDF938603446AE
:1083D000BDF93C309E4220DC079B03EB06080BEB0B
:1083E00046060FFA89F7049618F8013B03FB0AF3D7
:1083F000C3F307230293049A32F8023B0492ADF8C8
:108400000430009723B2069A059928466E69B04752
:108410000134BDF93C309C42E6DD079B099A1344C8
:108420000793089B9B4409F10109BDF93E3099452A
:10843000CBDD32E7BDF93E307345FFF62EAF4FEA94
:108440004909F046BDF938703C46BDF93C309F42C1
:108450001EDC0BEB47070FFA88F6049733465646A7
:10846000CA4699460296049A32F8023B0492ADF845
:108470000430CDF8009023B2069A059928466F691A
:10848000B8470134BDF93C309C42EBDDD146B246E1
:10849000CB4408F10108BDF93E309845D2DDFCE639
:1084A000002D40F09983B6F91030B6F8148008F129
:1084B0000108A8EB03080FFA88F80131069A891A17
:1084C0000AB2099215460130A0EB0B0B0FFA8BF2A2
:1084D0000892B7F90010B7F8049009F10109A9EB67
:1084E00001090FFA89F90EFB08C2059800EB420258
:1084F0000592B7F90220B6F91200121AAEEB020E7D
:10850000CB1AACEB030309FB0E33079A02EB4303D0
:108510000693244B98470646012C1BD0BAF1FA0F5C
:1085200000F2C580089B002B7FF7B7AE4FEA4803E7
:108530000A934FEA49030B93099B049A013A049268
:108540005B000D934FF0000BCDF81CA00C95DDF8EF
:10855000189036E3036A5BB30EA8144B9847F028D3
:1085600026D9BDF93A50BDF93E309D423FF795AE50
:108570004FEA48084FEA4909DDF814B0069FCDF8E4
:1085800000A0099B3A4659463046346AA047C34486
:108590004F440135BDF93E309D42F0DD7DE600BF20
:1085A00019150100695F0000DD0F0100FD140100D5
:1085B000BAF1FA0F10D8089B002B7FF76EAE4FEA86
:1085C000480304934FEA4909099B4FEA430B4FF0D4
:1085D0000008CAF1FF0E26E0089B002B7FF75DAE76
:1085E000099A56004FEA48084FEA49090024664DA7
:1085F0009B46059FDDF818A0324651463846A847ED
:108600004744CA440134A345F6D146E6059B049A83
:1086100013440593069B4B44069308F10108089BFD
:1086200043453FF43AAE002DF0DD069B1F46059C06
:1086300003EB0B0C7B78DB086278D2080EFB02F2AE
:108640000AFB032303EB032203EBC213C3F3C4535C
:108650003A88C2F345122188C1F345110EFB01F19E
:108660000AFB021202EB022102EBC112C2F3C55255
:1086700017F8021B01F01F01207800F01F060EFB07
:1086800006F60AFB016101EB012601EBC611C90DDB
:1086900061F304002070218862F34A112180090AE5
:1086A00063F3C70161700234BC45C3D1AEE7099BD7
:1086B000043B0A93089B002B7FF7EFAD4FEA48037A
:1086C0000C934FEA49030D930023079365E3B8F831
:1086D0000030AEF80030634601318D4200F0478330
:1086E00008F102080EF1020E1CF0030F00F02D83BA
:1086F0001CF8014B002CEED0FF2CE8D0C4F1FF0693
:1087000098F80130DB089EF80120D20806FB02F23F
:1087100004FB032303EB032203EBC213C3F3C45391
:10872000B8F80000C0F34510BEF80020C2F34512AF
:1087300006FB02F204FB002000EB002200EBC2105B
:10874000C0F3C55098F8002002F01F029EF8007098
:1087500007F01F0906FB09F604FB026202EB022484
:1087600002EBC412D20D3C4662F304048EF80040C2
:10877000BEF8002060F34A12AEF80020120A63F33C
:10878000C7028EF80120A6E75526010034F8065CE2
:1087900020F8065C34F8045C20F8045C34F8025CD1
:1087A00020F8025C25880580043104330834083041
:1087B0008E4540F347811A4653F8045C002DF3D0F0
:1087C000B5F1FF3FE2D013F804CCBCF1000F47D065
:1087D000BCF1FF0F00F02481CCF1FF0914F8055C17
:1087E000ED0810F8056CF60809FB06F60CFB0565AC
:1087F00005EB052605EBC615C5F3C45534F8066C24
:10880000C6F3451630F8067CC7F3451709FB07F792
:108810000CFB067606EB062706EBC716C6F3C55615
:1088200014F8067C07F01F0710F8068C08F01F0BE1
:1088300009FB0BF90CFB079707EB072C07EBCC1791
:10884000FF0D67F3040800F8068C30F8067C66F329
:108850004A1720F8067C3F0A65F3C70700F8057C35
:1088600012F803CCBCF1000F47D0BCF1FF0F00F0B1
:10887000DC80CCF1FF0914F8035CED0810F8036C00
:10888000F60809FB06F60CFB056505EB052605EB6E
:10889000C615C5F3C45534F8046CC6F3451630F854
:1088A000047CC7F3451709FB07F70CFB067606EBBC
:1088B000062706EBC716C6F3C55614F8047C07F066
:1088C0001F0710F8048C08F01F0B09FB0BF90CFBB9
:1088D000079707EB072C07EBCC17FF0D67F304088E
:1088E00000F8048C30F8047C66F34A1720F8047C06
:1088F0003F0A65F3C70700F8037C12F802CCBCF10D
:10890000000F47D0BCF1FF0F00F09480CCF1FF09BD
:1089100014F8015CED0810F8016CF60809FB06F686
:108920000CFB056505EB052605EBC615C5F3C4551F
:1089300034F8026CC6F3451630F8027CC7F34517CD
:1089400009FB07F70CFB067606EB062706EBC716B6
:10895000C6F3C55614F8027C07F01F0710F8028C06
:1089600008F01F0B09FB0BF90CFB079707EB072C13
:1089700007EBCC17FF0D67F3040800F8028C30F802
:10898000027C66F34A1720F8027C3F0A65F3C707AA
:1089900000F8017C12F8018CB8F1000F3FF404AF2D
:1089A000B8F1FF0F4BD0C8F1FF096578ED084678A4
:1089B000F60809FB06F608FB056505EB052605EB41
:1089C000C615C5F3C4552688C6F345160788C7F3F0
:1089D000451709FB07F708FB067606EB062706EBAB
:1089E000C716C6F3C556277807F01F0790F800C0D2
:1089F0000CF01F0A09FB0AF908FB079707EB072889
:108A000007EBC817FF0D67F3040C80F800C0078858
:108A100066F34A1707803F0A65F3C7074770C3E646
:108A200034F8065C20F8065C1AE734F8045C20F899
:108A3000045C62E734F8025C20F8025CAAE725884F
:108A40000580B1E60B9D8D4240F39481561E4FEA9E
:108A5000410C069B03EB0C08059B9C440BE0B8F80B
:108A60000030ACF80030013108F102080CF1020CC2
:108A70008D4240F37F8116F8014F002CF3D0FF2C7C
:108A8000EDD0C4F1FF0798F80130DB089CF8012015
:108A9000D20807FB02F204FB032303EB032203EBE0
:108AA000C213C3F3C453B8F80000C0F34510BCF8B8
:108AB0000020C2F3451207FB02F204FB002000EB8A
:108AC000002200EBC210C0F3C55098F8002002F05D
:108AD0001F029CF800E00EF01F0907FB09F704FBDA
:108AE000027202EB022402EBC412D20D744662F34E
:108AF00004048CF80040BCF8002060F34A12ACF883
:108B00000020120A63F3C7028CF80120ABE702379A
:108B10000236474545D01CF8011F0029F7D0F92936
:108B20009ABF01FB0AF1C1F30724079CC4F1FF05BA
:108B30007B78DB087278D20805FB02F204FB032382
:108B400003EB032203EBC213C3F3C4533A88C2F30B
:108B500045123188C1F3451105FB01F104FB0212F6
:108B600002EB022102EBC112C2F3C552397801F0C7
:108B70001F01307800F01F0E05FB0EF504FB0151BC
:108B800001EB012401EBC411C90D61F30400307045
:108B9000318862F34A113180090A63F3C7017170A9
:108BA000B5E7059B0A9A134405930B9B99440BF177
:108BB000010B049B099A13440493089B5B453FF403
:108BC0006CAB0C9B002BECDD4F46059E0D9B09EB1F
:108BD0000308DDF810C09EE7012D49D0022D3CD1DD
:108BE000DFF8E081B6F910300993B08A0130C01A7D
:108BF00000B2B7F90020BB8801339B1A1DB2F146C1
:108C00000EFB00FB059B03EB4B0BB7F90230B6F9EB
:108C100012609F1BAEEB070705FB07F7079B03EBF3
:108C20004707012C27D0049BA3EB0C031A46A7EBA4
:108C30004C030493089B9E453FF72FAB43000793DB
:108C40006B000893CDF814A04B1C06995B1A1BB25D
:108C50000993CDF818A0924666E0564B0093564B08
:108C600040F2533255490220554CA047FFF715BB3F
:108C7000DFF85481B6E7099B9B1A07EB4307089B73
:108C80009E453FF70AAB430004936B0005933B46B8
:108C900047469846BDF938301C46BDF93C20934202
:108CA00010DC5B000BEB030508EB0306524629883A
:108CB00036F8020BB84725F8020B0134BDF93C30F9
:108CC0009C42F3DD049B9B44059B984409F10109F8
:108CD000BDF93E309945DDDDFFF7DFBA01350236DB
:108CE0000234BDF93C309D420FDC17F8013B002BEC
:108CF000F4D0F92B9DBF069A5343C3F30722059A7C
:108D000031882088C0473080E8E7079B9B44099B57
:108D10009A44049B089A1344049309F10109BDF98C
:108D20003E3099453FF7B9AABDF938301D46BDF927
:108D30003C209342E9DC0AEB03075B000BEB0306E4
:108D4000049AD418D1E7049B00210A9A8A420ADDCA
:108D50000433C81C4000069A1418059A10440B9559
:108D6000DDF828E027E51A4670E6049B00210A9A00
:108D70009142EDDB059B0C9A13440593049B099AE1
:108D800013440493069B0D9A13440693079B0133E7
:108D90000793089A9A423FF480AA002DE5DD049AD1
:108DA00012F0030FCFD0DDF81880DDF814E0944600
:108DB00000219DE4904C0200544C0200604C0200E3
:108DC0005D2201009F760000E97500002DE9F04F5B
:108DD000BDB01B902391174608939DF818310A9354
:108DE0009DF81C3106934B1EC81D3AAA13F8011FAB
:108DF00002F8011B8342F9D1A34B9847A34B984734
:108E00001890018ABDF8E8305B1AADF8E830428A64
:108E1000BDF8EA309B1AADF8EA30BDF8EC305B1AC9
:108E2000ADF8EC30BDF8EE309B1AADF8EE30984B53
:108E30009847199030B9089A53881BB91389B3F52C
:108E4000807F71D0069B002B14BF4FF0030B4FF0B7
:108E5000020B1B990B46B1F900208D880135AD1A24
:108E60002DB2BDF9EA00189EB6F91210D846BDF928
:108E7000E840B6F91060B3F902305B1AC31A921BCE
:108E8000A21A05FB032303FB0B731493A4B2A219CC
:108E900092B2ADF89820BDF8EC3001331B1B9BB2A9
:108EA0001CB21694013B1344ADF89C3080B24318B9
:108EB0001BB2ADF89A30ADF89E30BDF8EE600136C9
:108EC000361A36B208994B88002B40F053830B8931
:108ED000B3F5807218BF01220592199A002A40F05A
:108EE0007083B3F5807F40F049830A9B23B98B7A66
:108EF00013B9069B002B31D13AA8664B9847B0F5C1
:108F0000F07F40F2AC804FF47070634CA0471A9031
:108F10004FF4F070A0471790482128A85F4B98475E
:108F20004FF4F0731C93E4E00A9B002B8AD1069B5C
:108F30008BB9937A13B14FF0020B8AE7937B0293BC
:108F4000137801930123009300233A461B99239839
:108F5000534CA0470BE34FF0030B7AE73AA84D4B75
:108F60009847B0F5F07F14D83AA84A4B9847814605
:108F70004FEA4900484CA04782464846A04704466D
:108F80000596002E4FDD08FB05F80025AC46149E23
:108F900025E04FF4F079EBE75B44023796450AD0C1
:108FA000997802F8011B0029F6D05878197801EB5E
:108FB00000213980F0E74644BDF8EC300133BDF8BC
:108FC000E8209B1A0CFA83F3994514D9BDF89E301A
:108FD0000133ADF89E300135059B9D4223D0169B91
:108FE000002BE8DD04EB0C020AEB4C079C4404EB7D
:108FF0000C0E3346D4E7089A937B029313780193BF
:10900000022300932346524626A92398244FB847AB
:10901000BDF89E3001331BB2ADF89A30ADF89E30EA
:109020004FF0000CD7E7BDF99E30BDF99A209A4267
:109030000FD0013BADF89E30089A937B02931378D2
:109040000193022300932346524626A92398144DE8
:10905000A8472046134CA0475046A04787E23AA8AD
:109060000C4B98471C901C9B58000B4CA0471A9027
:109070001C98A0471790482128A8084B9847059BA3
:10908000002B36D091E200BF695F0000DD0F0100C8
:10909000C5BE0000FD1401003D290100372B010071
:1090A0008182000071250100052208984388ADF8EF
:1090B000AC300389ADF8AE302897ADF8A4501B99B9
:1090C000CB88013349885B1AADF8A6308DF8B22001
:1090D0008388ADF8A830C388ADF8AA308389ADF88D
:1090E000B030C37BC3F300038DF8B33028A8934B93
:1090F00098470898837ADA43D2B2129203B39BB2AC
:10910000427BD20802FB03F210928289C2F345121D
:1091100002FB03F21192027B02F01F0202FB03F337
:109120001393069B8BB90A9B53BB089A538853BB76
:109130001389B3F5807F14BF022301231D9306E03A
:109140000023139311931093EBE702231D93199BB4
:10915000E3B9189BB3F91230BDF9EA2013441B9A06
:10916000B2F902209B1A22931F96002E40F3E4814D
:1091700008FB05F31E9300230E930F93D14654E191
:1091800002231D93E3E702231D93E0E71C99179840
:109190006B4B9847DDE70C9B2B441BB2BDF9A82015
:1091A0009B1ABDF9AA200D998A1ABDF8AE10B1F527
:1091B000807F56D0BDF9AC10002965D1BDF8D6101E
:1091C000319C01FB03430993329B01FB02330B9358
:1091D000099B1F12BDF9A4309F4280F2AB80002F83
:1091E000C0F2A8800B9A121210461592BDF9A62063
:1091F000904280F29F800028C0F29C809DF8D4208D
:1092000012F0040F6AD0289912F0020F55D103FB17
:1092100000735A00881811F813308DF8B430437871
:109220008DF8B53002219DF8D43013F0010F0DD028
:10923000209B6FF3040343F4FC636FF3CF23ADF87B
:109240008030BDF8B4009BB2984273D09DF8B33023
:10925000002B59D19DF8B6308AF80030BDF8B430F3
:1092600086E03498339900FB03F401FB1247319CEC
:1092700004EBE714099400FB02F201FB0323329A8A
:1092800002EBE3130B93A3E7BDF8D61001FB03F346
:1092900001FB02F23499339801FB03F400FB1247FF
:1092A000319C04EBE734099401FB02F200FB032339
:1092B000329A02EBE3330B938AE7159A03FB0273AE
:1092C00003EB43028B18895C8DF8B41059788DF844
:1092D000B5109B788DF8B6300321A4E739B2BDF9FB
:1092E0005420BDF8B030259224912EA8154CA047EB
:1092F000ADF8B400259A24992EA8134B98478DF801
:10930000B600002211468EE7BDF82430ADF8D83003
:10931000BDF82C30ADF8DA30ADF8DC70BDF8543063
:10932000ADF8DE3038928DF8E41028A8074B984746
:1093300000288FD100238AF800303DE04DEB00007B
:10934000ED2B010019E9000049EA0000FDED0000E5
:10935000E0070000FF238AF800307278337803EBCF
:1093600002239BB20A9A1AB13FF81C209A4236D0C7
:10937000089A927AEAB1BDF84820D90A109801FB00
:109380000201C1F30421C3F34510119C00FB02400C
:10939000C0F3052003F01F03139C03FB0243C3F338
:1093A000072363F3040960F34A1961F3CF291FFA15
:1093B00089F3079A22F8153001355E440AF1010A53
:1093C000454510D0059B002B7FF4E5AE069B002B96
:1093D000C0D0B3788AF80030002BEDD0BDE7002371
:1093E0008AF80030E8E7169B0F9A9C18199B002B0F
:1093F0003ED1149B1E9A13441493BDF8EC300133F4
:10940000BDF8E8209B1A04FA83F31C9A9A425CD9AF
:10941000BDF89E300133ADF89E300F940E9B0133A2
:109420000E931F9A934200F08780189BB3F9103077
:10943000BDF9E82013441B9AB2F900209B1A0C9343
:10944000169B9846002B11DD179B19460F9A01EBCE
:10945000020A1A9B194601EB42030793149E00254A
:10946000229B0E9A13441BB20D93ABE70F9CBDE7F2
:109470000F9B179A13441E46BDF8E810BDF8EC3058
:1094800001335B1ABDF8EA20189D688A02440E98E1
:109490000244288A01441BB212B209B230464E4D32
:1094A000A84728B102281D9A08BF02461D92A0E7CE
:1094B000BDF8EC100131BDF8E830C91A09B23046E8
:1094C000464B984702231D9393E7089DAB7B02937D
:1094D0002B7801931D9B0093179B1A9A26A923981A
:1094E0003F4CA047BDF89E3001331BB2ADF89A3017
:1094F000ADF89E30069B5BB90A9B83B96B888BB92C
:109500002B89B3F5807F14BF022301231D9301E053
:1095100002231D93199B43B900230F937EE7022377
:109520001D93F7E702231D93F4E71C9917982D4B21
:10953000984700230F9371E7BDF99E30BDF99A203B
:109540009A420FD0013BADF89E30089A937B02936C
:10955000137801931D9B0093179B1A9A26A92398B1
:109560001F4CA0471798204CA0471A98A0473DB021
:10957000BDE8F08F199B13BB012305933AA81B4B41
:109580009847B0F5F07F7FF66AAD4FF47070184CD5
:10959000A0471A904FF4F070A0471790482128A8D0
:1095A0000E4B98474FF4F0731C93069B002B7FF4EF
:1095B0007BAD0A9B002B0CBF0422062275E501231C
:1095C00005933AA8094B9847B0F5F07F7FF647AD71
:1095D0004FF4F0731C9346E51DBE0000372B0100CD
:1095E00081820000ED2B010071250100FD140100B6
:1095F0003D29010070B59EB004460D46164609A8E7
:109600000B4B98470B4B1B88ADF8263009AA29460F
:109610002046094B984702A8084B9847002300931F
:10962000334602AA29462046054CA0471EB070BD0D
:1096300069C20000B84C020031C30000CD9900009F
:10964000259A000010B5044610210C4B9847237B47
:109650006FF304032373A3896FF34A13A3811B0AD7
:109660006FF3C7036373FF2323704FF48073238169
:10967000E37B43F00103E37310BD00BF372B010010
:1096800004380A2813D8DFE800F00608060A0C0E92
:10969000100A0C0E1000102070471820704701208F
:1096A0007047022070470420704708207047002050
:1096B0007047032805D002D30638042801D90020BA
:1096C00070470120704702380C2808D8DFE800F006
:1096D00009070709070909090909090909000020FB
:1096E00070470120704700002DE9F04F8FB005460C
:1096F0000E463AB11C4610461B78052B10D80FB009
:10970000BDE8F08F844B0093844B4D2284490220A6
:10971000844CA047844A31462846844B9847EEE75C
:10972000A189834B98470746002800F0B58090F840
:109730000C9009F01F0948467E4B984780464846E2
:109740007D4B98478146BB696BB17C4B00937C4B4A
:10975000F72273490220734CA047BA693146284664
:10976000724B9847CBE73B69002B49D06B1EE81D35
:109770000AAA13F8011F02F8011B9842F9D1638865
:109780001BB92289B2F5807F28D0EA880132698826
:10979000521AA98801312888091A201D01902089B0
:1097A00000901BB212B209B20AA8DFF8B8A1D047E4
:1097B0002A88BDF828301344ADF828306B88BDF8EE
:1097C0002A101944ADF82A10BDF82C100A44ADF83F
:1097D0002C20BDF82E201344ADF82E300AAA3146B5
:1097E0000CA8584B9847002889D03A69CDF80490C6
:1097F000CDF8008023460CA92846534CA0477EE7AD
:109800002A46314608A84F4B984700283FF477AFC7
:10981000BDF824300133BDF820209B1A1BB20393FE
:1098200003EB4300494B984702900DF11F020AAB2E
:109830000CA812F8011F03F8011B8342F9D1012182
:109840000AA8434B9847BDF92030B5F90020BDF96F
:1098500022A0B5F90210AAEB01010846BDF92610B5
:109860008A4555DCDFF8DCB09B1A1BB205930795DF
:1098700006944446804623E0079D0498354B98475C
:10988000354B00932E4B4FF49A7225490220254CFC
:10989000A0470298314B9847284B00931F4B582202
:1098A0001F4902201F4CA0471F4A314628461F4B24
:1098B000984724E70AF1010ABDF926309A4527DCCA
:1098C0000AAA31460CA8D8470028F3D00497029B77
:1098D0000093039B0FFA88F205993846204DA8475C
:1098E0000128C9D1CDF804900094069B029A0CA9D6
:1098F0000AA8154DA847BDF82A300133ADF82A3023
:10990000BDF82E300133ADF82E3008F10108D1E753
:109910000298124B9847F2E60C4D0200BC4C020034
:10992000DC4C02005D220100244D0200F595000090
:1099300001F20000B3960000C79600002C4D020013
:10994000C84C020019150100CD8D00003D29010011
:10995000F314010035FF0000404D020071250100A5
:1099600011FF000065EC000058B10278A2F120035D
:10997000DBB25F2B07D952B2002AB4BF022000200D
:1099800070470320704701207047A0F13003DBB21D
:10999000092B17D9602884BF2038C0B24138052868
:1099A0000ED8DFE800F011030507090B0B20704704
:1099B0000C2070470D2070470E2070470F20704715
:1099C00000207047184670470A20704710B50446BB
:1099D0001C21124B9847FF23237223786FF3040353
:1099E000237023886FF34A1323801B0A6FF3C70386
:1099F00063700B4B63604FF6FF73E3812382A378A0
:109A000043F01F03A37063886FF34A1363801B0A3C
:109A10006FF3C703E3700023A37510BD372B01005C
:109A2000100000202DE9F04FD9B0629C157A052D69
:109A300001D91D7815B959B0BDE8F08F0A93934646
:109A40000A460D9105461390DBF804300593014654
:109A500056A8AA4B98470028EDD09BF8172012F083
:109A6000020F21D1AB8801332A889B1A1BB2059AB9
:109A7000B2F908A0BBF90A90D1441399B1F90020BA
:109A80001F92B1F90200BBF912201A92BBF914100F
:109A9000421892B215B2002C4AD000294BD10028AE
:109AA00014DB0E95002629E0BBF90C30029247F634
:109AB00018420192BBF90A200092DBF804200A99AF
:109AC0003AA88F4DA847BDF9E830D0E7A168081A39
:109AD00080EAE071A1EBE071C9F50070B1EB400FD5
:109AE00005DD4FF0FF3222600E95002606E0266865
:109AF000002E23DB61680A4412B20E921BB2194693
:109B00001093BBF90C209BF8173000930B46059976
:109B10000A9830447B4DA84783192F46DFF8F88117
:109B20003146CDF81890D1460E9D26461C460FE0D2
:109B30000E950026E2E70E950026DFE70E9500263B
:109B4000DCE721469AF80030002B3FF474AF04465E
:109B500005EB09030D9AB2F90220934220DA0A9B21
:109B600003EB040ABBF90C209BF817300093109B01
:109B700005995046B8472044069B1D442DB2002E3F
:109B8000DFD04545DDDB3368002BDADA3460139A29
:109B9000B2F90230EB1A7360B2F90230B360D0E769
:109BA0000E460794DDF818900E959BF8172012F0DA
:109BB000040F2FD112F0080F45D19BF808300B93FA
:109BC000BBF80E70BBF81030194608939F4202D9BB
:109BD0003B460F4608939BF8183013F0030F49D10A
:109BE0003DA8494B9847BBF80230ADF8F6300B9BC7
:109BF000FA2B88BFFF2316931FFA89F31793BDF83A
:109C0000383011931F9D00231993BA46D846B346A6
:109C100000F0D3BDBBF90C30A11B0092059A89B2AC
:109C20000A983044394CA047139A9388013312881C
:109C30009B1A1BB2181A00EBD0701F9B03EB60033A
:109C40001BB21F93B9E7BBF90C300799891B00922F
:109C5000059A89B20A9830442C4CA047139A9388ED
:109C6000013312889B1A1BB21B1A1F9A13441BB292
:109C70001F93A2E753A8264B9847BBF80030ADF8D6
:109C80004C31DBF80430B3F908300533214A82FB4C
:109C90000312DB17C3EBA203ADF84E319BF808307B
:109CA0008DF854319DF855319BF8192062F301036A
:109CB0008DF8553194E70025AAE00025A8E0069B21
:109CC0002BB9BDF848311993012306938AE0069B0E
:109CD000012B00F0F185022B00F03385B8F800600D
:109CE000B5E0202C7ED1529B199A9B1A072B15D0D8
:109CF000B8F800300C930223069373E019150100A5
:109D00007D400100B13D010069C20000DD3F01005E
:109D1000E1A800006766666600FCFFFF099B9818D3
:109D2000431E05303AAA13F8011F02F8011B8342B3
:109D3000F9D19DF8E8008C4CA04705469DF8E90054
:109D4000A04700EB05159DF8EA00A04706469DF8E0
:109D5000EB00A04700EB06169DF8EC00A047074675
:109D60009DF8ED00A04700EB0713C3F3C4032E9A40
:109D700063F304021346C6F3850666F34A13C5F37C
:109D8000C40565F3CF23ADF8B8309BB20C93022322
:109D9000069327E0ADF8E8A00E9AADF8EA20B8F8EF
:109DA0000C30013B53440344ADF8EC30179B013BAE
:109DB0001344ADF8EE303DAA0D993AA86B4B984785
:109DC00056E06B4B00936B4B40F297126A490220AE
:109DD0006A4CA047002F05DDB8F80C3053443B44D3
:109DE0000FFA83FA5299079BA3EB0B038B4240F2C5
:109DF000AC844FF6FF7399453FF45DAF089A9A42E1
:109E00003FF45BAF59440A985D4B1B68984785B295
:109E10005C4E336852A9099F384698470446336818
:109E2000002152983844984798F8173013F0010FE2
:109E300006D0232C3FF443AF069B012B3FF451AFD8
:109E4000B8F800600C9B069A022A08BF1E4602461C
:109E5000214605984C4B984707464FF6FF739945A6
:109E600006D00899994203D0A94501D8A94291D8B2
:109E70000B9B042BAED9059B002BA2D098F8193070
:109E80000F93002322463AA90598404DA84758B998
:109E90001F2C9FD93E4B0093364B40F2A1123649FE
:109EA0000220364CA04795E7BDF8EC201AB9BDF862
:109EB000EA30002B8ED0BDF9EE505544BDF8EA30A3
:109EC0002B440D98B0F900108B4283DBB0F90430BD
:109ED0009D423FF77FAF059BB3F90810B3F90A30F5
:109EE000CB1A0E990B44991ABDF9F030CB1A159381
:109EF0001A44B0F902309A42FFF66CAFB0F906305E
:109F0000159999423FF766AF21460598214B98472E
:109F10008646F0B1059B1B7B13F0030F00F05E82B9
:109F20002BB21893BDF954301D939DF8F230129363
:109F3000032B00F0FF80013B072B00F20281DFE8DA
:109F400013F00A012D000001FB00000100010001D7
:109F50001101114B0093074B40F2B7120649022042
:109F6000064CA04736E700BF8B99000031C30000C4
:109F7000E84E0200784E0200B84E02005D22010059
:109F80006400002058000020610001005900010019
:109F9000084F020051000100304F0200C0231B9304
:109FA000AC4B2093BDF8EA301E93BDF8EC10129A2A
:109FB00002FB03F20D9BB3F90030189C9C42BABF20
:109FC0001B1B03EB4303002327930D9BB3F90430C2
:109FD0001E980446A04880FB0440189C20449842E8
:109FE000C3BF1B1B013303EB43031E9B14930D9B49
:109FF000B3F902301D9C9C42B4BF1B1B0023259368
:10A000000D9BB3F906301D9C0819984240F3B180AE
:10A010001B1B0133289306F01F032293C6F345133D
:10A020002493C6F3C4232393129B1846279B00FB5B
:10A0300003F3259800FB02320EEBE206319602F0A4
:10A0400007061E9801FB00F1B1F5F07FA8BF4FF4A1
:10A05000F07129910846814CA04721902999480028
:10A06000A04730907E4B98477E4B9847B0F9104000
:10A07000838A01331B1B19B226918168279B764A7C
:10A0800082FB03E2A2EBE372B0F912301D98C31A0F
:10A090002698864618980EFB03031B1B259C0EFB77
:10A0A0000420034401EB43011891ADB22A44ADF8FA
:10A0B000E020149A9646684981FB0EE3A3EBE27315
:10A0C000013D2B44ADF8E430159D25442BB2ADF88D
:10A0D000E230ADF8E630644B98472A90289DAC42B8
:10A0E00080F261811499279A8C1A2B941E9D6B1A09
:10A0F0001344129901FB03F32C93574A82FB042368
:10A10000C3EBE473269803445B002D93002326934E
:10A110001593CDF8C8B0CDF8CC903497DDF86090A9
:10A12000DDF8C4B0CDF8C4A0DDF8C0A0CDF8D4806F
:10A130008846EAE004231293F0231B934B4B2093B1
:10A1400030E74B4B00934B4B40F27A224A490220B6
:10A150004A4CA0473EE60123129380231B93484BB1
:10A1600020931FE708231293FF231B93454B209353
:10A1700018E728914FE7B8F1080F04D0DBB2209A16
:10A18000D25C00E0159A58AB0B4403F8842C0131E3
:10A19000032928D0B44540F39480129B43441E46C3
:10A1A0002EFA08FE0135149BAB4200F09080129607
:10A1B0009BF8003003EA0E02ACEB060322FA03F32D
:10A1C00013F0FF02DED01698FF28D4D0B8F1080FA4
:10A1D0000FBFDAB2DBB2209AD25C169B03FB02F20D
:10A1E000C2F30722CFE79DF8DC109AF80130DB08B4
:10A1F000C1F1FF00239A01FB02F200FB0323C3F32A
:10A2000004231D939DF8DE3018939AF8002002F085
:10A210001F02C3F1FF00229B189C04FB03F300FB09
:10A220000232C2F304231E939DF8DD00BAF8003019
:10A23000C3F34514C0F1FF03249A00FB02F203FBB1
:10A240000423C3F30523F9B9F0B9189AE2B9219AA6
:10A25000D1551DE0644D0200565555553D2901006C
:10A26000695F0000DD0F0100C5BE0000684D0200FF
:10A27000604F0200884E0200B84E02005D220100CD
:10A28000604D0200784D0200219A4FF0FF31D15508
:10A2900009EB470019F817101E9A62F3040109F838
:10A2A000171039F8172063F34A1229F81720120AF9
:10A2B0001D9B63F3C702427001370AF1020A0021B5
:10A2C00068E70BF1010BDDF86CE0159E6AE7534679
:10A2D000CA4699462A9B4BBB2B9B3B44299A9A42E0
:10A2E00041DDBDF8E6300133ADF8E63026972C9B12
:10A2F0001E440BEBE60B06F007062D9B9944259BAD
:10A3000001332593289A934244DA1B9B23FA06FED5
:10A31000279D149A954207DA269F0021C8F1080C60
:10A320004B46D1469A4642E7269FD3E7269B219A81
:10A3300013441C46BDF9E010BDF8E43001335B1A4C
:10A340001BB2BDF9E6202046AB4DA8470028C3D17B
:10A35000BDF8E4100131BDF8E030C91A09B2204659
:10A36000A64B9847B8E70F9B0293169B01930223D5
:10A370000093219B524638A90D98A14CA047BDF8E7
:10A38000E63001331BB2ADF8E230ADF8E630002321
:10A390002693ACE7DDF8C8B0DDF8CC90349FDDF84B
:10A3A000C4A0DDF8D480BDF9E630BDF9E2209A42C0
:10A3B0000ED0013BADF8E6300F9B0293169B019344
:10A3C00002230093219B309A38A90D988C4CA0470A
:10A3D00021988C4CA0473098A047FBE42CB2BDF9E3
:10A3E0005400ADF88C609DF8F2302093032B00F000
:10A3F000C180013B072B00F2C580DFE813F0CD00E0
:10A400000800C300BD00C300C300C300D50004237F
:10A41000C02212927C4A22921699F9292BD87B4AA3
:10A4200092F800218A4200F0C880D3B1229E721EA9
:10A4300076490139013B06EB030C169B1E46CDF80D
:10A4400050B09B4612F8013FFF2B1ABF0BFB03F3E2
:10A45000C3F30723334601F8013F9445F2D1DDF8F9
:10A4600050B06A4B9DF8582083F80021209AC3F819
:10A4700004211C9B2293BDF8EA302493BDF8EC2004
:10A48000209901FB03FC0D9BB3F900309C42B4BF43
:10A490001B1B002314930D9BB3F904302499214412
:10A4A0009942C6BF1B1B0133249B25930D9BB3F917
:10A4B00002309842B4BF1B1A002326930D9BB3F9B8
:10A4C000063011189942C3BF1B1A01331B931B920C
:10A4D000149B2193209903FB01F4269800FB0C4464
:10A4E0000EEBD40604F00704249902FB01FE724629
:10A4F000BEF5F07FA8BF4FF4F0721D921046444B9A
:10A5000098471890ADB2149BEB18ADF8E030013DC0
:10A51000259AAB18ADF8E430159D269805442BB26A
:10A52000ADF8E230ADF8E6303A4B98471E902099EE
:10A53000C1F10805249A149BD318259A9B1A01FB94
:10A5400003F3209326981B9B984280F2DF804FF004
:10A55000000ECDF890B0CDF8989027970F4615953E
:10A56000CDF8A0A0DDF894A08146CDF89480DDF868
:10A5700088807AE0042320931023F0221292264A46
:10A58000229249E7254B0093254B40F2E5122549DD
:10A590000220254CA0471DE40123209302238022A2
:10A5A0001292224A229237E7082320934FF48073B5
:10A5B000FF2212921E4A22922EE7144AD2F8042158
:10A5C000209991427FF431AF4BE701361298002475
:10A5D00001318C452ED0337803402A1BD34013F031
:10A5E000FF0F1ABFDBB218F8033000230B70A5422F
:10A5F000EBD93C44F840EBE71DBE0000372B0100CF
:10A600008182000071250100644D0200502A002063
:10A610003D290100C5BE0000684D0200884F0200C0
:10A620009C4E0200B84E02005D220100604D020007
:10A63000784D020015951E9B53BB149BAAEB030398
:10A640005B441D9A9A423FD9BDF8E6300133ADF81C
:10A65000E630DE46209B1C4406EBD40604F00704DB
:10A6600009F101091B9B994547DA129B23FA04F073
:10A67000149B53450ADA189A02EB0E01219BAAEBB0
:10A68000030BF34402EB0B0C159DA4E7F346D2E752
:10A69000189B734418462293BDF9E010BDF8E430CE
:10A6A00001335B1A1BB2BDF9E620854DA84700288F
:10A6B000C3D1BDF8E4100131BDF8E030C91A09B2C8
:10A6C0002298804B9847B8E70F9B0293FF23019392
:10A6D00002230093189BBDF88C2038A90D98DFF851
:10A6E000E8B1D847BDF8E63001331BB2ADF8E2302F
:10A6F000ADF8E6304FF0000EACE7DDF890B0DDF8D5
:10A700009890279FDDF8A0A0DDF89480BDF9E63091
:10A71000BDF9E2209A420FD0013BADF8E6300F9B25
:10A720000293FF23019302230093189BBDF88C2012
:10A7300038A90D98644CA0471898644B9847FFF7C8
:10A7400049BB00230693FFF74DBB5346CA469946C3
:10A7500098F8183013F0020F46D198F8183013F01B
:10A76000010F62D10A9A079D5619B8F90C2098F882
:10A7700017300093109B05993046554CA04744195B
:10A78000139BB3F9005098F8172012F0040F6CD106
:10A7900012F0080F7ED10E9B17990B441BB2119A31
:10A7A0000A4492B21192DDF81CB00E930D9AB2F9E0
:10A7B00006209A42FFF63FA907940A9A13465B4483
:10A7C000099312F80B30002B3FF435A91A9B1D4456
:10A7D0000FFA85F90023529306933E4B1C934B4688
:10A7E000D1469A46FFF7FEBABDF87C30ADF8E030AE
:10A7F000D8F80430B3F9083003EBD372BDF94E3109
:10A8000003EBD3735B1003EB6203119A13441BB287
:10A81000ADF8E230ADF8E890ADF8EA3053AB0D9A00
:10A820003AA938A82C4CA04797E7BDF87C30ADF882
:10A83000E030D8F80420BDF94E3103EBD3735B1040
:10A84000013311890B4452899B1A119A13441BB28C
:10A85000ADF8E230ADF8E890ADF8EA3053AB0D9AC0
:10A860003AA938A81C4CA0477CE7B8F90C300092F4
:10A87000059A01463046194EB047139A9388013322
:10A8800012889B1A1BB2181A00EBD07005EB6005FA
:10A890002DB280E7B8F90C300092059A0146304697
:10A8A0000E4EB047139A9388013312889B1A1BB23D
:10A8B000181A05442DB26EE700230693FFF70EBA6F
:10A8C0001DBE0000372B01005177000071250100EB
:10A8D000B13D0100502A002011A90000DD3F010018
:10A8E00010B504460A21094B984701236380FF23D2
:10A8F000237223786FF30403237023886FF34A13C2
:10A9000023801B0A6FF3C703637010BD372B010050
:10A910002DE9F04FCBB0B3F90250002D00F01884B0
:10A920001C7A052C40F21484B0F90060B1F9007073
:10A93000BE4200F030811C46964608920791069070
:10A9400005EBD575C5F34F05BE42D4BFC5EB060375
:10A95000C5EB0703ADF82031BE42ACBFAB19EB1914
:10A96000ADF824310F46B1F902200646B0F90230A5
:10A970009A42D4BFC5EB0201C5EB0301ADF8221129
:10A980009A42ACBFAD18ED18ADF82651724648A9F1
:10A990000846AB4B9847002800F0DA83B6F902600E
:10A9A000B7F90250AE4200F0FE80069BB3F90030CA
:10A9B0001A460593079BB3F900A0524500F00182A7
:10A9C000AE4206DB33462E461D46059BCDF814A04D
:10A9D0009A46059BAAEB03030993AA1B0A92002B34
:10A9E000B8BF5B429B46002AB8BF52429046B4F9BA
:10A9F00002909342C7BF530193FBFBF34FEA4B1303
:10AA000093FBF2F38F4AD35C09FB03F909F13F0989
:10AA10004FEAE9131F469BB205988245D4BFC3EBAA
:10AA20000A02C3EB0002ADF838208245ACBF03EB4D
:10AA30000A021A18ADF83C20B542D4BFC3EB050298
:10AA4000C3EB0602ADF83A20B542ACBF5B199B19C7
:10AA5000ADF83E3048AA0EA90846794B9847002821
:10AA600000F072834FEA292907F001034B440B934E
:10AA7000C34540F3B682099A002A40F38E821FFA3A
:10AA800086FB1FFA89F31FFA85F9ABEB030200215D
:10AA90000191A9EB03031BB20093534612B205992F
:10AAA00012A8694FB847BDF82C800BEB08020123B0
:10AAB0000193C1440FFA89F30093534612B20599EA
:10AAC0001DA8B847002112A8DFF89C81C0470B9051
:10AAD00000211DA8C0470C90637A13F0100F00F0FE
:10AAE000A4824FF0FF330D930A93584B9847584B6D
:10AAF00098478246068ABDF83850AD1BAAB2ADF819
:10AB00003820408ABDF83A10091AADF83A10BDF85D
:10AB10003C309B1B9BB2ADF83C30BDF83E10091A8F
:10AB2000ADF83E105D1CAD1A2DB20EA8494B9847EA
:10AB3000B0F5F07FC0F0A2824FF4F07B5846464B50
:10AB400098478146BAF81030BDF838201A4412B23E
:10AB50000592ADF84020BDF83C201344ADF84430D8
:10AB6000BDF83A30BAF8122013441BB2ADF84230A7
:10AB7000ADF846305946394B9847BAF91220BDF91D
:10AB80003A601644BDF93E3013449E4200F3B98248
:10AB900000270994A0E2B0F902E0B1F90240A6450D
:10ABA0007FF4C9AED4E294F80890284B9847284B1C
:10ABB00098470746B4F90230013B5E1003F00103E9
:10ABC0009D19B4F90630002B35D0B4F9048018F182
:10ABD000000818BF4FF00108214B984770BB88F060
:10ABE0000102079BB3F900300699B1F9001018462D
:10ABF0008B42A8BF0846ADF8A0008B42B8BF0B46F9
:10AC0000013BADF8A43006994B885D1BADF8A2500E
:10AC10003344ADF8A6304AB3637A03F003030293DA
:10AC2000CDF80490012300930023228828A948A886
:10AC30000C4DA84788E24FF00008CDE70022D0E78E
:10AC400019150100A44F0200E9BE0000695F000071
:10AC5000DD0F0100FD1401003D290100ED2B010075
:10AC6000C5BE000051770000C1BD000028AA48A958
:10AC70001046A14B9847002800F06682BDF9A0E07D
:10AC8000B7F910108BB2AEEB030292B20FFA82FC4E
:10AC9000ADF8A0C0BDF9A200B7F81290A0EB09056D
:10ACA000ADF8A250BDF9A460F31A9BB2ADF8A43080
:10ACB000BDF8A650A5EB0905ADF8A65001339A1AC8
:10ACC00015B2ADF8CCE0ADF8D060ADF8CE00ADF87F
:10ACD000D200B8F1000F1CD06144B4F90620B4F9D9
:10ACE00004301A4491FBF2F302FB13110BB20A93E6
:10ACF00009952846814B98478246BDF9A260BDF967
:10AD0000A630B34259DBDFF81092DFF808B20595A0
:10AD100035E00021EAE7B4F906E073449A42BABF8D
:10AD20000AF8001013460B46013000B201331AB284
:10AD3000854207DDB4F904309342ECDB1844801AF5
:10AD400000B2F1E705950220637A03F00303029352
:10AD5000237A019300905346228833A948A8D84704
:10AD6000BDF8CE300133ADF8CE30BDF8D23001336E
:10AD7000ADF8D2300136BDF9A6309E421DDC0999EE
:10AD80005046C8477A8A3244398ABDF8A0301944FF
:10AD9000059B12B209B25046594DA847B8F1000FB1
:10ADA000D2D00028D0D0059B002B04DD0A9A0020C9
:10ADB00001461D46BEE70220C6E75046514B984764
:10ADC000C2E194F80890504B9847504B9847804602
:10ADD000B4F90250013D6F1005F001053D44B4F98E
:10ADE00006302BB1B4F90460003618BF012600E02C
:10ADF0000026474B984710B986F0010200E0002278
:10AE000006990B885D1BADF8A0501F44ADF8A470E7
:10AE1000079BB3F90230B1F9021018468B42A8BF64
:10AE20000846ADF8A2008B42B8BF0B46013BADF817
:10AE3000A63072B1637A03F003030293CDF8049055
:10AE4000012300930023228828A948A8314DA84750
:10AE50007AE128AA48A91046274B9847002800F015
:10AE60007381BDF9A000B8F81030C51AADB2ADF8C5
:10AE7000A050BDF9A220B8F81270D11BADF8A210F5
:10AE8000BDF9A410CB1A9BB2ADF8A430BDF8A6E072
:10AE9000AEEB0707ADF8A67001335B1B1BB209933D
:10AEA000ADF8CC00ADF8D010ADF8CE20ADF8D22082
:10AEB0000A931846114B9847059076B1B8F91020BF
:10AEC000BDF9A0703A44B4F90630B4F904703B44BB
:10AED00092FBF3F703FB172700E000273FB2BDF911
:10AEE000A250BDF9A6309D4253DCDFF82C90DFF86C
:10AEF00010A0DFF820B02CE0191501003D29010059
:10AF00001DBE000071250100695F0000DD0F01001A
:10AF1000C5BE000051770000ED2B010001373FB2A4
:10AF200000230293237A01930090059B228833A982
:10AF300048A8D847BDF8CE300133ADF8CE30BDF8C3
:10AF4000D2300133ADF8D2300135BDF9A6309D4283
:10AF50001FDC0A990598C847B8F812202A44B8F8A7
:10AF60001010BDF8A0301944099B12B209B205981F
:10AF7000D047002ED4D00028D0D0B4F90420BA4253
:10AF8000B8BF0020B4F9063013449F42A8BF002781
:10AF9000C4E70598974B9847D6E01FFA86FBBDF8A3
:10AFA0002C80A9B20BEB0802002301930F468844C2
:10AFB0000FFA88F30093534612B2059912A8DFF8EE
:10AFC0003882C0471FFA89F3ABEB030201210191DC
:10AFD000FB1A1BB20093534612B205991DA8C04735
:10AFE00070E5BDF814B0BDF82C801FFA8AF31F4637
:10AFF0004344D8440022019200951BB232460FFA16
:10B0000088F112A8DFF8F081C0471FFA89F9A7EB91
:10B010000903ABEB09090122019200951BB23246EC
:10B020000FFA89F11DA8C0474CE5BDF82880BDF88E
:10B0300024900599A1EB08030322019209EB060273
:10B0400012B200921BB2324628A86B4EB047AAEB50
:10B0500008030222019209EB050212B200921BB210
:10B060002A46514633A8B047002128A8634DA84777
:10B070000A90002133A8A8470D9036E50EA8604B32
:10B08000984783465AE5294640465E4B98472DE04F
:10B09000099A537A03F003030293137A019302236C
:10B0A00000934B46128848A910A8574CA047BDF8FA
:10B0B000463001331BB2ADF84230ADF84630594648
:10B0C0004846524B984700270136BDF93E30BAF941
:10B0D000122013449E4213DC09EB07082B4632B2C0
:10B0E000059940464A4CA0470028CCD02F44EB1984
:10B0F0009B45CDD9BDF846300133ADF84630E3E786
:10B10000099CBDF94630BDF942209A4210D0013B5E
:10B11000ADF84630637A03F003030293237A019378
:10B12000022300934B46228848A910A8364DA84711
:10B130004846304B98470B98364DA8470C98A8477F
:10B140000A98A8470D98A847637A13F00C0F02D10C
:10B150004BB0BDE8F08F33A82F4B98472388ADF84C
:10B16000CE3047F6FF73ADF8CC30237A8DF8D83067
:10B17000B4F902305E1083F0010303F00105637A35
:10B1800013F0040F1CD1637A13F0080FE0D0079975
:10B190000A88B6B2931BADF8A03049888B1BADF876
:10B1A000A230ABB23244D21AADF8A4200E44F31A46
:10B1B000ADF8A63033AA089928A8184B9847C7E7D6
:10B1C00006980288B3B2D11AADF8A0104088C11A0F
:10B1D000ADF8A210A9B21A44521AADF8A420034443
:10B1E0005B1AADF8A63033AA089928A80B4B9847EC
:10B1F000C9E700BF71250100E9BE0000C1BD000024
:10B20000FD140100372B010051770000ED2B0100E8
:10B210001DBE00006DBE000069C2000031C3000009
:10B220002DE9F041069CA58A521B12B2658A4D1B7E
:10B230002DB2216A00294BD194F8281011F0010F8A
:10B2400016D0237C03F00303012B40F2DB81022B99
:10B2500004D0032B06D00020BDE8F0810132D00FCE
:10B26000BDE8F081002AD4BF00200120BDE8F081B4
:10B27000227C02F00302911EC9B2012940F2C5816D
:10B28000012A0CD0B2B9E91800F1C2816D42002D3B
:10B29000C0F2C181AB4207DC0220BDE8F081002D85
:10B2A00008DD0120BDE8F0812844CD4B98470220FD
:10B2B000BDE8F081DD4200F1B181694221EAE1712E
:10B2C0008B4240F3AE81C64B98470220BDE8F08127
:10B2D00094F8286016F0010F0FD1A76902FB07F15F
:10B2E0008912002FCCBF01F1010E8E46754540F347
:10B2F0009880C6F34000BDE8F081E16905FB01F7E5
:10B30000BF12002906DD974240F3B881C6F3400022
:10B31000BDE8F081974280F2ED81C6F34000BDE8C0
:10B32000F08186F00200C0F34000BDE8F08186F0B5
:10B330000200C0F34000BDE8F0810025D4E1F446EE
:10B3400088F800C0636AD21A01350136BD4249DA75
:10B35000636A9A421DDD002DF4DBBD42F2DAA2EBF6
:10B360006303DBB294F828C01CF0020F1CBFDB4360
:10B37000DBB2B04696F800C0F92BE1D8052BDED938
:10B3800003FB0CF303EB032C03EBCC13C3F3C75CFD
:10B39000D6E7BD4226DA002D24DBA36903FB02F3C6
:10B3A0009B1202FB03F2C2F34722E369002BBCBFEE
:10B3B000D243D2B294F8283013F0020F1CBFD2430C
:10B3C000D2B24619435DF92A0BD8052A08D902FBE7
:10B3D00003F202EB022302EBC312C2F3C75300E0F5
:10B3E0000023337094F8283013F0020F0AD08F42F4
:10B3F000C0F21A810029C0F21A81794B98470220C5
:10B40000BDE8F081013500F11581BD4202DD022069
:10B41000BDE8F081791B2844714B98470220BDE8B4
:10B42000F08105EB030E714505DD86F00200C0F3E7
:10B430004000BDE8F081110207FB01F14FEAA1488D
:10B44000C1F387210132120207FB02F24FEAA24C3C
:10B45000A8EB050EE04563D0002F5BDBC1F1FF01D7
:10B46000E26902FB01F29512BEF1000F1CDB73458D
:10B470001ADD05FB01F1C1F3472216F0020F04BFEC
:10B48000D243D2B200EB0E0610F80E10F92A0AD8F9
:10B49000052A40F2A18002FB01F202EB022102EB3D
:10B4A000C112C2F3C75131701EF1010120D48B4289
:10B4B0001EDDC5F1FF02A56905FB02F5AD1202FB19
:10B4C00005F2C2F3472294F8285015F0020F1CBF72
:10B4D000D243D2B2455CF92A09D8052A7ED902FBAB
:10B4E00005F202EB022502EBC512C2F3C755455423
:10B4F00094F8282012F0020F74D07345C0F2B28085
:10B50000BEF1000FC0F2B1807146354B9847022062
:10B51000BDE8F081002940F000810EF1FF3EFF21DF
:10B52000BEF1000F1EDB73451CDDC2F387220A4407
:10B53000C2F3470216F0020F1CBFD243D2B200EB97
:10B540000E0610F80E10F92A0BD8052A08D902FBAE
:10B5500001F202EB022102EBC112C2F3C75100E07B
:10B560000021317094F8282012F0020F0AD0ACEBC1
:10B5700005018B4261DD002962DB194B98470220EF
:10B58000BDE8F0810EF101029A42A8BF1A46002AD6
:10B5900059D0002A5ADD991A1044114B98470220BD
:10B5A000BDE8F0810025DCE0002500E1002950DD48
:10B5B0000B4B98470220BDE8F0810EF1010E734558
:10B5C0004ADBBEF1000F4ADBA3EB0E017044044BD3
:10B5D00098470220BDE8F081002164E7002586E756
:10B5E000372B01000EF102029A42A8BF1A46002A28
:10B5F0003ED0002A3FDD991A1044734B9847022031
:10B60000BDE8F0810120BDE8F0810120BDE8F081B6
:10B610000120BDE8F0810020BDE8F0810020BDE8F8
:10B62000F0810020BDE8F0810020BDE8F08102201B
:10B63000BDE8F0810020BDE8F0810020BDE8F08188
:10B640000220BDE8F0810020BDE8F0810220BDE8C5
:10B65000F0810220BDE8F0810120BDE8F0810220E8
:10B66000BDE8F0810020BDE8F0810220BDE8F08156
:10B670000020BDE8F0810220BDE8F0811F462B4488
:10B6800001FB03F1B2EBA12F3FF74BAE1202A3690E
:10B6900003FB02F39B12191213F0FF0339D0C3F11D
:10B6A000FF03626A02FB03F24FEA222ECEF1FF0291
:10B6B000491B1AD4B94218DA0EFB03F3C3F347232C
:10B6C00016F0020F04BFDB43DBB24618455CF92BD2
:10B6D0000AD8052B7FF631AE03FB05F303EB0325F8
:10B6E00003EBC513C3F3C75535704D1C46194FF016
:10B6F000000E2DE61F462B4401FB03F1B2EBA12FF8
:10B70000FFF615AE01321202A36903FB02F39B128E
:10B71000C1E74D1B2946FF22E8E7E269524201FBDF
:10B7200002F29212BEF1000F1CDB73451ADD02FB20
:10B7300001F1C1F3472116F0020F1CBFC943C9B282
:10B7400000EB0E0610F80E50F9290AD805297FF6ED
:10B7500029AF01FB05F101EB012501EBC511C1F397
:10B76000C7553570BEF1010122D48B4220DDC2F1F4
:10B77000FF02A5696D4202FB05F5AD1202FB05F261
:10B78000C2F3472294F8285015F0020F04BFD243A9
:10B79000D2B2455CF92A0AD8052A7FF605AF02FB2A
:10B7A00005F202EB022502EBC512C2F3C755455460
:10B7B00094F8282012F0020F3FF4FFAE8B42BFF640
:10B7C000F5AE0220BDE8F081372B01002DE9F04FE6
:10B7D0008DB0169DAE7C06F00106B5F91080EC1D0B
:10B7E00005F10F090DF1280E14F8017F0EF8017B09
:10B7F0004C45F9D1002E3DD1BDF92A40944200F3C9
:10B800002B82BDF92E409442C0F22A829B460F46FD
:10B810000290BDF9289008EB0903994206DB5944D0
:10B82000BDF92C30A3EB080399420BDDBDF92A309A
:10B8300003EB08018A4253DBBDF92E10A1EB08018E
:10B840008A424DDC86BBA9EB07045C4500F30C8201
:10B85000002C03DB214602989F4B9847BDF92C0032
:10B86000C01B0130002840F3018283450DDCBCB1D0
:10B870000220F2E1BDF92A40944200F3F381BDF9C0
:10B880002E409442C2DA0120E7E1ABEB0001029BBB
:10B8900003441846904B9847002CE9D10220DCE184
:10B8A0008345E5D10120D8E1A9EB070020EAE0704B
:10B8B000584501DD0220D0E1BDF92C10C91B091A41
:10B8C000013143189B45B8BFABEB00010029C0F222
:10B8D000CF81029B034418467F4B98470220BCE16E
:10B8E000BDF92CA09BB2BDF82E100131C91A09B2C6
:10B8F000D21A08FB08F3019312B2904500F3D181EC
:10B90000A1EB0803013B9A4200F3B4810220A4E1B9
:10B910006B8BADF81A302B8BADF81830D6E1049A4A
:10B9200007A9019B00FB10306C4B9847049A06A9AD
:10B93000019B04FB1430694B98476C61BDF81A30C9
:10B940006B83BDF818302B83D1E1BDF81E100029A0
:10B9500040F0D581013AADF81C20FF22ADF81E2041
:10B96000CDE1BDF81A20BDF81E100A44C2F347020B
:10B970000EB1D243D2B2A8EB0303013BF91811D4A4
:10B9800059450FDA0298405CF92A09D8052A35D9B9
:10B9900002FB00F000EB002400EBC410C0F3C75022
:10B9A000029C6054A9EB0303013BDF1911D45F45EE
:10B9B0000FDA029BDB5DF92A09D8052A20D902FBA0
:10B9C00003F202EB022302EBC312C2F3C753029A43
:10B9D000D355BEB1481C20EAE0705F45D4BF391A88
:10B9E000ABEB0001584580F219810029C0F21681A5
:10B9F000029B03441846384B98470FE10020CFE7DD
:10BA00000023E4E7594500F32581002902DB029871
:10BA1000314B9847013700F11D815F4500F3FE80EF
:10BA2000ABEB0701029B3B4418462B4B9847F5E0D4
:10BA3000049A09A9019B08FB1830284B9847BDF8C8
:10BA40002610BDF81A30C3F1FF02C1F1FF0303FB5A
:10BA500002F3C3F347230EB9DB43DBB2039802467C
:10BA6000002811DB58450FDA029C2018A25CF92B44
:10BA700009D8052B29D903FB02F202EB022402EBC1
:10BA8000C412C2F3C7520270BAF1000F13DBDA45D9
:10BA900011DA029C04EB0A0014F80A20F92B09D8E9
:10BAA000052B14D903FB02F303EB032203EBC213B0
:10BAB000C3F3C7520270039B013B03930AF1010ACF
:10BAC000ADF8221008F101085EE10022DBE7002258
:10BAD000F0E7002739E000BF372B01001D230100EC
:10BAE00000270EF808700138013401311A46019D13
:10BAF000A94240D809EB121701FB11A307FB07FC71
:10BB0000CCEB03234FEA470C93FBFCF31F44C7F332
:10BB10000F1C3F0107F0F0031A44C2F347020EB1B5
:10BB2000D243D2B2002812DB834510DD80461EF8D6
:10BB30000070F92A09D8052ACBD902FB07F505EBD5
:10BB4000052705EBC717C7F3C7570EF80870002C79
:10BB5000C9DBA345C7DDA0461EF80470F92AC0D88A
:10BB6000052ABDD902FB07F202EB022702EBC71739
:10BB7000C7F3C757B5E7DDF81080DDF814A0EA4336
:10BB800042440399114403910135AA44AAEB080ADF
:10BB9000ADF82230ADF824C0ADF82630BDF8223023
:10BBA000002B3AD0BDF81E2003FB02F3C3F347235A
:10BBB0000EB1DB43DBB2039A002A12DB934510DDA2
:10BBC000029801461144825CF92B09D8052B27D92C
:10BBD00003FB02F202EB022002EBC012C2F3C752D7
:10BBE0000A70BAF1000F13DBD34511DD029800EBA8
:10BBF0000A0110F80A20F92B09D8052B12D903FBEA
:10BC000002F303EB032203EBC213C3F3C7520A7020
:10BC1000039B013B03930AF1010A2EB102201CE0B1
:10BC20000022DDE70022F2E703990131594511DCDA
:10BC3000002902DB0298604B9847BAF1000F09DB3C
:10BC4000DA45EBDAABEB0A01029B534418465A4B38
:10BC50009847E3E7002000E000200DB0BDE8F08F3A
:10BC60000020FAE70120F8E70020F6E70020F4E7DB
:10BC70000220F2E7B8F5807FD4BF4FF400634FF4A1
:10BC800000430493891AA8EB0100441C6B69984295
:10BC90007FF445AE6B8BADF81E302B8BADF81C30AE
:10BCA00044E6B8F5807FD4BF4FF400634FF40043FF
:10BCB0000493A8EB02046B699C423FF429AE049AFA
:10BCC00006A9019B04FB14303C4B9847631E049A61
:10BCD00007A90393019803FB1300384B9847039B74
:10BCE0006B61BDF81E306B83BDF81C302B83BDF833
:10BCF0001830BDF81C20511E8B423FF426AEA9EB34
:10BD000007070AF1010AAAEB09090FFA89F9BDF838
:10BD10001C209A423FF425AE0133A8EB030807EB41
:10BD200008030393A9EB080808F1FF3ABA4486B167
:10BD3000581C20EAE070DA45D4BFAAEB0001ABEB57
:10BD40000001584505DA002903DB029B18441A4B11
:10BD50009847BDF8180000F10108049A08A9019B52
:10BD600000FB1030154B9847BDF822303BB9BDF8A9
:10BD70002030013BADF82030FF23ADF82230BDF874
:10BD800020309C427FF754AEBDF81C50A8453FF6CA
:10BD900005AFBDF820904FEA0919BDF822204146B1
:10BDA00054460398CDF81080CDF814A0DDF804A017
:10BDB0000195DDF808E09DE6372B01001D23010009
:10BDC00010B582B0104B1B689BB10F4A01239468D9
:10BDD00084B10133DBB20832102BF8D10B4B009346
:10BDE0000B4B57220B4902200B4CA0474FF0FF3062
:10BDF00007E00023044A42F8330002EBC30251601B
:10BE000018B202B010BD00BF6C6D002024500200BB
:10BE1000C84F0200F44F02005D2201002DE9F047F7
:10BE200082B0114C2468ECB19A4691468846074688
:10BE30000D4E00250094246853464A464146384634
:10BE4000A047044650B1022808BF012556F8084F04
:10BE5000002CEFD1002D14BF02240124204602B093
:10BE6000BDE8F0870124F9E76C6D0020B0F1FF3FD9
:10BE70000AD0064B53F83010002243F8302003EB71
:10BE8000C0035A60084670470021FBE76C6D002034
:10BE900070B40B4B1A1D03F180040026354603E0F5
:10BEA00008330832A34208D059688142F8D152F8C9
:10BEB000046C42F8045C5D60F2E7304670BC704789
:10BEC0006C6D002000231846064902E00133102B58
:10BED00006D051F83320002AF8D00130C0B2F5E77F
:10BEE000704700BF6C6D00202DE9F04104460F46FD
:10BEF00015469846BDF918602C214A4B9847B54223
:10BF000005DD2B4635461E463B464746984627816B
:10BF10006581A4F80C80E681237C9DF81C2062F3E7
:10BF2000010323746782A582A8EB0707751B87EAC4
:10BF3000E771A1EBE77185EAE573A3EBE57399423D
:10BF4000D4BF0021012194F8282061F3000284F875
:10BF500028200021E161A161334B2360217112F09F
:10BF6000010F25D03FB14FF4801393FBF7F305FB8E
:10BF700003F39B12E3613DB14FF4801696FBF5F598
:10BF800007FB05F7BF12A761E3692362237C13F067
:10BF9000030322D194F828306FF3410384F828304A
:10BFA000236A9A10002BB8BF52426262BDE8F0814A
:10BFB0003DB14FF4801393FBF5F307FB03F39B12A2
:10BFC000A3613FB14FF4801898FBF7F705FB07F525
:10BFD000AD12E561A3692362D8E7012B0FD0022BD4
:10BFE00014D0032BDCD1236A002B94F82830CCBF6B
:10BFF0006FF3410343F0020384F82830D0E794F84C
:10C00000283043F0020384F82830C9E7236A002B64
:10C0100094F82830CCBF43F002036FF3410384F857
:10C020002830BDE7372B010021B2000070B4CC8866
:10C0300001344D88641B8D8801350E88AD1B24B2F8
:10C040002DB2AC42A8BF2C466410A242C8BF22B297
:10C05000013900F1100600F1080411F8015F04F83D
:10C06000015BB442F9D10282827C63F300028274E4
:10C07000054B0360022303714FF00043436100232B
:10C080004383038370BC7047CDB700002DE9F04FA8
:10C090008BB00690894607924FEA610BCDF808B045
:10C0A00011F0010F06BF0BF1FF330893CDF820B05C
:10C0B000069C67003846694B98470590002C40F372
:10C0C000BE80BA1EC1190391079D4FF0000804F10C
:10C0D000FF3A0899AAEB010104910646CDF824B075
:10C0E0009346CDF8049035F80B3009FB03F3BAF111
:10C0F000000F1BDB029A02EB0A01049A013A039833
:10C100004FF0000E20F8023D8C42CCBF35F811C034
:10C11000F446A3EB0C03002AB4BFB5F800C035F811
:10C1200012C063440139013AB042EBD13A4631467C
:10C1300028464B4B98473D4408F10108A045D0D113
:10C14000DDF824B0079A1388019993FBF1F313806B
:10C15000069B03FB03F5012D11D9079A0121019ECE
:10C16000104632F8023F008898421CBF93FBF6F35A
:10C1700013800131A942F3D3069B002B59DD079EA2
:10C180000296089901FB07726FEA0B035B1A069D82
:10C1900005FB03F306936B1E05FB03F306EB43035A
:10C1A00007934FF0000A931E089301F10109029BC7
:10C1B0001E4602331A4602933388019901FB03F3AA
:10C1C00008998D18059AA2F1020CE046B6460022A5
:10C1D000CDF80CC00496069EDDF81CC0002BACBF49
:10C1E0009911002128F8021F1146A2EB0B0000282C
:10C1F000D4BFBEF8000035F816001B1A49448C4223
:10C20000CCBF29883CF81A100B440132BE443D448F
:10C21000A242E3DBDDF80CC0049E00233CF8022FB1
:10C22000328001333E44A342F8DB0AF1010AA24501
:10C23000BDDB05980B4B98470BB0BDE8F08FCDF8F0
:10C240000490079A138893FBF9F9A2F80090069BD3
:10C2500003FB03F5012D80D8EBE700BF3D2901006A
:10C26000552601007125010010B5044654212D4BBF
:10C2700098472D4B1B88638023796FF30403237148
:10C28000A3886FF34A13A3801B0A6FF3C70363717C
:10C29000A37B6FF30403A373E3896FF34A13E38172
:10C2A0001B0A6FF3C703E37394F834306FF304038E
:10C2B00084F83430A38E6FF34A13A3861B0A6FF3FE
:10C2C000C70384F8353094F846306FF3040384F8DC
:10C2D0004630B4F846306FF34A13A4F846301B0AD0
:10C2E0006FF3C70384F84730A37F6FF30403A3778A
:10C2F000E38B6FF34A13E3831B0A6FF3C703E37700
:10C30000FF23638123732377237584F83630074A2C
:10C31000226384F84430226484F828300F23638237
:10C3200010BD00BF372B01007C5002001000002020
:10C330002DE9F04FB1B0C4884588631C5B1B1BB26C
:10C34000002B41F30F808688B0F80080731CA3EBAC
:10C3500008031BB2002B41F305809246049106901E
:10C36000B2F92070002F00F0198792F82830099355
:10C37000052B40F21387136A012B00F0F680BAF800
:10C380002220BAF82630D11A88441FFA88F8ADF86E
:10C3900050801A441644B6B2ADF85460BAF824205E
:10C3A000D11A0D44ADB2ADF8525013441C44A4B29E
:10C3B000ADF8564007EBD7736FEA630292B208EB11
:10C3C0000201ADF858105B1001339BB2F118ADF8C3
:10C3D0005C102A44ADF85A202344ADF85E30099B26
:10C3E000FB2B28BFFF230993BE4B9847BE4B9847B2
:10C3F0008146049A16A918A8BC4B9847002800F05B
:10C40000CD86B9F81010BDF860305B1AADF8603019
:10C41000B9F81220BDF862309B1AADF86230BDF851
:10C4200064305B1AADF86430BDF866309B1AADF825
:10C430006630069A531ED01D1AAA13F8011F02F87F
:10C44000011B9842F9D1BDF8683001331FFA83FE11
:10C45000ADF868E0BDF86A10013188B2ADF86A0045
:10C46000BDF86C305A1EADF86C20BDF86E104A1E37
:10C47000ADF86E20BAF90020A3EB0E031BB2091A27
:10C4800009B28B42A8BF0B465B109342A8BF13466C
:10C490000E930136A6EB0806B6B233B20134641B24
:10C4A000A4B225B29D42A8BF1D466D109542A8BFFB
:10C4B000154607EB050909FB09F040008C4B98472E
:10C4C0000A90BAF920B02AB202EB0B070DF14F0126
:10C4D00022AB0DF1900E11F8010F03F8010B73451B
:10C4E000F9D10BEBDB71C1F34F014B1E1BF00100C7
:10C4F00010900CBF012000201B1A2B449BB2ADF8FA
:10C500008C30013189B2ADF88A109B1BADF88830B0
:10C510002144ADF88E10002322A929A8754CA0470C
:10C52000BBF1010F02F0D8814FEA6B030B93079721
:10C5300038466F4B98470C90002F5CDD079B4FEA05
:10C54000430B07F10043013B5B000A9C0025DFF829
:10C55000B8813AB20892CDF8349005970C9E99466E
:10C56000CDF83CA0DDF82CA014E0B2F92430002B6B
:10C570007FF405AFB2F92630002B3FF700AF00F093
:10C580000DBE594620465C4B98475C440135059BDF
:10C59000AB422BDD07993046C04729AB0093089B7F
:10C5A0002AB200213046299FB8470028E9D0D64654
:10C5B00033789B0193FBFAF32380059B012BE4DD89
:10C5C0003146224604EB09001F468C4611F8013F14
:10C5D0009CF800C09C450EBF13889B0193FBFEF3A3
:10C5E000538002329042F0D10597CEE7DDF83490C7
:10C5F0001F46DDF83CA00C98404B98470B9B012B45
:10C6000002F04D813CB20A9E32460B9D29462046DF
:10C610003B4B9847109A2A4411B2012922DD0D465E
:10C6200033889B0193FBF1F332463380079800FB7C
:10C6300000F0012812D900F10040013806EB40005B
:10C6400001E082420AD0164632F8023F36889E4206
:10C65000F7D09B0193FBF5F31380F2E70A9A20468B
:10C66000274B984707FB07F757B10A990B464A1E15
:10C6700001EB470033F8021B02F8011F8342F9D196
:10C68000BDF85A20BDF85E3001339B1A1BB203EB94
:10C69000D37302EB63039BB20F931BB20C93BDF8F1
:10C6A0005820BDF85C3001339B1A1BB203EBD373E7
:10C6B00002EB63039BB210931BB20D93114B98478F
:10C6C00020BBBAF92230002B40F0BC81BAF92430EB
:10C6D000002B40F0BA81BAF92630B3FA83F35B0934
:10C6E000079315E0695F0000DD0F010019150100D7
:10C6F0003D2901002DC00000372B010071250100EC
:10C700008DC00000C5BE0000ED2B01000023079383
:10C71000BDF85C000130BDF85830C01A00B2C24B01
:10C720009847059001230E9A1AA929A8BF4CA04743
:10C73000002129A8BE4B98470E90BDF95C30ADF89A
:10C7400074301FFA89FB0133A3EB0B03ADF8703093
:10C75000BDF95A30ADF87230013B5B44ADF876302C
:10C76000049A1CA91EA8B34B9847002872D0BDF9A3
:10C770007E300C998B42C4BF0B46ADF87E30BDF9BC
:10C7800078300D9A934203DC109B0133ADF878307A
:10C79000BDF97820BDF87C3001339B1A1BB2089399
:10C7A000002B57DDBDF97E70BDF97A40BDF972509E
:10C7B000651BBDF97030D21A09FB05250A9B1D4483
:10C7C0000DF1770222AB24A812F8011F03F8011B18
:10C7D0008342F9D1BDF88A30ADF88E3001373F1B66
:10C7E0003FB2002F36DD0026DFF85482CDF844B08A
:10C7F000BB46099B0B93089A2946059F38468E4CE9
:10C80000A04730AC089BBDF98A2034F9381D059744
:10C8100038468A4FB847012808BF02209AF82930C5
:10C8200002930B9A01920090059BBAF81E202146B4
:10C830000498C047BDF88A300133ADF88A30BDF89E
:10C840008E300133ADF88E304D4401365E45D2D185
:10C85000DDF844B0BDF95C30ADF874300133A3EBC2
:10C860000B03ADF87030BDF95E20531CA3EB0B0336
:10C87000ADF87230ADF87620049A1CA91EA86D4B55
:10C880009847002873D0BDF97A300C9A934203DCA4
:10C890000F9B0133ADF87A30BDF978300D9A934291
:10C8A00003DC109B0133ADF87830BDF97820BDF87A
:10C8B0007C3001339B1A1BB20893002B57DDBDF966
:10C8C0007E40BDF97A60BDF976502D1BBDF9703000
:10C8D000D21A09FB05250A9B1D440DF1770222ABF4
:10C8E00024A812F8011F03F8011B8342F9D1BDF8F7
:10C8F0008E30ADF88A30671CBF1B3FB2002F36DD8B
:10C900000026DFF83C81CDF840B0BB46099B0B9375
:10C91000089A2946059F3846474CA04730AC089BEB
:10C92000BDF98A2034F9381D05973846434FB8477A
:10C93000012808BF02209AF8293002930B9A01922D
:10C940000090059BBAF81E2021460498C047BDF808
:10C950008A30013BADF88A30BDF88E30013BADF82E
:10C960008E304D4401365E45D2D1DDF840B0BDF980
:10C970005C30ADF874300133A3EB0B03ADF87030CD
:10C98000BDF85A305B44ADF87230BDF85E30A3EBB1
:10C990000B03ADF87630049A1CA91EA8254B9847C6
:10C9A000002800F08580079B4BB1069BB3F904304B
:10C9B000BDF978209342B8BF1346ADF87830BDF981
:10C9C0007830BDF87C200132D21A0FFA82F8B8F123
:10C9D000000F6DDDBDF87E400134BDF87A20A41A49
:10C9E00024B209F1FF31BDF970209B1A09FB013314
:10C9F0000A9AD31808930DF1770222AB24A812F8F3
:10CA0000011F03F8011B8342F9D1BDF88A30ADF84C
:10CA10008E302546002C4BDD0024074FCDF82C909E
:10CA2000A946079D3AE000BF3D2901002DC0000046
:10CA3000C1BD000019150100552601001DBE0000F2
:10CA4000517700000023079362E6002307935FE617
:10CA50004346BDF98A20BDF988100598234EB0479A
:10CA6000012808BF02209AF8293002939AF828304A
:10CA700001930090059BBAF81E2022A904981C4E31
:10CA8000B047BDF88A300133ADF88A30BDF88E303A
:10CA90000133ADF88E3001344C4507D04246089939
:10CAA0000598B847002DD3D00220DCE7DDF82C90A4
:10CAB000B9F1000F1EDD09EBD9777F100A9D002622
:10CAC0000CE0197812F8010C03F8010B02F8011DB3
:10CAD000A342F6D14D440136B1450BD0002FF9DD0C
:10CAE0002B4605EB0902EC19EBE700BF1DBE000069
:10CAF00051770000BDF95830ADF87030013B5B4410
:10CB0000ADF87430BDF95A30ADF87230013B5B447A
:10CB1000ADF87630049A1CA91EA8AE4B98470028A1
:10CB200071D0BDF97E300C998B42C4BF0B46ADF875
:10CB30007E30BDF97C300D998B42C4BF0B46ADF8F9
:10CB40007C30BDF97820BDF87C3001339B1A1BB2D4
:10CB50000893002B57DDBDF97E70BDF97A40BDF911
:10CB60007250651BBDF97030D21A09FB05250A9B6E
:10CB70001D440DF1770222AB24A812F8011F03F81F
:10CB8000011B8342F9D1BDF88A30ADF88E300137F0
:10CB90003F1B3FB2002F36DD0026DFF84482CDF880
:10CBA00040B0BB46099B0B93089A2946059F38461F
:10CBB000894CA04730AC089BBDF98A2034F9381D58
:10CBC00005973846854FB847012808BF02209AF8D4
:10CBD000293002930B9A01920090059BBAF81E200F
:10CBE00021460498C047BDF88A300133ADF88A3039
:10CBF000BDF88E300133ADF88E304D4401365E45C0
:10CC0000D2D1DDF840B0BDF95830ADF87030013BFD
:10CC10005B44ADF87430BDF95E20531CA3EB0B03ED
:10CC2000ADF87230ADF87620049A1CA91EA8694BA5
:10CC30009847002872D0BDF97A300C9A934203DCF1
:10CC40000F9B0133ADF87A30BDF97C300D998B42E2
:10CC5000C4BF0B46ADF87C30BDF97820BDF87C3000
:10CC600001339B1A1BB20893002B57DDBDF97E40A0
:10CC7000BDF97A60BDF976502D1BBDF97030D21A1E
:10CC800009FB05250A9B1D440DF1770222AB24A860
:10CC900012F8011F03F8011B8342F9D1BDF88E3051
:10CCA000ADF88A30671CBF1B3FB2002F36DD00266F
:10CCB000DFF82C81CDF830B0BB46099B0B93089A66
:10CCC0002946059F3846444CA04730AC089BBDF927
:10CCD0008A2034F9381D05973846404FB847012857
:10CCE00008BF02209AF8293002930B9A0192009013
:10CCF000059BBAF81E2021460498C047BDF88A302B
:10CD0000013BADF88A30BDF88E30013BADF88E3076
:10CD10004D4401365E45D2D1DDF830B0BDF9583012
:10CD2000ADF87030013B5B44ADF87430BDF85A305B
:10CD30005B44ADF87230BDF85E30A3EB0B03ADF889
:10CD40007630049A1CA91EA8224B9847002879D057
:10CD5000079B4BB1BDF97C30069AB2F90020934293
:10CD6000A8BF1346ADF87C30BDF97830BDF87C80A3
:10CD700008F10108A8EB03080FFA88F8B8F1000FD2
:10CD800060DDBDF87E400134BDF87A20A41A24B2DB
:10CD900009F1FF31BDF970209B1A09FB01330A9A92
:10CDA000D31808930DF1770222AB24A812F8011FC3
:10CDB00003F8011B8342F9D1BDF88A30ADF88E30FB
:10CDC0002546002C3EDD0024034FCDF82C90A946CB
:10CDD000079D2DE019150100552601001DBE00001C
:10CDE000517700004346BDF98A20BDF988100598A7
:10CDF000AA4EB047012808BF02209AF829300293B2
:10CE00009AF8283001930090059BBAF81E2022A9B9
:10CE10000498A34EB047BDF88A300133ADF88A308C
:10CE2000BDF88E300133ADF88E3001344C4507D05B
:10CE3000424608990598B847002DD3D00220DCE778
:10CE4000DDF82C90BDF858305B44ADF87030BDF87B
:10CE50005C30A3EB0B03ADF87430BDF95A30ADF87C
:10CE60007230013B5B44ADF87630049A1CA91EA8D1
:10CE70008C4B984700287DD0079B4BB1069BB3F99C
:10CE80000230BDF97E209342A8BF1346ADF87E3034
:10CE9000BDF87C300133BDF878209B1A1BB2089393
:10CEA000BDF97A30BDF87E500135ED1A2DB2C84675
:10CEB000BDF972401C1B09F1FF3309FB04340A9BC6
:10CEC0001C440DF1770222AB24A812F8011F03F8CD
:10CED000011B8342F9D1BDF88A30ADF88E302B4664
:10CEE000002D47DD0025704FCDF82C90DDF8249003
:10CEF000CDF830B09B462AE0B9F1FF0F2AD1494660
:10CF00002CE0089BBDF98A20BDF988100598634E76
:10CF1000B047012808BF02209AF829300293FF2366
:10CF200001930090059BBAF81E2022A904985C4E3C
:10CF3000B047BDF88A300133ADF88A30BDF88E3085
:10CF40000133ADF88E30444401355D450ED0237871
:10CF5000FF2BD1D003FB09F3C3F30721089A0598EF
:10CF6000B847079B002BCCD00220D5E7DDF82C90EA
:10CF7000DDF830B0BDF858305B44ADF87030BDF826
:10CF80005C30A3EB0B03ADF87430BDF95E20531C8D
:10CF9000A3EB0B03ADF87230ADF87620049A1CA910
:10CFA0001EA8404B9847002800F08280079B4BB199
:10CFB000069BB3F90630BDF97A209342B8BF1346F9
:10CFC000ADF87A30BDF87C300133BDF878209B1A7B
:10CFD0001BB20893BDF97E305D1CBDF87A20AD1AF6
:10CFE0002DB2C846BDF97640E41A09F1FF3309FBBA
:10CFF00004340A9B1C440DF1770222AB24A812F8DA
:10D00000011F03F8011B8342F9D1BDF88E30ADF842
:10D010008A30A946002D4BDD0025234FCDF82CB0DA
:10D02000DDF824B02AE0BBF1FF0F2AD159462CE0ED
:10D03000089BBDF98A20BDF988100598174EB047A6
:10D04000012808BF02209AF829300293FF23019398
:10D050000090059BBAF81E2022A90498104EB047F4
:10D06000BDF88A30013BADF88A30BDF88E30013B07
:10D07000ADF88E30444401354D4517D02378FF2B51
:10D08000D1D003FB0BF3C3F30721089A0598B847E7
:10D09000079B002BCCD00220D5E700BF1DBE0000AF
:10D0A0005177000019150100812A0100DDF82CB02C
:10D0B000BDF858305B44ADF87030BDF85C30A3EB80
:10D0C0000B03ADF87430BDF85A305B44ADF87230E4
:10D0D000BDF85E30A3EB0B0BADF876B0049A1CA93B
:10D0E0001EA8A24B9847002850D0079B002B4DD17B
:10D0F000BDF87C600136BDF87830F61A36B2BDF85E
:10D100007E400134BDF87A30E41A24B20DF1770282
:10D1100022AB24A812F8011F03F8011B8342F9D1A6
:10D12000BDF88A30ADF88E30A346002C2EDD0025E8
:10D13000DFF85492DFF854828D4F32469AF8281067
:10D140000598C84730AC3346BDF98A2034F9381DFC
:10D150000598C047012808BF02209AF82930029399
:10D16000FF2301930090059BBAF81E2021460498E6
:10D17000B847BDF88A300133ADF88A30BDF88E303B
:10D180000133ADF88E3001355D45D6D10E98794B1F
:10D1900098470598784CA0470A98A0479AF80C70D1
:10D1A000052F42D9069A531ED01D1AAA13F8011F43
:10D1B00002F8011B9842F9D1BAF91030012B24DD95
:10D1C0009AF81430F92B20D9BAF90030EBB1BAF83B
:10D1D0001230C3F38002BDF868100A44ADF868202D
:10D1E000C3F34002BDF86A100A44ADF86A20C3F3E5
:10D1F000C001BDF86C20521AADF86C2003F0010399
:10D20000BDF86E20D31AADF86E30FB2F28BFFF2774
:10D210005A4B98475A4B98478046049A1AA91CA81B
:10D22000524B9847002840F0B380DAF82C0020B128
:10D230009AF83630052B00F2EB839AF81440052C4F
:10D2400015D9BAF9103093B1BAF912307BB1FB2C71
:10D2500028BFFF24494B9847494B98470546049AF5
:10D26000069918A8414B9847002840F04685DAF8FF
:10D270003C1021B19AF84430052B01F253809AF802
:10D280001CB0BBF1050F6DD9BAF91830002B69D06D
:10D29000BBF1FB0F28BF4FF0FF0B3A4B98470990AB
:10D2A000069A531ED01D16AA13F8011F02F8011B7F
:10D2B0008342F9D1BAF81A50BDF858305B1B9BB2C3
:10D2C0000693ADF85830BDF85A305B1B9BB20793FC
:10D2D000ADF85A30BDF85C602E44B6B2ADF85C6073
:10D2E000BDF85E301D44ADB2ADF85E50BAF9003005
:10D2F0000893BAF9183005930DF1570218AB1AA824
:10D3000012F8011F03F8011B8342F9D1BDF8144044
:10D31000BDF86090A9EB04091FFA89F30A93ADF8F0
:10D320006030BDF864702744BFB2ADF86470BDF8DA
:10D330006280A8EB04081FFA88F8ADF86280BDF897
:10D3400066301C44A4B2ADF866400C4B98470C4BB9
:10D3500098478146049A18A91AA8044B98470028B0
:10D3600041F0448031B0BDE8F08F00BF19150100D5
:10D37000517700006DBE000071250100695F00005B
:10D38000DD0F0100C5BE0000812A01001DBE0000A6
:10D39000B8F81010BDF870305B1A9AB2ADF8702072
:10D3A000B8F81200BDF872301B1AADF87230BDF833
:10D3B00074305B1A9BB2ADF87430BDF87610091A60
:10D3C000ADF8761001339B1A1BB209930A931846E5
:10D3D000934B98470590934B984783B20B9343BB6D
:10D3E0009AF80630023B18BF01230793BDF86C5032
:10D3F0000135BDF86830ED1A2DB22C46BAF900207F
:10D40000BDF86E300133BDF86A609B1B1EB2334617
:10D41000AE42A8BF2B465E109642A8BF1646079B99
:10D42000DBB1D6B99AF8063033B14FF0FF330E9323
:10D4300021E000230793D9E79AF80D300293019772
:10D44000012300930023BAF802201AA90498764C0D
:10D45000A0474FF0FF330E9376E2002E32DD00231B
:10D4600032461AA929A8DFF8D091C847002129A877
:10D470006E4B98470E90BAF802B09AF80630022B1D
:10D4800024D000230D93BDF96C20BDF96810531C06
:10D490005B1A1BB2A3EB4609ADF87810ADF87C20FF
:10D4A000BDF97220B8F8123013441BB2ADF87A30CF
:10D4B000ADF87E301546BDF976309A4200F33782DA
:10D4C0000897FAE04FF0FF330E93D4E7BAF8043030
:10D4D0009B4500F089806800514B98470D90002DC6
:10D4E000D1DD4FF00009089606461BE09AF802309D
:10D4F00003F01F03BAF80210C1F345119AF8032094
:10D50000D208287863F3040028702B8861F34A134B
:10D510002B801B0A62F3C7036B7009F10109023605
:10D520004C455FD03546BAF9080000FB04F31B12E6
:10D530000FFA89F18B42D9DABAF90A2002FB04FE0C
:10D54000B1EB2E2F42DA121A04FB02F2A9EB03030D
:10D550001BB2C3EB0323121293FBF2F3DBB2C3F152
:10D56000FF0E9AF80520D2089AF80310C9080EFB9E
:10D5700001F103FB021202EB022102EBC112C2F322
:10D58000C452BAF80410C1F34511BAF80200C0F34E
:10D5900045100EFB00F003FB010101EB012001EB44
:10D5A000C011C1F3C5519AF8040000F01F009AF8A9
:10D5B00002C00CF01F0C0EFB0CFE03FB00E303EBA0
:10D5C000032003EBC013C3F3C4539AE79AF8043063
:10D5D00003F01F03BAF80410C1F345119AF80520AF
:10D5E000D2088EE7089E4EE700230D934BE70A9979
:10D5F000059F38460E4B9847B8F812202A44B8F8D1
:10D600001010BDF870301944099B12B209B23846A7
:10D61000084FB84707469AF80630012B29D17AE01F
:10D620003D290100C5BE000051770000C1BD0000CA
:10D63000ED2B01001DBE00002DC000000A99059FC2
:10D640003846B64B9847B8F812202A44B8F810105C
:10D65000BDF870301944099B12B209B23846B04F78
:10D66000B84707469AF80630012B54D0079A002A8B
:10D670003AD1022B00F044810B9B13B9B9F1320F60
:10D680000BDC9AF80D300293089B01930097059BE1
:10D690005A461EA90498A34CA047BDF87A3001331E
:10D6A000ADF87A30BDF87E300133ADF87E3001350B
:10D6B000BDF976309D4200F33981B8F912402C440F
:10D6C000BDF96A30334401339C42B7DDBDF96E3099
:10D6D0009B1B013B9C42B1DA079B002B87D09AF839
:10D6E0000630012B16D00127B9F1320F00F39380D9
:10D6F000022B00F00581012BBED19AF80D30029368
:10D70000089B01930097059B5A461EA90498854CD7
:10D71000A047C2E70127BAF80220BAF804309A42BB
:10D720006FD0BDF86A10621A93B21A460C93BAF918
:10D7300008E0BDF86E3001335B1A1BB203FB0EF13B
:10D74000091210B281424BDABAF90AC00CFB03F29B
:10D75000B0EB222F80F2B080ACEB0E0E03FB0EF389
:10D760000C9A521A12B2C2EB02221B1292FBF3F372
:10D77000DBB2C3F1FF019AF80520D2089AF8030042
:10D78000C00801FB00F003FB020202EB022002EBE7
:10D79000C012C2F3C452BAF80400C0F34510BAF87C
:10D7A00002E0CEF3451E01FB0EFE03FB00E000EBA2
:10D7B000002E00EBCE10C0F3C5509AF804E00EF036
:10D7C0001F0E9AF802C00CF01F0C01FB0CF103FBBA
:10D7D0000E1303EB032103EBC113C3F3C4530AE09D
:10D7E0009AF8023003F01F03BAF80200C0F34510A4
:10D7F0009AF80320D20863F3040B60F34A1B62F328
:10D80000CF2B079B002B3FF478AFB9F1320FC8BF85
:10D8100001237FF772AFBDF96A203244013294428E
:10D8200006DBBDF96E20921B013A94427FF760AF90
:10D83000BDF96830ADF88830B2B20C92013B1344A8
:10D84000ADF88C30BDF87A30ADF88A30BDF87E3056
:10D85000ADF88E309AF80D300293089B0193009733
:10D86000059B5A4622A904982E4CA0479AF80630E8
:10D87000012B2DD0BDF96C305A1C0C99541AADF8FF
:10D880008840ADF88C309B1B0133B8F91020BDF9EE
:10D8900070100A449B1A9AF80D200292089A01927D
:10D8A0000097059A002BA8BFD21813465A4622A902
:10D8B00004981C4CA047F0E69AF8043003F01F03CC
:10D8C000BAF80400C0F345109AF80520D20892E790
:10D8D000BDF868300C9A1344ADF88830BDF86C3050
:10D8E0009B1AADF88C309AF80D300293089B019387
:10D8F0000123009300235A4622A90498A047B9E7C0
:10D900009AF80D300293089B01930097059B0D9A9E
:10D910001EA90498044CA047BFE600BFED2B0100F0
:10D920001DBE00005177000081820000089F9AF818
:10D93000063023B90B9B13B9B9F1320F0BDC0D9BE9
:10D9400013B11846B34B98470E98B34B98470598B8
:10D95000B04B984769E4B6B2BDF868303344ADF8CF
:10D960007830BDF86C309B1BADF87C30BDF96A3067
:10D97000ADF87A303344ADF87E309AF80D3002932A
:10D980000197012300930023BAF802201EA90498EE
:10D99000A24CA047BDF96E108A1B12B2ADF87A20D6
:10D9A000BDF97E309A42DCBF0133ADF87A30ADF874
:10D9B0007E109AF80D3002930197012500950023FF
:10D9C000BAF802201EA9DDF810804046934CA0470B
:10D9D000BDF86830ADF87830BDF86C30ADF87C300B
:10D9E000BDF86A302B443344ADF87A30BDF86E3060
:10D9F000013B9E1BADF87E609AF80D3002930197B3
:10DA000000950023BAF802201EA94046A04796E7D9
:10DA1000834B98470546012812D9022839D0814BFB
:10DA20000093814B40F2AE5280490220804CA047C7
:10DA300000231A46049906987E4CA047FFF7FDBBC9
:10DA400029A9DAF82C007C4B984701280AD07B4B97
:10DA50000093754B40F2945274490220744CA047D5
:10DA6000FFF7EBBB299BC3F38A29BDF8A670C7F368
:10DA70004A171EA8724B98479AF836308DF87830BE
:10DA80009AF837308DF88230BAF83430ADF88430F7
:10DA900020E022A86B4B9847BAF83430ADF88830B4
:10DAA000DAF8302023929AF836308DF89030BDF9AC
:10DAB00094300021029147F618410191BDF992106E
:10DAC0000091DAF82C1029A85F4CA047BDF9A4906A
:10DAD000BDF9A6709AF8383013F0010F3FD1069CBB
:10DAE00021886088E2880132121A12B2A3880133B9
:10DAF0005B1A1BB2A3EB090303EBD37301EB6303C4
:10DB00009BB2ADF87030D21B02EBD27100EB610119
:10DB100089B2ADF8721009F1FF399944ADF87490EB
:10DB20007B1E0B449BB2ADF87630022D00F0BD8019
:10DB3000BAF9002006991CA8444B98474FF0FF34CF
:10DB4000002800F0D4861EABDAF82C2004991CA81B
:10DB5000384DA8472046304B9847FFF76EBB00234F
:10DB6000BAF90020069E314629A8394CA047002169
:10DB700029A8384B98470790B38801333446328838
:10DB80009B1A1BB293FBF9F209FB123303EBD3731D
:10DB90004FEA630BB6F9061073884A1CD21A10B20A
:10DBA00090FBF7F207FB120202EBD272A3EB6203C7
:10DBB0009BB21AB2ADF87220BFB2781E0344ADF822
:10DBC000763091426CDBDFF890801A4ECDF81490DD
:10DBD000A14652E000230093DAF82C3022AA0499DF
:10DBE0001CA8C047BDF8703023441BB2ADF870309C
:10DBF000BDF874202244ADF87420B9F904209A428B
:10DC00002CDB022DE6D01EABDAF82C2004991CA8E0
:10DC1000B047E7E7712501006DBE000051770000B5
:10DC200069990000E050020080500200905002000C
:10DC30005D220100E9960000EDFD0000C0500200E9
:10DC400045960000CD9900007D4001006D17010050
:10DC50002DC00000C1BD0000259A0000BDF8723043
:10DC60003B441BB2ADF87230BDF876203A44ADF8B3
:10DC70007620B9F906209A4212DBB9F80030A3EBFE
:10DC80000B039BB21AB2ADF87020BDF81440611EB0
:10DC90000B44ADF87430B9F904309342B1DADDE7E2
:10DCA00007988A4B9847FFF7C8BA02F0010211445F
:10DCB000ADF872101344ADF87630BAF90020214661
:10DCC0001CA8834B9847A8B90023BAF900200699ED
:10DCD00029A8804CA047002129A87F4B98470446DB
:10DCE00000230093DAF82C3022AA04991CA87B4D5B
:10DCF000A8472FE74FF0FF34F2E7298ABDF86030DC
:10DD00005B1A9AB2ADF86020688ABDF862301B1ABF
:10DD1000ADF86230BDF864305B1A9BB2ADF8643088
:10DD2000BDF86610091AADF8661001339B1A1BB2D4
:10DD30000893099318466A4B98478346694B98475E
:10DD400048B9BAF91280B8F10F0F14BF4FF00008AC
:10DD50004FF0010801E04FF00008BAF90020069EDC
:10DD6000B388013331885B1A19B2F38801337088A4
:10DD70001B1A1BB28B42A8BF0B465B109342A8BF75
:10DD800013461A460A93002B40F38880002331463D
:10DD900022A8504EB047002122A84F4B98470E9022
:10DDA000BAF91060069A531ED01D1AAA13F8011F63
:10DDB00002F8011B8342F9D1BDF86820BAF812308D
:10DDC00013F0040F6ED0B1B20A44ADF86820BDF86C
:10DDD0006C2013F0080F6AD0B1B2521AADF86C2063
:10DDE000BDF86A2013F0020F66D0B1B20A44ADF854
:10DDF0006A20BDF86E2013F0010F62D0B3B2D31ABF
:10DE0000ADF86E30DDF828901FFA89F7BA1B0123B0
:10DE100012B21AA929A82F4EB047002129A82E4BCB
:10DE200098470F90BAF91030013B4B45B8BF4B46AD
:10DE300019460D93BAF80E30ADF814309AF8156003
:10DE4000B8F1000F00F0BF81B5F912300698B0F9B3
:10DE50000220D21A0A44BDF966109142A8BF1146A9
:10DE60000B910288ADF870208288ADF87420BDF95E
:10DE7000622013441BB2ADF87230ADF87630904694
:10DE80000B9B9342C0F2B380DFF85C90CDF81CB0DE
:10DE9000B3462646CDF830A0824655E04FF0FF331A
:10DEA0000E937DE70A997118494289B28CE70A9965
:10DEB0007118494289B290E70A997118494289B2AA
:10DEC00094E70A9BF3185B429BB298E76DBE000093
:10DED0006D1701002DC00000C1BD0000259A000093
:10DEE0003D290100C5BE000051770000BAF9043099
:10DEF0005A1CD21BADF87820ADF87C300A9A9B1AD8
:10DF00000133B5F91020BDF960100A449B1ACDF811
:10DF100008B001960094079A002BA8BFD2181346A8
:10DF2000BDF814201EA90498C847BDF8723001330B
:10DF3000ADF87230BDF876300133ADF8763008F1C7
:10DF400001080B9B43454CDB0999079C2046C74BB6
:10DF500098476A8A4244298ABDF860301944089B70
:10DF600012B209B207942046C14CA0470446BDF83E
:10DF70007230ADF87A30BDF87630ADF87E30BAF94F
:10DF80000030ADF87830013B3B44ADF87C30CDF843
:10DF900008B001960090079BBDF814201EA90498B4
:10DFA000C847BDF97E20BAF902300C99B1F91010BA
:10DFB0000B449A429ADABAF800303B44ADF8783014
:10DFC000BAF80430DB1BADF87C30CDF808B0019610
:10DFD000012300930023BDF814201EA90498C8470C
:10DFE00084E734465E46DDF81CB0DDF830A0B5F9B4
:10DFF0001230069AB2F90620D21A0D99521ABDF9BA
:10E0000062809045B8BF90460B994145A8BF01F189
:10E01000010843441BB2ADF87230ADF87630BDF95B
:10E020006630984500F38D80DFF84892CDF81CB03B
:10E03000B3462646CDF82CA0DDF818A02EE0BAF99C
:10E0400004305A1CD21BADF87820ADF87C300A9A07
:10E050009B1A0133B5F91020BDF960100A449B1AD0
:10E06000CDF808B001960094079A002BA8BFD218EB
:10E070001346BDF814201EA90498C847BDF8723095
:10E080000133ADF87230BDF876300133ADF876303B
:10E0900008F10108BDF9663098454CDC0999079CE8
:10E0A0002046724B98476A8A4244298ABDF86030FC
:10E0B0001944089B12B209B2079420466C4CA04741
:10E0C0000446BAF90030ADF87830013B3B44ADF876
:10E0D0007C30BDF87230ADF87A30BDF87630ADF8EE
:10E0E0007E30CDF808B001960090079BBDF8142053
:10E0F0001EA90498C847BDF97E20BAF906300B99CD
:10E10000B1F910105B1A9A4299DDBAF800303B441D
:10E11000ADF87830BAF80430DB1BADF87C30CDF8C0
:10E1200008B00196012300930023BDF814201EA916
:10E130000498C84783E734465E46DDF81CB0DDF836
:10E140002CA0BDF8342006994B8801331344ADF858
:10E150007230CB88013B9B1AADF87630B1F90030B4
:10E16000ADF87030BAF81020013A1344ADF87430AD
:10E1700002960194012700970023BDF814904A46A7
:10E180001CA9DDF8108040463A4DA847069BB3F91C
:10E190000420BAF81030FB1A1344ADF87030ADF813
:10E1A000742002960194009700234A461CA9404619
:10E1B000A8470F98304CA0470E98A04758462F4BC1
:10E1C0009847FFF754B8069AB2F90010ADF87010EE
:10E1D000B2F90420ADF87420BDF962006B8A0344E3
:10E1E0001BB2ADF87230ADF87630BAF91230042BAC
:10E1F00029D0082B44D000228DF84E208DF84F20D6
:10E20000022B29D101238DF84E309DF84E301BB9D9
:10E210009DF84F8088F0010808F001088DF85080C3
:10E220000746BDF966309842C3DCDFF84080DFF86E
:10E2300044900A94CDF81CB0DDF818B0CDF82CA0AD
:10E24000DDF834A04EE00D9A1144ADF874100022B0
:10E250008DF84E208DF84F20012B16D0032BD4D1F2
:10E2600001238DF84E308DF84F30CEE7ED2B0100B5
:10E270001DBE0000517700006DBE00007125010039
:10E280000D99521AADF87020E1E78DF84F30BCE7D8
:10E290000999079C2046C0476A8A3A44298ABDF8F2
:10E2A00060301944089B12B209B207942046984C7A
:10E2B000A04702960A9A01920090079BBDF814208D
:10E2C0001CA90498C847BDF872300133ADF872300C
:10E2D000BDF876300133ADF876300137BDF96630E0
:10E2E0009F421ADC9DF85030002BD1D19DF84E3062
:10E2F00033B1BDF97220BBF9023053449A42C7DDF5
:10E300009DF84F30002BDED0BDF97220BBF90630EE
:10E31000A3EB0A039A42D6DBBAE7DDF81CB0DDF8BE
:10E320002CA046E7BAF94C300024029447F6184274
:10E330000192BAF94E200092DAF840201CA8754DDF
:10E34000A847ADF88840ADF88A40BDF87030013B71
:10E35000ADF88C30BDF87230013BADF88E301EAB9D
:10E360009AF8502022A906986B4DA847BDF878204E
:10E37000BAF848301A4492B2BDF888301344ADF868
:10E380008830BDF87A30BAF84A100B449BB2BDF819
:10E390008A101944ADF88A10BDF88C100A44ADF803
:10E3A0008C20BDF88E201344ADF88E3029A85B4B2D
:10E3B0009847DAF840302A93BAF84C30ADF8B030CC
:10E3C000BAF84E30ADF8AE30BAF84630ADF8A430F9
:10E3D0009AF844308DF8AC300094DAF83C3029AA31
:10E3E000049922A84E4CA047FEF749BF721C069B19
:10E3F000D21A12B26B1C07995B1A1BB29A42A8BFC1
:10E400001A465210089B9A42A8BF1A46059B13440D
:10E4100001370A99791A08B2611CA1EB080109B207
:10E420008142A8BF014649109942A8BF19460F462C
:10E430000691B9F81000BDF868301B1A99B2ADF812
:10E440006810B9F81240BDF86A301B1BADF86A308D
:10E45000BDF86C301B1A9BB2ADF86C30BDF86E0085
:10E46000001BADF86E0001335B1A1BB21E4607930A
:10E47000012316A922A82B4DA847002122A82A4C27
:10E48000A0470C9000233AB218A929A8A847002158
:10E4900029A8A0470D9008963046244B98470B902A
:10E4A000BAF91830BAF81620ADF814209AF81D50B1
:10E4B000099A002A40F0A681013BBB42B8BF3B4607
:10E4C00019460E93B9F91230BDF96220D21A0A44E6
:10E4D00011460992BDF86020ADF87020BDF86420A7
:10E4E000ADF87420BDF96A2013441BB2ADF8723048
:10E4F000ADF8763016469142C0F29D80DFF830804C
:10E500002B465D46CDF828A082469B463FE000BFE3
:10E510001DBE00007D40010025180100CD990000BE
:10E52000259A00002DC00000C1BD00003D2901005A
:10E5300051770000BDF964305A1C141BADF87840C7
:10E54000ADF87C30069A9B1A0133B9F91020BDF959
:10E5500068100A449B1ACDF808B001950097002B6B
:10E56000ACBF53440AF10003BDF814201EA904985F
:10E57000C047BDF872300133ADF87230BDF8763067
:10E580000133ADF876300136099BB3424EDB089972
:10E590005046CC4B9847B9F812203244B9F81010C5
:10E5A000BDF868301944079B12B209B25046C64CF8
:10E5B000A0470746BDF87230ADF87A30BDF8763026
:10E5C000ADF87E30BDF96030ADF87830BDF8184058
:10E5D000013B2344ADF87C30CDF808B001950090A4
:10E5E0005346BDF814201EA90498C047BDF97E20EB
:10E5F000BDF962300A99B1F918100B449A4299DAC0
:10E60000BDF860302344ADF87830BDF864301B1B92
:10E61000ADF87C30CDF808B00195012300930023BC
:10E62000BDF814201EA90498C04783E75B46AB469B
:10E63000DDF828A01D46B9F91230BDF96660F61A5A
:10E640000E9AB61A09990A46B142A4BF013216467B
:10E6500033441BB2ADF87230ADF87630BDF96E3090
:10E660009E4200F38C80DFF864822B465D46CDF835
:10E6700024A0DDF82CA09B462DE0BDF964305A1C87
:10E68000141BADF87840ADF87C30069A9B1A013324
:10E69000B9F91020BDF968100A449B1ACDF808B0EA
:10E6A00001950097002BACBF53440AF10003BDF85D
:10E6B00014201EA90498C047BDF872300133ADF88C
:10E6C0007230BDF876300133ADF876300136BDF9E1
:10E6D0006E309E424EDC089950467A4B9847B9F806
:10E6E00012203244B9F81010BDF868301944079B65
:10E6F00012B209B25046744CA0470746BDF96030CB
:10E70000ADF87830BDF81840013B2344ADF87C30BB
:10E71000BDF87230ADF87A30BDF87630ADF87E30A5
:10E72000CDF808B0019500905346BDF814201EA9FD
:10E730000498C047BDF97E20BDF966300999B1F94A
:10E7400018105B1A9A4298DDBDF860302344ADF88A
:10E750007830BDF864301B1BADF87C30CDF808B0C4
:10E760000195012300930023BDF814201EA90498ED
:10E77000C04782E75B46AB46DDF824A01D46BDF8E6
:10E780003830BDF8622001321A44ADF87220BDF86D
:10E790006620013AD31AADF87630BDF96030ADF895
:10E7A0007030013BBAF818201344ADF8743002956C
:10E7B000CDF804B0012600960023BDF8148042462F
:10E7C0001CA9049F3846414CA047BDF96420931909
:10E7D000BAF818105B1AADF87030ADF874200295D5
:10E7E000CDF804B00096002342461CA93846A04745
:10E7F0000C98374CA0470D98A0470B98354B98477D
:10E80000FEF7B0BDBDF86030ADF87030BDF86430D3
:10E81000ADF87430BDF96A20B9F8123013441BB258
:10E82000ADF87230ADF876301446BDF96E309A42CC
:10E83000DEDCDFF89080244F244EDDF82CA02B4640
:10E840005D469B4608995046C047B9F812202244BD
:10E85000B9F81010BDF868301944079B12B209B21C
:10E860005046B847CDF808B0019500905346BDF822
:10E8700014201CA90498B047BDF872300133ADF8DC
:10E880007230BDF876300133ADF876300134BDF921
:10E890006E309C42D6DDABE70C980E4B984707FBD9
:10E8A00007F7002F3DF4ECAE0A980246411E00EB3C
:10E8B000470032F8023B9B0901F8013F9042F8D132
:10E8C000FDF7DEBEED2B01001DBE000051770000FC
:10E8D0006DBE000071250100079738460B4B984725
:10E8E0000C90002FD8DD01230B93FDF727BE0023EA
:10E8F000BAF90020069929A8054CA047002129A8AB
:10E90000044B98470446FFF71EB900BF3D2901009C
:10E910002DC00000C1BD0000F0B583B09DF80440DB
:10E920006FF304048DF80440BDF804406FF34A14FB
:10E93000ADF80440240A6FF3C7048DF805408668DB
:10E94000047804F01F04251FEDB2022D0ED9072C08
:10E9500028D0082C3BD0092C50D00A2C66D00B3C78
:10E96000E4B2032C98BFADF8043017E014460F460C
:10E970000546007800F01F00324B98472B68C3F320
:10E980008A2304FB0372C0F3C70000FB02F2B31832
:10E99000B25C8DF804205B788DF80530BDF804007A
:10E9A00003B0F0BD01F00703C3F107040368C3F32C
:10E9B0008A230733DB1002FB036606EBE1010B7AC7
:10E9C0000122A24013402341ADF80430E6E701F0F4
:10E9D00003046400C4F106040368C3F38A23033309
:10E9E0009B1002FB036606EBA1010B7C0322A240F5
:10E9F000134043FA04F4ADF80440CFE701F00104FA
:10EA0000A400C4F104040368C3F38A2301335B1038
:10EA100002FB036606EB610191F840300F22A24031
:10EA2000134043FA04F4ADF80440B7E70368C3F3B6
:10EA30008A23314402FB031191F80034ADF804300D
:10EA4000ACE700BF81960000F0B585B004460D46E6
:10EA500017468668037803F01F03052B0AD00B2B9B
:10EA600012D00C2B27D00D2B49D00E2B64D0FF20B9
:10EA700005B0F0BD0268C2F38A2207FB021505EB60
:10EA800045053544A878F3E701F00703C3F1070112
:10EA90000268C2F38A220732D210ED1007FB02622D
:10EAA000535D01228A4013400B4113F0FF0F0CBF4E
:10EAB000FF200020DCE700238DF8003055238DF87F
:10EAC0000130AA238DF80230FF238DF8033001F0C6
:10EAD00003035B00C3F106010268C2F38A2203321A
:10EAE0009210AD1007FB0262535D03228A4013406F
:10EAF0000B4104AA52FA83F313F8100CB8E7124B37
:10EB00000FCB0DF1100E0EE90F0005F001039B0075
:10EB1000C3F104012268C2F38A22013252106D103F
:10EB200007FB0262535D0F228A4013400B415EFADD
:10EB300083F313F8100C9BE70268C2F38A2207FBE9
:10EB40000262505C94E700BF0C5102002DE9F84FBF
:10EB50000446B0F908301B024362B0F90A301B02C8
:10EB60008362B0F90C00DFF8F48088FB0023C5173E
:10EB7000C5EBA3052DB26FF0090707FB05071FFAC8
:10EB800085FACAF1000000B2DFF8D490C847064603
:10EB90000135ADB2684200B2C8478346CAF15A0097
:10EBA00000B2C8478246C5F15A0528B2C847C7F126
:10EBB0000A0307FB0BFB03FB06B688FB062BF617C5
:10EBC000C6EBAB06E66207FB00F003FB0A0088FB1E
:10EBD0000038C017C0EBA8002063A07C1D4B9847ED
:10EBE00094F8343060F3000384F83430A07C1A4B7E
:10EBF000984794F8343060F3410384F83430A27CB1
:10EC0000131FDBB2022B94F8343094BF43F004039B
:10EC10006FF3820384F8343023682362237E03F089
:10EC20001F0362F304032376A369A28862F394238B
:10EC3000A3611B0CE28862F34F136383E2894FF4F4
:10EC4000803393FBF2F3E386FF23A375238AA38229
:10EC5000BDE8F88FB3960000C79600006766666649
:10EC6000A52201002DE9F04F87B003900491059291
:10EC7000BDF840400194DDF844B05E4F87FB03606F
:10EC8000DD17C5EBA0052DB205F101096FF00906EE
:10EC900006FB05362846DFF86081C04704460FFAB8
:10ECA00089F0C047824605F15A0000B2C0470546C8
:10ECB00009F15A0000B2C047C6F10A0306FB0AFA7E
:10ECC00003FB04A487FB04EAE417C4EBAA0406FBD5
:10ECD00000F003FB050587FB0537ED17C5EBA7071C
:10ECE000BBF900C0BBF90280CCF10003019D05FB1C
:10ECF00003F343F30F2303FB07FAC8F1000205FBFC
:10ED000002F242F30F2202FB04FE1FFA8CF6AAEB7A
:10ED10000E0B06EBEB3B0FFA8BFB03FB04F302FB42
:10ED200007F21FFA88F0991800EBE13109B202915D
:10ED30000499A1EB0C0C05FB0CFC4CF30F2C0CFB09
:10ED400007F9A9EB0E0E06EBEE3E0FFA8EFE0CFB5A
:10ED500004FC624400EBE23212B20599A1EB080810
:10ED600005FB08F848F30F2808FB04F4AAEB040598
:10ED700006EBE5352DB208FB07F73B4400EBE33328
:10ED80001BB2A9EB040406EBE43636B2BC4400EB3C
:10ED9000EC3000B25C46F345A8BF7446AC42A8BF55
:10EDA0002C46B442A8BF344603990F460C80DE457A
:10EDB000B8BFDE467545B8BF7546AE42B8BF2E46F1
:10EDC0008E8002990C469142A8BF14469C42A8BF6F
:10EDD0001C468442A8BF04467C809142B8BF1146BD
:10EDE0008B42B8BF0B469842B8BF1846F88007B0B0
:10EDF000BDE8F08F67666666A52201002DE9F04F39
:10EE000089B00446B0F93850EAB2B0F93A60F3B2CA
:10EE10006F2A74DCB0F93C104942C917803DEDB24D
:10EE20006F2B7EDCB4F93EB0CBF1000B4FEAEB7BED
:10EE3000803EF6B294F8149009F01F09B4F81480DB
:10EE4000C8F34518677DFF08A37D009394F834C08C
:10EE50001CF0040F7BD02368206C94F844E00EFB78
:10EE600001015A1813F801A08DF81CA052788DF8F2
:10EE70001D20B4F904200EFB02F20BFB02FB5844E8
:10EE80001A1813F800A08DF818A052788DF81920E0
:10EE900001EB0B0203EB020A13F802B08DF814B079
:10EEA0009AF801A08DF815A01CF0020F00F08180E7
:10EEB0000EF1FF3E734413F801B013F800A0985C04
:10EEC000C5F1FF0303FB0BF1009A05FB021103FBE5
:10EED00000F305FB0A33C3F30723C6F1FF02C1F3B6
:10EEE000072106FB01FE02FB03E21212A2750529AF
:10EEF00000F2DC80052B40F27D810026D9E0902ACB
:10EF00000CDDB0F93C100131B0F904209142ACBFE6
:10EF100000210121C5F17F05EDB281E7FF25002128
:10EF20007EE7902B0FDDB4F93EB00BF1010BB4F985
:10EF300006209345ACBF4FF0000B4FF0010BC6F11C
:10EF40007F06F6B276E7FF264FF0000B72E704F17A
:10EF5000180318468BB2A18F02931944238AB4F97F
:10EF60003E2009B20190DFF894A2D047ADF81C0012
:10EF70001FFA8BF1E28F03910A44238A12B2B4F98B
:10EF80003C10DDF804B05846D047ADF81800E28FC9
:10EF900003990A44A18F029B1944238A12B209B231
:10EFA0005846D047ADF8140094F8343013F0020FEF
:10EFB00052D1FF23A3752B46002B40F08B809DF888
:10EFC0001C9009F01F09BDF81C80C8F345189DF876
:10EFD0001D70FF08002D40F0AC809DF8145005F026
:10EFE0001F05BDF81430C3F345139DF81510C9086B
:10EFF000002E00F0E380FF2E00F0EE80C6F1FF024D
:10F0000002FB05F506FB095505EB052905EBC915BE
:10F01000ED0D207D65F30400207502FB03F306FB74
:10F02000083808EB082308EBC3184FEAD858A38A1E
:10F0300068F34A13A38202FB01F106FB071606EBF5
:10F04000062706EBC716F60D1B0A66F3C7036375A2
:10F05000012009B0BDE8F08FA18F029B1944B4F9DB
:10F060003E2009B2DDF804A05046634B9847834622
:10F07000E28F03990A4412B2B4F93C10CDF804A00F
:10F0800050465D4B98478246E28F03990A44A18F10
:10F09000029B194412B209B20198574B984794F851
:10F0A000343013F0020F7FF40BAF82E7052B98BFCB
:10F0B000FF26009B052B8CBF2B460023BBF1050FC1
:10F0C00098BFFF23BAF1050F98BF0025052898BF08
:10F0D000FF2571E7FF2B3FF47DAFC3F1FF019DF8E2
:10F0E0001D20D20803FB07F701FB027707EB07227D
:10F0F00007EBC217C7F3C457BDF81C20C2F3451273
:10F1000003FB08F801FB028808EB082208EBC21891
:10F11000C8F3C5589DF81C2002F01F0203FB09F933
:10F1200001FB029909EB092309EBC319C9F3C4597F
:10F1300050E7FF2D36D0C5F1FF009DF81910C90822
:10F140009DF81530DB0800FB03F305FB013101EBF3
:10F15000012301EBC311C1F3C451BDF81830C3F34F
:10F160004513BDF81420C2F3451200FB02F205FB63
:10F17000032303EB032203EBC213C3F3C5539DF830
:10F18000182002F01F029DF814E00EF01F0E00FB85
:10F190000EF005FB020505EB052205EBC215C5F3D4
:10F1A000C45525E79DF8185005F01F05BDF8183027
:10F1B000C3F345139DF81910C90819E7227D65F3BB
:10F1C00004022275A28A63F34A12A282120A61F330
:10F1D000C702627501203CE7237D69F304032375B0
:10F1E000A38A68F34A13A3821B0A67F3C7036375F4
:10F1F00001202EE700202CE749EA000019E9000071
:10F200002DE9F04F83B088465D4B1988E1B1074680
:10F210005C4B1E683346013989B2013101EBC101F3
:10F2200006EB810158481A6A8242A4BF02F1FF32FC
:10F230001A6224338B42F6D10024DFF88091DFF884
:10F2400080B1DFF83CA111E0504B0093504B4422B9
:10F2500050490220504CA047002525E0012827D026
:10F260000134A4B2BAF80030A3422AD904EBC40591
:10F2700006EB85056868C8470028EFD16B68BB427C
:10F28000EED128891FFA88F3984214BF002001208C
:10F290000028E5D02B6A6A691344B3F57A7F0EDD46
:10F2A0004FF47A732B6265B1284603B0BDE8F08F46
:10F2B00039466868D847B0FA80F04009E8E72B6221
:10F2C000F1E72F4B1A88012A37D906F12403023AB5
:10F2D00092B202EBC20206EB820248323546186A4D
:10F2E000296A8842B8BF1D4624339342F7D16B6820
:10F2F0002BB32846294B9847294B0093244B772260
:10F3000024490120244CA047264B9847044600235B
:10F310006B61424639462846234B9847C0B10023CB
:10F320002B626B69002BBFD12046204B9847686148
:10F330000028B9D101236B61B6E73546D7E71C4BEE
:10F340000093134B7A2213490120134CA047DBE7AB
:10F35000184B00930E4B83220E4902200E4CA047FF
:10F3600028460E4B984720212846134CA0472421BD
:10F370002846A0474FF000432B62002594E700BFCA
:10F38000582B0020586D0020020000809051020090
:10F3900034510200605102005D22010035FF00007F
:10F3A000B85102005910010049FE0000711001001F
:10F3B000EC51020020520200372B01006999000035
:10F3C000FBB401002DE9F047144B1F68144B1B8858
:10F3D0000BB306460024DFF84C90DFF84CA0DFF8B2
:10F3E00040800EE00BB12846D04720212846C84770
:10F3F00024212846C8470134A4B2B8F80030A342FB
:10F4000009D904EBC40507EB85056B68B342E9D065
:10F41000002EF0D1E6E7BDE8F08700BF586D002070
:10F42000582B0020372B010035FF00002DE9F0415B
:10F4300082B00446214B1B6833B10020204B984713
:10F440001E4B18681F4B984704EBC40080001E4BEE
:10F4500098471A4B18601D4B9847E8B1174B1B682B
:10F4600043B31B4B1C80A4B10024144F194E984683
:10F4700004EBC405AD00386820212844B047386843
:10F4800024212844B0470134A4B2B8F80030A34284
:10F49000EED802B0BDE8F0810F4B0093A8220F49CF
:10F4A00003200F4CA047054B1A6800230D480E4956
:10F4B0008847FEE70022064B1A80EAE7586D0020D5
:10F4C000C5F30000C5240100DD230100B1220000C6
:10F4D000582B0020372B01004851020060510200D8
:10F4E0005D220100D83F0200B922000030B587B08C
:10F4F0000C4615460846334B9847D8B92378C3F3D2
:10F500000403043BDBB20A2B59D82368C3F38A23D4
:10F510002A6863F394222A606388C3F34A136A88D3
:10F5200063F34F126A8022782B7862F304032B7006
:10F5300001200DE001280DD0022832D0224B00938B
:10F54000224B4FF49A7222490220224CA0470020FD
:10F5500007B030BD0222214604A81F4B984738B19E
:10F560002B781C3303F01F030A2B18D80120EFE778
:10F5700003AB0422294604A8184CA047044604A85B
:10F58000174B984714B9039B042BE9D0154B0093F4
:10F590000E4B40F221120E4902200E4CA0470020D3
:10F5A000D6E72B68012060F394232B601A0C60F3DC
:10F5B0004F126A800B2262F304032B70C8E700200D
:10F5C000C6E700BF699900006C5302004C5202006C
:10F5D000185302005D2201004D1D0100BD1C0100F9
:10F5E0008D1C01004853020038B5CC69A4B10D460A
:10F5F000206820B1094B98472068094B98476068FC
:10F6000008B1074B9847A06808B1054B98472046BA
:10F61000034B98470023EB6138BD00BF8D1C0100F0
:10F62000C52401002DE9F04385B005460C468B7AD0
:10F63000012B16D0002B40F0AA814B689B68002B51
:10F6400000F0A381087B00F01F00031FDBB2022B38
:10F6500000F2858063689B682361012005B0BDE8E6
:10F66000F0834868964B98479649974B98470028EF
:10F670002AD10222616802A8944B9847D8B9E3695D
:10F6800023B3E6690820924B98473060914B984726
:10F69000002840D03368002B4BD18F4B00938F4B09
:10F6A00040F25F128E4903208E4EB0472146284615
:10F6B0008D4B984708E08D4B0093884B4FF4A67212
:10F6C00087490220874CA0470020C7E70C20804BC9
:10F6D0009847E0617F4B984768B9804B009340F2B0
:10F6E00053127F4903207F4DA847E26900238048D9
:10F6F00080498847FEE7E06948B9774B0093774B2C
:10F7000040F2551276490320764CA047DCE70C21E5
:10F71000794B9847B5E7714B009340F25D12704901
:10F720000320704CA0473268002371487149884714
:10F73000FEE70DF1070203F1080112F8010F03F8CB
:10F74000010B8B42F9D1207B00F01F00031FDBB2BD
:10F75000022B04D8A37A002B3FF47CAF1FE1C31F18
:10F76000DBB2032B09D9A0F10B03DBB2032B00F2B0
:10F77000FD8000232361012070E7604B9847074616
:10F78000E369BBB1E6690220B840514B984770600D
:10F79000504B9847002837D1504B009340F29712B6
:10F7A0004F4903204F4CA0477268002350485149ED
:10F7B0008847FEE70C20464B9847E061454B984749
:10F7C00068B9464B00934FF4C67245490320454D36
:10F7D000A847E2690023464846498847FEE7E069B2
:10F7E00070B93D4B00933D4B4FF4C7723C49032029
:10F7F0003C4EB047214628463B4B984700202DE71A
:10F800000C213D4B9847BDE7012303FA07F7384623
:10F810002F4B9847B0602F4B9847002832D0736821
:10F82000002B3DD0B368002B3AD0A37A012B67D0D0
:10F8300063689A68002F00F095800023706800EBE1
:10F84000430C92F801E04FEA9E0E9578ED0811788E
:10F85000C90810F8138061F3040800F8138030F829
:10F8600013106EF34A1120F81310090A65F3C7014B
:10F870008CF80110D078B168C854013304329F422B
:10F88000DCD16FE0154B009340F29912144903202C
:10F89000144CA047B2680023154816498847FEE774
:10F8A0000D4B00930D4B40F29B120D4903200D4E62
:10F8B000B047214628460C4B98470020CEE600BFB3
:10F8C000211E010094530200FBB401004D1D0100F4
:10F8D000DD230100B1220000C45302006C5202007B
:10F8E000185302005D220100E9F500009853020060
:10F8F000D83F0200B9220000372B0100819600009A
:10F9000004213068284B984767B30025A946DFF8E3
:10F91000B0804B46042202A93068C047726802EBEF
:10F92000450E9DF8090080089DF80A10C9089DF849
:10F930000830DB0812F815C063F3040C02F815C098
:10F9400032F8153060F34A1322F815301B0A61F3C0
:10F95000C7038EF801309DF80B20B3685A55013566
:10F96000AF42D6D100232361012077E62146284605
:10F970000E4B98470E4B00930E4B40F2D3120E499C
:10F9800002200E4CA047002068E6002066E6087BB7
:10F9900000F01F00031FDBB2022B3FF6E0AE002396
:10F9A000236101205AE600BFF91C0100E9F50000BF
:10F9B000F05302006C520200185302005D22010055
:10F9C000BD1C01002DE9F04F8BB00D4614469A4640
:10F9D000BDF950600B7B03F01F031A1FD2B2022A3D
:10F9E00045D88B7A012B03D000200BB0BDE8F08FF7
:10F9F000D1F81C80087B00F01F009E4B98470746FB
:10FA0000E968C1F38A210AFB014100FB01F1C91039
:10FA10000431D8F80000984B9847D8B9C7F3C70706
:10FA200006FB07F60AAB002243F8102D3246159963
:10FA3000D8F80000914CA047069B9E4215D0904BF1
:10FA40000093904B40F235228F4902208F4CA04703
:10FA50000020CAE78E4B00938A4B40F22E228A493F
:10FA600002208A4CA0470020BFE70120BDE7A3F198
:10FA70000B02D2B2032A0FD9073BDBB2032B40F2B1
:10FA8000DF80844B0093844B4FF4FE727E4902204A
:10FA90007E4CA0470020A8E700228DF81020FF230D
:10FAA0008DF811308DF8142055228DF81520AA22DA
:10FAB0008DF816208DF81730784B0FCB0AAF07E979
:10FAC0000F002989002E0CDD080A159B721E92B2C8
:10FAD000013202EB42021A441970587003339A4201
:10FAE000FAD1287B00F01F00624B9847804601271F
:10FAF0008740013FBFB22B7B03F01F030B3B032B5F
:10FB000000F28380DFE803F0024C6176EB68C3F318
:10FB10008A23DA1013F0070F0CBF0FFA82FB02F1F1
:10FB2000010BE3100AFB0B3AE44304F007040DF168
:10FB30001009EB6903935846594B98470290AB7AEA
:10FB4000002B6BD16B689B689A44002E23DD159ABD
:10FB5000711E89B2013101EB41011144C8F1080065
:10FB600040B29AF8003007FA04F6334023412E7B66
:10FB700006F01F060E2EDBB218BF19F80330937083
:10FB8000A4EB080464B2002CBCBF04460AF1010ACD
:10FB900003328A42E5D10298424B9847012024E77C
:10FBA000EB68C3F38A239A1013F0030F0CBF0FFA0C
:10FBB00082FB02F1010BA3100AFB0B3AE44304F0B1
:10FBC000030464000DF11409B3E7EB68C3F38A235F
:10FBD0005A1013F0010F0CBF0FFA82FB02F1010B58
:10FBE00063100AFB0B3A14F0010F13D000240DF13F
:10FBF00018099EE7EB68C3F38A239AB20FFA83FBD6
:10FC00000AFB024A0024A14693E70024A246A34629
:10FC1000A1468EE704240DF118098AE70AF10401D0
:10FC2000039B1868144B984700235A46DDF808B028
:10FC3000594603980068DFF844A0D047DA4684E7C5
:10FC4000087B00F01F000B4B984781464FF00108DE
:10FC500008FA00F808F1FF381FFA88F82B7B03F048
:10FC60001F03073B032B00F2A580DFE803F01D68AC
:10FC70007E9600BF81960000F91C0100BD1C0100AA
:10FC8000405402008C520200185302005D22010011
:10FC90001C54020064540200C4520200B452020018
:10FCA0003D29010071250100EB68C3F38A234FEA67
:10FCB000E30B13F0070F0CBF0FFA8BFB0BF1010BDB
:10FCC000E3100AFB0B3A0AF1080AE44304F00704C4
:10FCD000EF695846414B98470290AB7A002B6ED1A2
:10FCE0006B689B689A44002E24DD159A711E89B2B8
:10FCF000013101EB41011144C9F108056DB29AF8D7
:10FD0000003008FA04F003402341DBB2786830F891
:10FD100013001070000A5070B868C35C9370A4EBB5
:10FD2000090464B2002CBCBF2C460AF1010A03325C
:10FD30008A42E4D102982A4B9847012055E6EB68A5
:10FD4000C3F38A234FEAA30B13F0030F0CBF0FFA80
:10FD50008BFB0BF1010BA3100AFB0B3A0AF1100A03
:10FD6000E44304F003046400B2E7EB68C3F38A23BE
:10FD70004FEA630B13F0010F0CBF0FFA8BFB0BF173
:10FD8000010B63100AFB0B3A0AF1400A04F001046C
:10FD9000002C0CBF042400249AE7EB68C3F38A2BE1
:10FDA0001FFA8BF30FFA8BFB0AFB034A0AF5806AF2
:10FDB00000248DE74FF0000A5446D34688E70AF145
:10FDC00004013868074B984700235A46DDF808A01D
:10FDD00051463868044DA84785E700BF3D2901001A
:10FDE00071250100F91C0100BD1C01002DE9F0473F
:10FDF00081460E460B786FF347130B700F48104B7C
:10FE00009847C8B104464FF0000ADFF830800D4F24
:10FE100005E0554621464046B847044648B12368A8
:10FE2000002BF6D032464946204698470546012821
:10FE3000F0D12846BDE8F0870025FAE7A46C002041
:10FE4000A91F0100BD1F01002DE9F0478246884629
:10FE500002810846264B98478AF80A000023CAF810
:10FE60001C3001280DD0CAF804802248224B984744
:10FE70000446002836D000250AF10C091D4F1F4EFC
:10FE800010E040461E4B984701301E4B9847CAF879
:10FE9000040041461C4B9847E7E721463846B047E7
:10FEA0000446D8B12368002BF7D06268002AF4D04A
:10FEB0004A4641462046984705460128EDD1002391
:10FEC000CAF81830CAF81030CAF8004063685146C2
:10FED0002046984705460128DFD100E01DB128469D
:10FEE000BDE8F087002520215046084B9847F6E7EB
:10FEF00069990000A46C0020A91F0100BD1F01002A
:10FF00001FB50100DD2301000FB50100372B0100F3
:10FF100070B582B00668B46854B11D4613460A46EF
:10FF200001460698019000953046A04702B070BD8A
:10FF30000020FBE7036883B110B50446DA6812B10C
:10FF4000014618469047A37A012B00D010BD606887
:10FF5000024B984700236360F8E77047C52401000F
:10FF600030B583B00D480E4B984704460D4B98476B
:10FF700038B11CB1102120460B4B9847204603B0E6
:10FF800030BD0A4B0093C92209490320094DA847F7
:10FF900022460023084809498847FEE7A46C002050
:10FFA000111F0100B1220000372B0100E8520200AE
:10FFB000185302005D220100D83F0200B922000060
:10FFC00010B582B010211448144B9847144B984731
:10FFD00048B1144A0260144A4260144A8260144ACA
:10FFE000C26002B010BD134B0093134B472213495C
:10FFF0000220134CA0470020124B98470028F0D154
:020000021000EC
:100000000D4B009348220D490320A04700220023F6
:100010000D480E498847FEE7A46C0020F91E010038
:1000200061FF0000EDF4000025F60000C5F90000B6
:10003000E9F50000A054020000530200185302002A
:100040005D220100B1220000D83F0200B922000069
:1000500008B54368984708BD10B50468A04710BDAF
:1000600010B584B013460A4601A9044CA04718B144
:10007000BDF8040004B010BD0020FBE759000100EA
:1000800003780A78934211BF981A40784B78C01AC7
:10009000704703880A88934211BF981A40884B889A
:1000A000C01A704700880B88C01A70470B46002999
:1000B0006CD0F0B585B00469A269914215D0678A09
:1000C000C7F30907002F5DD0A16808681A1A0392C8
:1000D000888882420BD800261D468B7CE3B9C888ED
:1000E0001044A561E06105B0F0BDE069FBE70025C3
:1000F0000135ADB2BD4245DA05EB850082001646FA
:1001000001EB020E51F820209A1A0392BEF8040067
:100110008242EDD87146DFE7012B05D0022B08D0D3
:10012000032B18D00020DCE7CB689B5CC888184400
:10013000D7E70A8A8968164B0093022303A8154F54
:10014000B8470346D0B1A2681644B068181AF388BD
:1001500003EB5000C5E70A8A89680D4B0093022320
:1001600003A80C4FB84758B1A2681644B268831A66
:100170005B08F268D35CF0881844B2E70020B0E76F
:100180000020AEE7A3610020E061ACE708467047BD
:10019000A5000100854101002DE9F04F9FB009291C
:1001A000056908BF2021A04B9847002800F0EA8489
:1001B00080466F6807EBC0062B7D13F0030F0BD151
:1001C000002E00F0E28457F83030C3F313032868A0
:1001D00018441FB0BDE8F08F3379747904FB03F441
:1001E000002C00F0D584EB7CC3F38303013B032B8D
:1001F00005D8DFE803F00275787B0734E4088B4B01
:1002000018688B4B9847844211D9DFF82092214619
:10021000D9F80000874B9847C9F80000864B9847EB
:10022000002866D0814B1B68002B00F0B48457F87F
:100230003810C1F313012B6819447C4BD3F800909C
:1002400033790C939B461AB217461892727915921D
:10025000EA7CC2F38302D3B20F93032B14BF184678
:1002600004200890714B59601A7200225A72DA60A9
:100270001A745A745846714CA04716905846A047B5
:100280001790002F00F05182684B197C03915C7C21
:100290005F68DD6893F808A0012202FA0AF2511E95
:1002A000D046CAF108060A96CAF11006099693F8D4
:1002B00009C0169800F1FF3E0BF1FF339BB20D937E
:1002C00000EB030B76460023059307931A460AF1C9
:1002D000FF3A01230493CBB20B930692614634E0BC
:1002E0000334A4088BE70134640888E70134640808
:1002F00085E7534B0093722252490320524CA0478A
:10030000D9F800200023514851498847FEE70320CF
:10031000EB0805F0070202EB080CBCF1070F35D81B
:1003200017F803C00A9B9A1A4CFA02F3034015B15E
:10033000039A934238D045440393012204980690CF
:1003400006F8013F5E4500F04E81A1BBBAF1070FF0
:1003500018D801A353F82AF0890301000F03010004
:10036000790301007D03010085030100850301007D
:1003700085030100810301000720C9E70F20C7E7BB
:10038000FF20C5E70B98C3E70120C1E717F803C0BA
:100390003B445B7803EB0C231FFA83FC099B9A1AFE
:1003A0004CFA02F30340C2E7012205920024049AAA
:1003B00007921146BFE7012904D0022900F0CD8041
:1003C0000023BDE7EB0805F0070202F1010CBCF1C8
:1003D000070F13D8FB5CD2430832134103F001032B
:1003E0000134E4B26A1CB3B9BAF1070F00F2A58078
:1003F000DFE80AF0A5849D9FA3A3A3A117F803C07B
:100400003B445B7803EB0C239BB2D2431032134185
:1004100003F00103E4E70B2C1CD01546039B0122DB
:100420000592049A8CE700BFAD0001005C2B002010
:100430005125010099280100B12200003D29010049
:10044000C4540200E05402005D220100D83F0200C3
:10045000B9220000D30802F00702911D072913D822
:10046000FC5CC2F1020244FA02F202F03F040735DA
:10047000002C40F0AD80BAF1070F26D8DFE80AF073
:1004800027101F2125252523F95C3B445C7804EBCC
:100490000124A4B2C2F10A02144104F03F04E6E7C9
:1004A0000320EA0805F0070303EB0801072910D829
:1004B000BA5C0A99CB1A42FA03F3034014E007200E
:1004C000EFE70F20EDE7FF20EBE70B98E9E70120CE
:1004D000E7E7B95C3A44527802EB012292B20999FB
:1004E000CB1A42FA03F303404544039301220592D9
:1004F0000498024607900021069021E70320D108C6
:1005000002F0070303EB0805072D1AD8795C0A9D52
:10051000EB1A41FA03F3034002EB080503930122AF
:1005200005920498024607900021069008E70720EC
:10053000E5E70F20E3E7FF20E1E70B98DFE7012085
:10054000DDE77D5C3944497801EB052189B2099DDD
:10055000EB1A41FA03F30340DEE7013C14F0FF0419
:100560003DD1BAF1070F23D8DFE80AF024041C1E9E
:10057000222222200320EA0805F0070303EB0801EA
:10058000072919D8BA5C0A99CB1A42FA03F3034037
:1005900045440393012205920498024607900021E6
:1005A0000690CDE60720E6E70F20E4E7FF20E2E72C
:1005B0000B98E0E70120DEE7B95C3A44527802EBA1
:1005C000012292B20999CB1A42FA03F30340DFE702
:1005D000039B01220592049A07920221B0E6039B35
:1005E00001200590ACE606988C46C8B90AB19F4B2D
:1005F000DD60079B13B19D4B83F809C0059B0BB1D0
:100600009A4B5C7400200F9B039304274FF00F0C50
:100610004FF00D084FF00B0A4FF0090B049728E03C
:10062000924B9DF80C101974E0E707293DD8DFE8DC
:1006300001F004272A2D303336393D46002100F0E1
:100640000702C2F10802521BC0F3CF044FF0FF3380
:10065000AB4063F0FF03934019F804502B4001FABC
:1006600002F2134309F80430089A13461044B645C1
:100670001DD01EF8011F0F9B032BD6D0039DDEE774
:100680003D460221DBE73D460499D8E73D46062179
:10069000D5E73D465946D2E73D465146CFE73D4670
:1006A0004146CCE73D466146C9E73D46C7E70D9A5E
:1006B00002FB03330E93159B012B40F355826B4BCA
:1006C000D3F804801A7A10461992012202FA00F136
:1006D0000139C9B21B9101468246587C0790C1F18D
:1006E00008010B91CAF110010D91197C0391D3F807
:1006F0000CC093F809B0089912910C9B013B9BB276
:1007000001FB03F11A9100210A910C9106910891C5
:100710001092179AD3181C93012304930F9A0992ED
:1007200004221D9205936646F5E100230E93C2E76D
:100730004FF003090CE04FF0070909E04FF00F09F3
:1007400006E0E14604E0DDF8449001E0DDF81090B9
:10075000F30806F0070202EB0A0BBBF1070F31D8D2
:1007600018F803300B9DAA1A43FA02F202EA0909AB
:100770005FFA89F916B1039B4B4533D05644CDF847
:100780000C90049B0693059B089304F8019FA042DC
:1007900000F05D8169BB079B1A46072AD3D801A3E5
:1007A00053F822F04D07010031070100370701001F
:1007B0003D07010047070100470701004707010007
:1007C0004307010018F803B043445B7803EB0B23A5
:1007D0009BB20D9DAA1A43FA02F202EA09025FFADD
:1007E00082F9C7E7049B0A937746059B0C93194649
:1007F000C4E7012904D0022900F0D780F146C4E7FC
:10080000F30806F0070202F10109B9F1070F15D844
:1008100018F80330D2430832134103F001037A1C65
:10082000D7B2721CBBB9079B1946072900F28E800C
:10083000DFE801F08E8486888C8C8C8A18F803900F
:1008400043445B7803EB09239BB2D243103213413C
:1008500003F00103E3E70B2F0AD01646DDF80C90F6
:10086000049B0A93059B06938FE700BF5C2B002037
:10087000D30802F00702911D072915D818F8033094
:10088000C2F1020243FA02F202F03F070736002FDC
:1008900040F0CF80079B1A46072A39D8DFE802F0DC
:1008A0003B1230333838383618F8031043445B783D
:1008B00003EB01239BB2C2F10A0243FA02F202F0F7
:1008C0003F07E3E74FF00309F30806F0070202EBE6
:1008D0000A01072922D818F803300B998A1A43FA1B
:1008E00002F202EA09025FFA82F95644CDF80C904E
:1008F000049B0A93059B0C9371460693089344E767
:100900004FF00709E0E74FF00F09DDE7E146DBE7CD
:10091000DDF84490D8E7DDF81090D5E718F803101B
:1009200043445B7803EB01239BB20D998A1A43FA87
:1009300002F202EA09025FFA82F9D6E7032608E02A
:10094000072606E00F2604E0664602E0119E00E05E
:10095000049ED30802F0070101EB0A09B9F1070F61
:1009600014D818F803300B9D691A43FA01F131408D
:100970005FFA81F902EB0A06CDF80C90049B0A930A
:10098000059B0C93714606930893FEE618F80390B6
:1009900043445B7803EB09239BB20D9D691A43FA2C
:1009A00001F131405FFA81F9E4E77B1E13F0FF07A4
:1009B00048D1079B1A46072A0DD8DFE802F00E043B
:1009C00006080C0C0C0A032108E0072106E00F21A1
:1009D00004E0614602E0119900E00499F30806F092
:1009E000070202EB0A09B9F1070F13D818F8033010
:1009F0000B9DAA1A43FA02F20A405FFA82F95644A2
:100A0000CDF80C90049B0A93059B0C9371460693BA
:100A10000893BAE618F8039043445B7803EB092384
:100A20009BB20D9DAA1A43FA02F20A405FFA82F9BC
:100A3000E5E7DDF80C90049B0A93059B0C930221DB
:100A40000693A2E6DDF80C90049B0A939DE6DDF880
:100A50004C900797149F169B03F1FF3E0E9DDDF807
:100A60003CC011961391DDF848B021E0072A40D828
:100A7000DFE802F0042A2D303336393C042300220B
:100A800005F00701C1F10801C91AC5F3CF0001261D
:100A900006FA03F35B4263F0FF038B4019F8006032
:100AA00033408A40134309F800305D44BC4222D0F1
:100AB00017F8012F9EF801305A400EF8012FBCF1B3
:100AC000030FD3D0099BDBE704230222D8E70423DA
:100AD0001D9AD5E704230622D2E704230922CFE793
:100AE00004230B22CCE704230D22C9E704230F22A1
:100AF000C6E70423C4E7119EDDF84CB01A9B129A96
:100B000013440E9A1A440E92109B01331BB2109399
:100B1000159A9A4215D0189B002BF5D0179B5F1E93
:100B20003C464FF0000E199B5D1E1B9B11934FF02E
:100B3000FF0CCDF84C9059461497079F07951C98C9
:100B400028E6B446089BC3B9069B13B1134BC3F800
:100B50000CC00C9B13B1114B83F809B00A9B1BB15D
:100B60000E4B9DF81C205A7416980D4CA0471798F0
:100B7000A0470A4B1868FFF72CBB084B9DF80C20C8
:100B80001A74E1E70020FFF724BB0020FFF721BB28
:100B90000020FFF71EBB0020FFF71BBB5C2B0020D3
:100BA000712501002DE9F04784B007460C469946AF
:100BB000092A06BF01252022002506691146494B56
:100BC00098478046002800F08680F368002B7CD090
:100BD00049463846434B9847034618BB0023706884
:100BE00000EBC800328A03FB02F31B114288C2F3F8
:100BF0000B1205B15200083313441B0923804379BB
:100C0000A3800279628090F90630E38090F9073082
:100C10002381F37CC3F38303A372002D60D05200C1
:100C2000628059E03A69D17C11F0400F3CD1D7681D
:100C3000FA7A12F0030203D0012A1BD00023CEE778
:100C4000D7F8009008EB002304A820F8043DBA6808
:100C5000254B0093022322F07F424946DFF890A003
:100C6000D04728B1A0EB09035B087A68D356B6E7F2
:100C70000023B4E7D7F8009008EB002304A840F85D
:100C8000043DBA68194B0093042322F07F42494681
:100C9000DFF85CA0D04728B1A0EB09031B097A68F4
:100CA000D3569CE700239AE7D1684A6812F80820D7
:100CB0006AB18868C35C63B1013A487B09680B4438
:100CC00000FB023212F9013C89E7002387E7002389
:100CD00085E7002383E70025284604B0BDE8F087B8
:100CE0000125F9E7AD00010081000100930001003A
:100CF0008541010008B5044B186820B1034B9847A3
:100D00000022014B1A6008BD5C2B0020C5240100A5
:100D100010B504462C21154B98470023E3604FF48F
:100D2000F07222804FF4887262806360227A63F3EB
:100D30004102227294F8282063F3040284F82820E8
:100D4000228D42F4FC622285120A63F3C70284F802
:100D500029202289822161F38B02228142F0010243
:100D6000227223626362636110BD00BF372B0100F2
:100D7000F8B504460D4617461E462421034B9847F6
:100D800025606760A560E660F8BD00BF372B0100F5
:100D9000F0B583B005463F483F4B984704460028CE
:100DA00054D04FF4B8713D4B98472C222946204629
:100DB0003B4B98474C2104F130003A4B98470023B5
:100DC000C4F86C31384B1B68002B50D0364B1F6871
:100DD0001C60234603221E213448354DA847E0629B
:100DE000344B9847002845D0E36A002B4FD0B4F825
:100DF00068316FF30903A4F868310025C4F86C5119
:100E0000294628462C4EB047E06329462846B0477D
:100E1000206429462846B04760642946206C274E46
:100E2000B0472946606CB0472946206C244EB04735
:100E30002946606CB047E06B224B98471A4B1F6005
:100E4000E06A214B9847204603B0F0BD194B984704
:100E50000028F8D11D4B00937C221D4903201D4C16
:100E6000A047002200231C481C498847FEE70E4B80
:100E70001C60ABE7154B00938D2215490320154DDF
:100E8000A847E26A0023144814498847FEE7002473
:100E9000D9E700BF986C0020111F0100372B01001B
:100EA00055260100F91E0100702B0020755F00001F
:100EB000E5390100B1220000253E00009D3B000005
:100EC000A129000021330000553A0100BC91020025
:100ED000D49102005D220100D83F0200B922000037
:100EE000014B1868704700BF702B0020034640B1CB
:100EF0001A7A12F0020F0CBFB3F90000B3F9020026
:100F00007047034B1B68002BF2D14FF4F070704711
:100F1000702B0020034640B11A7A12F0020F0CBF6A
:100F2000B3F90200B3F900007047034B1B68002BB4
:100F3000F2D14FF488707047702B0020034618B12F
:100F40001889C0F389007047024B1B68002BF7D14A
:100F500082207047702B002038B50546A0B1284686
:100F60000F4B9847044628460E4B984704EB8404E1
:100F70006400B4FBF0F01D280DD931280DD94628A6
:100F800034BF0220032038BD074B1D684FF4F074B6
:100F9000002DE8D0E3E7002038BD012038BD00BFB8
:100FA000ED0E01003D0F0100702B00204268002370
:100FB00093614268D361704708B520B10146044887
:100FC000044B984708BD0248034B984708BD00BF33
:100FD000986C0020BD1F0100A91F010040687047E8
:100FE00043681A6822B15868003018BF0120704762
:100FF0000020704710B50446084B9847034658B187
:10100000B4F90020B4F9023003FB02F36268D2683D
:10101000934214BF00230123184610BDE10F0100C5
:1010200008B520B101460448044B984708BD024862
:10103000034B984708BD00BF8C6C0020BD1F01000A
:10104000A91F0100034B00221A705A68104458600F
:10105000704700BF742B0020044B4FF00101197042
:101060001A78002AFBD0014B58687047742B002077
:1010700010B50446014B9847001B10BD59100100E4
:101080000A6A486A82421ABF800290FBF2F04FF46B
:1010900080608A69CB699B1A00FB03F002EBA020F9
:1010A00000B2704708B50122084B1A700848094B76
:1010B000984728B10421054B5868074B984708BD4D
:1010C0000021024B5868044B984708BD7C2B002038
:1010D0005C6D0020A91F0100593901002DE9F04382
:1010E00091B06348634B984768B10146604D624CCC
:1010F00091F83C306FF3410381F83C302846A0471B
:1011000001460028F4D15D4B98685D4B98478046B6
:101110005748584B98470446002800F08980574D9F
:101120004FF00007524EDFF84C911CE013EB080320
:1011300000F18580A268002A00F088802046904750
:101140001EE0214604F110004E4B984728E0626AE9
:10115000236A9A422BDA2B78002B71D03046C8478D
:101160000446002C64D02F7094F83C3013F0020F2A
:1011700066D143F0020384F83C30636A002BD5DD6E
:10118000636A43446362002BE5DB226A9A42B8BF7C
:1011900062622369002BD4D0214604F110009847E5
:1011A0006368002BD3D001B220689847CFE794F84A
:1011B0003C3013F0010308D1A28E002A48D04FF62C
:1011C000FF718A424BD0013AA286A28ECAB1226B2D
:1011D00052426262E26A002ABDD0002B3BD083F00B
:1011E000010394F83C1063F3000184F83C10A369F8
:1011F000E069A061E36111F0010F08BFA26B2262F8
:10120000A9E7E26A02B133B34022214668461E4B89
:101210009847214630461D4B984720461C4B98471F
:101220001C4B9847039B002B95D06846984792E744
:10123000194B9847114B986011B0BDE8F083636279
:10124000214630460C4B984704468AE763629CE788
:10125000E26A002AD8D0A16A49426162BFE7226BE4
:1012600052426262E26A002A3FF475AFF3E700BFC0
:101270005C6D0020A91F0100BD1F01007C2B002018
:101280007110010081100100552601009520010018
:10129000C5240100A51001005910010038B54021F6
:1012A00009480A4B98470A4B98470A4CA06000230C
:1012B00004221E210848094DA8476060084B984742
:1012C0000023237038BD00BF5C6D0020F91E0100B3
:1012D000591001007C2B0020DD100100E5390100D0
:1012E000A510010010B5044640210D4B98474FF45E
:1012F000FA7323620023A3616423E361094B1A7824
:1013000022745A7862749A78A274DB78E3740123A9
:10131000A38694F8363043F0010384F8363010BDCC
:10132000372B0100009202002DE9F84F074689464D
:101330001548164B984710B304464FF0000ADFF8E3
:101340004880134EDFF854B00BE021464046D847A2
:101350002046104B9847104B98474FF0010A2C46F7
:101360007DB121464046B04705462368BB42F6D1D1
:1013700063684B45E9D0B9F1000FF0D1E5E74FF0D4
:10138000000A5046BDE8F88F5C6D0020A91F0100DF
:10139000BD1F0100C5240100A5100100952001001A
:1013A00030B583B00546416811B100681B4B9847C2
:1013B0001B481C4B9847F0B919481B4B98470446EB
:1013C0001A4B9847E8B1A4B12B6AAB634022294677
:1013D0002046174B984794F8363013F0010F06D08B
:1013E000636823B1206810B1B4F918109847114B05
:1013F000984703B030BD104B984701380F4B9860A9
:10140000DAE70F4B00936A220E4903200E4DA847DE
:10141000224600230D480E498847FEE729130100A4
:101420005C6D002045220100111F0100B122000067
:1014300055260100A5100100591001007C2B002049
:1014400008920200189202005D220100D83F0200BB
:10145000B9220000F8B504460F460A480A4B9847DF
:10146000014660B1074E094D03E03046A8470146EA
:1014700028B10B68A342F8D14B68BB42F5D10846AE
:10148000F8BD00BF5C6D0020A91F0100BD1F010059
:10149000891A0029B8BF49424FF47A7202FB01F25F
:1014A00092FBF0F04FF6FF72904228BF10460028E2
:1014B00008BF012080B2704730B4B0F90050B0F9D5
:1014C00004305B1B03EBD3735B109CB20A88521B86
:1014D000121B49884088081A001B13FB03F310FBFA
:1014E00000F012FB02029342B4BF0020012030BC86
:1014F0007047013943881944C1807047B0F904200E
:10150000B0F90030D21AB0F90630B0F90200181A5A
:10151000013002FB0000704770B4B2F90050B1F91D
:1015200000309D42B8BF1D460580B2F90230B1F9C6
:101530000240A342B8BF23464380B2F90440B1F948
:101540000460B442A8BF34468480B2F90620B1F9E1
:1015500006108A42A8BF0A46C280A54205DC934213
:10156000CCBF0020012070BC70470020FBE710B406
:10157000B2F90030B1F90040A342A8BF234603806E
:10158000B2F90230B1F90240A342A8BF234643801A
:10159000B2F90430B1F90440A342B8BF23468380B6
:1015A000B2F90630B1F906209342B8BF1346C380A2
:1015B0005DF8044B704700002DE9F04F85B0B1F99C
:1015C0000050B0F900E07545C0F29D80B0F904808C
:1015D000454500F39C80B1F90230B0F902A05345B3
:1015E000C0F29780B0F906000190834200F3938027
:1015F000002A40F392808C461FFA88F91FFA8EF673
:1016000087B21FFA8AF5ADF808E009F101039B1BC8
:101610001BB203EBD3747B1C5B1B1BB203EBD371BC
:1016200064104B10A342A8BF23469342A8BF1346A1
:101630009CB22644B6B2ADF80C60ADF80AA02544C1
:10164000ADB20FFA85FBADF80EB00022CDF800C0A8
:10165000614602A8FFF7B0FF50B12644ADF80C6018
:101660002C44ADF80E40009902A82E4B98474BE051
:101670003F1BBFB2ADF80A70BDF80430ADF80E30B4
:101680000022009902A8FFF797FF50B12644ADF859
:101690000C603C1BADF80A40009902A8214B98470A
:1016A00032E0A9EB04091FFA89F9ADF80890ADF80A
:1016B0000C800022009E314602A8FFF77DFF58B142
:1016C000A9EB0409ADF808903C1BADF80A4031467F
:1016D00002A8144B984717E0ADF80AA0ADF80EB079
:1016E0000022009E314602A8FFF766FFB8B1A9EBC1
:1016F0000409ADF808902C44ADF80E40314602A81C
:10170000084B984700E0002005B0BDE8F08F0020AE
:10171000FAE70020F8E70020F6E70120F4E70120CF
:10172000F2E700BFB9140100B0F90020B1F90430AC
:101730009A4214DCB0F90420B1F900309A4210DB6F
:10174000B0F90220B1F906309A420CDCB0F906007B
:10175000B1F902309842B4BF002001207047002048
:101760007047002070470020704700002DE9F041CD
:1017700082B0B0F90050B1F90030AB4214DCB0F9DE
:101780000240B1F902309C4214DBB0F90440B1F9D7
:1017900004309C4210DCB0F90630B1F90640A34297
:1017A000CCBF0023012300E000233AB9184602B061
:1017B000BDE8F0810023F8E70023F6E717460C4662
:1017C0000646ADF804504388ADF8063001A920461E
:1017D000134B984703460028E8D0B6F9048002A9C5
:1017E00021F8048D3A4620460D4B984703460028C1
:1017F000DCD0ADF80450F388ADF806303A4601A9C4
:101800002046074B984703460028CFD002A921F86D
:10181000048D3A462046024B98470346C6E700BF70
:10182000B915010030B4142A3AD8DFE812F01500D7
:10183000430047005C00670072008D009E00B3000B
:10184000CE00D600EE00FC0004011C012A0132018A
:101850004A01580160017801828801320488121B14
:1018600012B202EBD2748A8801320D88521B12B276
:1018700002EBD2725210C2EB64021A80C2880132AB
:101880004488121B12B202EBD274CA880132498812
:10189000521A12B202EBD2725210C2EB64025A8098
:1018A0001A8801880A441A805A8841880A445A8052
:1018B00030BC704700221A805A80F1E782880132DA
:1018C0000488121B12B202EBD2748A880132098892
:1018D000521A12B202EBD2725210C2EB64021A8098
:1018E00000225A80DCE782888C88121B0488121B35
:1018F00009880A441A8000225A80D1E700221A80FF
:10190000C288CC88121B4488121B49880A445A801A
:10191000C6E7828801320488121B12B202EBD2742D
:101920008A8801320D88521B12B202EBD272521019
:10193000C2EB64021A80C288CC88121B4488121B36
:1019400049880A445A80ABE782888C88121B048835
:10195000121B0C8822441A80C288CC88121B44882F
:10196000121B49880A445A809AE700221A80C288CA
:1019700001324488121B12B202EBD274CA880132BF
:101980004988521A12B202EBD2725210C2EB6402B0
:101990005A8085E782888C88121B0488121B0C8869
:1019A00022441A80C28801324488121B12B202EB10
:1019B000D274CA8801324988521A12B202EBD2722A
:1019C0005210C2EB64025A806AE700221A80CA8869
:1019D0004988521AD2435A8062E7828801320488C9
:1019E000121B12B202EBD2748A8801320D88521B8C
:1019F00012B202EBD2725210C2EB64021A80CA8891
:101A00004988521AD2435A804AE782888C88121B2E
:101A10000488121B0C8822441A80CA884988521AEA
:101A2000D2435A803CE700221A80C28801324188A2
:101A3000521A5A8034E7828801320488121B12B28B
:101A400002EBD2748A8801320988521A12B202EB70
:101A5000D2725210C2EB64021A80C28801324188ED
:101A6000521A5A801CE782888C88121B0488121B29
:101A700009880A441A80C28801324188521A5A8061
:101A80000EE78A880988521AD2431A8000225A80A7
:101A900006E78A880C88121BD2431A80C28801325A
:101AA0004488121B12B202EBD274CA8801324988F0
:101AB000521A12B202EBD2725210C2EB64025A8076
:101AC000EEE68A880C88121BD2431A80C288CC8822
:101AD000121B4488121B49880A445A80E0E6828817
:101AE00001320188521A1A8000225A80D8E6828870
:101AF00001320488121B1A80C28801324488121BEA
:101B000012B202EBD274CA8801324988521A12B258
:101B100002EBD2725210C2EB64025A80C0E6828895
:101B200001320488121B1A80C288CC88121B448898
:101B3000121B49880A445A80B2E630B48DB210F0C4
:101B4000030F1CBF20F8021B02F1FF3205EB054119
:101B5000102A21D900F12003144643F8201C43F831
:101B60001C1C43F8181C43F8141C43F8101C43F8C1
:101B70000C1C43F8081C43F8041C103C2033102CA8
:101B8000EBD8A2F111031B09591C103AC3EB0373E4
:101B900002EB031200EB41101AB120F8025B013A8C
:101BA000FBD130BC704730B4C1EB4115C1F1FF042B
:101BB000C0F3C42304FB035303EB032203EBC21360
:101BC000C3F3C452C0F34513C1EB811104FB0311ED
:101BD00001EB012301EBC311C1F3C55100F01F005C
:101BE00004FB005000EB002300EBC310C30D4FF0CB
:101BF000000063F3040061F34A1062F3CF2030BCAD
:101C0000704710B4C1F1FF01C0F3C42301FB03F31B
